:040000050000DA51CC
:020000040000FA
:1000000018430020B580000001CA011001CA011088
:1000100001CA011001CA011001CA011001CA011070
:1000200001CA011001CA011001CA011001CA011060
:0C00300001CA011001CA01103FCA0110F2
:100100003C0000000000000000000000340100007E
:1001100000000000000000000100000000000000DE
:1001200000000000000000000000000001000000CE
:100130000000000008000000000000003400000083
:100140000000000000000000680100000000000046
:10015000000000000100000000000000010000009D
:100160000000000000000000080000000000000087
:1001700030000000000000000000000098010000B6
:10018000040000000000000001000000FFFFFFFF6E
:10019000FF00000001000000080000000000000057
:1001A0002C0000000000000000000000C40100005E
:1001B000040000000000000001000000FFFFFFFF3E
:1001C000FFFFFFFF080000000000000034050000F2
:1001D000E401000099A1011095A70110A5C201102A
:1001E00009B2011045B80110000000000000000035
:1001F0002F000000280000000000000000000000A8
:10020000140200000000000000000000FFFFFFFFDC
:1002100000000000080000000000000030050000A1
:100220003002000069C201106DC101101FC201102F
:1002300095BA011000000000000000002D00000031
:10024000300500005402000075C20110A9B601106B
:100250009DBF011049B60110000000000000000021
:100260002E0000002400000000000000000000003C
:1002700080020000000000000000000000000000FC
:100280000800000000000000240000000000000042
:1002900000000000A40200000000000000000000B8
:1002A0000000000008000000000000002400000022
:1002B0000000000000000000C80200000000000074
:1002C0000100000000000000080000000000000025
:1002D00000000000FC0600200400000000000000F8
:1002E000000000002000000070010000300000004D
:1002F0001C0200001C070020040000000000000099
:10030000000000000C000000300400001800000095
:10031000400200002407002004000000000000004C
:100320000000000024000000480400001800000045
:10033000000000006407002004000000000000002E
:100340000000000010000000A00100002C000000D0
:10035000CC0100006C070020040000000000000039
:1003600000000000200000006402000024000000E3
:10037000FFFFFFFF8C0700200400000000000000CA
:100380000000000028000000880200002400000097
:10039000FFFFFFFFB4070020040000000000000082
:1003A00000000000580000003C0100003400000084
:1003B000FFFFFFFFBC07002004000000000000005A
:1003C00000000000100000006004000018000000A1
:1003D000FFFFFFFFC4070020040000000000000032
:1003E000000000001C000000AC020000240000001F
:1003F000FFFFFFFFCC07002004000000000000000A
:100400000000000038000000F40100002800000097
:10041000FFFFFFFF34080020040000000000000080
:100420000000000054000000000100003C0000003B
:100430001800000000000000000000004004000060
:10044000080000000000000018000000000000008C
:100450000000000058040000080000000000000038
:100460001800000000000000000000007004000000
:10047000080000000000000001000000FC800000F7
:100484000100000000000E0000000F003200000018
:10049400010000000407002000020000000000002A
:1004A40001CA011000000000000000000800000064
:1004B400000023002C070020010000007407002026
:1004C4000800000000000000000000000000000020
:1004D400000000000000000001000000D40700201C
:1004E40006000000010000003C080020000000009D
:0C04F400000000000002000000000000FA
:0F0502002900010025002D002E002F000100010F
:1005140004000000E0800000000000000000000073
:10052400000001000000030087C40110380500002A
:10053400380500000000000090000000900000005A
:100544000000000074070020492E00002000000075
:10055400CC800000B87E00000DC30110FB1D00001C
:10056400FD1D000099C801109BC801100000000087
:10057400E62A0000207E0000387E0000087E00008D
:090584000800090001000000015B
:10059000000000000000000000000000000000005B
:1005A000E1190000011A0000051900002B1A0000D3
:1005B0004D190000231900007F190000571A000090
:1005C000C12D0000D12F0000D52F00000800000031
:1005D0002400000018000000280000002000000097
:1005E0003C0000000C00000034000000DFF800F0C8
:1005F00049C10110DFF800F019C20110DFF800F066
:1006000041AC0110DFF800F0CDA00110DFF800F0E0
:1006100085C10110DFF800F0C1C20110DFF800F061
:10062000E3BF0110DFF800F0C1C10110DFF800F0F6
:1006300009B70110DFF800F03DC10110DFF800F04C
:1006400029AF0110DFF800F0CDC10110DFF800F094
:1006500085B00110DFF800F0DDB20110DFF800F026
:1006600079B50110DFF800F0D5C00110DFF800F017
:10067000E1B5011020B1082328220021FFF7E2BFD5
:10068000704720B1082330220021FFF7D3BF704705
:1006900038B500F091FF25680DB129682160FFF79A
:1006A000A9FF284632BD70B504460D4626680020D5
:1006B00028601EB9FFF79AFF25600DE0FFF796FF4F
:1006C00000E0366831680029FBD1AE4203D1FFF764
:1006D00091FF002070BD3560FFF78CFF012070BDD9
:1006E0000022DFF8541C01EB4211CB7F1B0605D51D
:1006F000B1F91C30834201D108467047521C082AC8
:10070000EFDB0020704770B50646FFF76FFFDFF89C
:10071000545C0446A87E01001AD0401EA876C0B2E0
:10072000B0B9082100F026FC96B1A86B703001F03A
:100730007CF800F010FE301AB0FBF1F1022938BF4E
:100740000121EC352846FFF765FF2846FFF766FFD5
:10075000204600F065BE10B50446207B00F00F0077
:1007600002280FD100F012FDA168081ADFF8F41B6F
:10077000896BC968800801F57A71814238BFB0F190
:10078000405F00D3002010BD38B5DFF84C0ADFF819
:100790004C2A0168DFF87C4C02EA0105E94301605C
:1007A000A90608D54068800605D54FF4005104F12C
:1007B0004C0001F064F815F4602F08D0206905F4AE
:1007C000602108432061002104F19C00D0E131BD8B
:1007D00070B5FFF70BFFDFF83C4C0646206910F4BC
:1007E000602F27D02069C5012D0EE80748BF0025DE
:1007F00006D4A80748BF012502D4680748BF0225D0
:10080000681D40B200F040FF2069012105F111028E
:100810009140884320613046FFF7ECFE04EB8500F1
:100820004668300009D0206800224FF00063691D3F
:10083000B04702E03046FFF7DDFE206930B104F139
:100840009C00BDE87040002101F019B870BD70B582
:1008500001F0E0FBDFF80C5BDFF8BC4BAB6A024653
:1008600090071DD4D3E90401104007D0EB629969C9
:10087000084398614FF4804100F07CFBA86A00288F
:1008800047D16E6A002E44D0F068A96B884224D00C
:1008900005F14C00BDE870404FF4805100F0EFBF0F
:1008A0000BB9A86AEAE70020A862D3E904019E69AF
:1008B000024042F0020232439A61626982436261FD
:1008C000E26822EA0100E060194605F13000FFF716
:1008D000EAFE022100F04EFBE3E7B068FFF73BFFC2
:1008E000A86408B1A86CD8E0D6E9040162690243A3
:1008F0006261E26841EA0200E0600020E061B06805
:100900002060E0690028FCD005F12400FFF7C0FE5C
:10091000AE6270BD0020F6E6F8B506461446376EA6
:100920001D4607B1B847A00708D4D6E916012040F4
:1009300029400022914208BF904207D0C6E91A45DB
:1009400006F13800BDE8F240FFF758BEF1BDFEE702
:1009500080B500F084FFDFF8BC2A0146906BD26BB3
:10096000BDE80840104710B5DFF8A84A0FF2311172
:10097000E06B884202D101F0A9FB206404F14C0035
:10098000BDE81040042100F07ABF80B501F042FBC1
:10099000DFF8881A084207D0BDE804404FF0005144
:1009A000DFF8100C00F06BBF01BD70B5040073D010
:1009B000A168202001E04968401E79B1C2B26AB145
:1009C0000A8840F603039A421CBF40F604039A4289
:1009D000F1D1E0681822203001F094FBA0690021D9
:1009E000A1616168D9B140F00202E07F002300F00C
:1009F0000700012807D0022809D0042804BF0022DC
:100A00004FF0805306E000224FF0005302E0002236
:100A10004FF08043B4F91C10E0686568A847FFF701
:100A2000E5FDDFF840590646E88E401CC0F30B0098
:100A3000E8860020296BC87705F13000FFF728FE13
:100A40003046FFF7D7FDB5F93610E06800F1B8027F
:100A5000B2F90030994204BF297E00291CD1917857
:100A600009B9016811B90020907016E0AA6B1268EC
:100A700012F1010F10D0DFF8F42B1268B1FBF2F184
:100A8000022938BF01217030FFF7C4FDE068BDE8DE
:100A900070407030FFF7C2BD70BDBDE8704032E6F7
:100AA00038B50D46A807DFF8BC4816D5206BFFF710
:100AB0007CFF206B25F0020510B145F0020109E032
:100AC000680702D4606A002851D004F1EC0000F0FD
:100AD000ACFE042104F14C004AE0680747D5606A87
:100AE00008B1C068A063A06BDFF8E42A41680B7806
:100AF0001360126809788A421CBF8569002D05D0F1
:100B000000224FF000736FF0FF01A847022001F0B0
:100B10005DFC112001F06FFC01206077A06BE17E8D
:100B2000007C084204BF0E2001F065FCA06BDFF8DA
:100B3000E81840688268002A04BFC068002804D012
:100B40000020C861DFF8D80A086040F2FF70DFF8C3
:100B5000D42A106000208861DFF8C00848610FF2D5
:100B60001900E0631920BDE83240FFF773BD31BDC5
:100B7000BDE8344000F083BE2DE9FF478046880081
:100B800040F1B580DFF8DC57A86B40684068010091
:100B900018BF8047A86BDFF88098406881680029FB
:100BA00004BFC168002914D0D9F81C100029FBD05B
:100BB0000021C9F81C108068010018BF8047A86B8D
:100BC0004068C068010018BF8047DFF8B40A01F030
:100BD00029FA0020C9F81C0040F60A0ADFF8A40A26
:100BE000DFF8E07AC9F8000008F10804012001F0FC
:100BF00061FA0FF25110E863A7F800A00020788096
:100C0000002100F0B0F900F0A7F9206806467180D5
:100C1000E97E09B1617A99B1018840F602029142F8
:100C200005D1318A4FF60F421140318204E0318BF9
:100C30004FF60F42114031830021617201F028FA12
:100C40002068694601F016FA684601F022FA00E0D1
:100C50000646706800281CBF01885145F8D17760AE
:100C600040F60301707B00F0F0007073686A8068E2
:100C7000008888421CBF40F60401884202D100204F
:100C8000286417E0208BA8B100206083E06108F1A0
:100C90002C00017801F0F0010170417801F0F001C1
:100CA00041F00101417008F120007860787B00F08C
:100CB000F0007873D9F81C000028FBD00020C9F898
:100CC0001C00012001F056FE012808D0707B00F0C6
:100CD000F00040F0010070730FF21900E8634FF666
:100CE000FF322068018A11400182C9F80000BDE886
:100CF000FF870000DFF8D009014200D170470120D2
:100D000010B501F037FE0128DFF8584608D10FF280
:100D10003500DFF80417E063DFF8A809086010BDAC
:100D2000DFF8481909683220B0FBF1F1022938BF19
:100D30000121EC342046FFF76DFC2046BDE8104051
:100D4000FFF76CBC2DE9FE4306460C466004DFF855
:100D5000145619D5FFF74AFCEE6AB769B9070ED4E5
:100D60006EB10021B161FFF745FC706848B1B6F97A
:100D70001C10F06876683A460023B04701E0FFF7A0
:100D800039FC24F48044E1E0A0070AD5286BFFF782
:100D90000CFE286B002824F0020401D044F0020469
:100DA000D4E0A00005F1800840F60909DFF81479C5
:100DB00071D5B068018840F60202914205D1028ADD
:100DC0002D2161F30912028204E0028B2D2161F3CF
:100DD00009120283286CB8B1042001F0CBFD98B150
:100DE00001F074F9296C814228BF401E401A718AB3
:100DF00011EB1030F06040F2D761A0F2EE20884293
:100E000024BF40F6C410F060D6F818C0BCF1000F43
:100E10001CBFDFF8BC188C450DD0787B0F21084231
:100E200004BF708C484506D100224FF000736FF468
:100E300080713046E0470022DFF89818404600F005
:100E400031FD287F50B10220ADF80000684601F066
:100E5000E9F8BDF80800A88200202877012068760C
:100E6000A87E401CA87600206877686A18B119200F
:100E700000F01BFD01E044F00204D6F81480B8F144
:100E8000000F05D000224FF0806300213046C0479C
:100E900024F000545AE095F8200024F0080628B108
:100EA000200703D5002085F820003CE020073CD532
:100EB000002068760120A877002001F0FBF80FF2EF
:100EC000BD00DFF81418DFF86047E86300224046F1
:100ED00000F0E8FC297FE87E81F00101084202D1A0
:100EE0000120E8760FE0A86CB8B101F0EFF8296CAA
:100EF0006A6C401A02EB10306864A96CB0EBC11F39
:100F00000BD300206864A7F8009000F025F80020BB
:100F1000788000F028F8276003E04FF0005100F0DF
:100F200029F800202864344610E0A0040ED5AE6AEB
:100F3000002E1CBF7068002806D0B6F91C10F0689F
:100F4000766800222023B04724F4005414B12146CF
:100F500000F010F8BDE8F783787B00F0F00040F077
:100F6000010078737047387B00F0F0003873002080
:100F70007860704705F14C0000F081BC70B5054603
:100F80000E46B007DFF8DC430BD5206BFFF70DFDF5
:100F9000206B08B1022129E0B0002DD54FF000519F
:100FA00024E0B00028D501F04AF8DFF83007DFF878
:100FB0003067E063307818B905F13800FFF71EFBA1
:100FC000DFF8601600200860022001F095F911207A
:100FD00001F0A6F9287C10B90E2001F0A1F900203B
:100FE000E083B07840B10020B070042104F14C00DF
:100FF000BDE8704000F043BC70BD30B58DB001F06D
:10100000FCF8DFF8E006DFF8E0460168DFF854534B
:1010100041F00201016001A8FFF72CFBA078DFF886
:10102000CC160790002301AA05F14C00FFF70EFB38
:1010300001A8FFF726FB0020ADF81C0001AB2078CB
:10104000DFF89426099019210020009005F1800016
:10105000FFF7F4FA01A8FFF70DFBE078DFF8901630
:101060000790002301AA05F19C00FFF7EFFA01A801
:10107000FFF707FB0120ADF81C0001AB6078DFF83B
:10108000742609901A210020009005F1D000FFF786
:10109000D5FA00230022DFF8601605F1EC00FFF717
:1010A000DDFADFF83806E8630DB04FF6FF70A8826E
:1010B000012028770020E875E8766877E88385F8CE
:1010C0002000286430BD2DE9F041DFF814660446A5
:1010D00030788EB00F4690461D4618B9FFF78DFF49
:1010E00001203070002F1CBF6760B8F1000F4BD09B
:1010F000C4F80880FFF77AFA7178002942D10121FB
:101100007170FFF777FA35B909A80FF2246114223C
:1011100000F0F8FF09AD286820606868E060287C6E
:101120002074A868606101206074688A6082E86841
:10113000010018BFA061A02104F1200001F0D0FC43
:101140000823242200216846FFF76CFA01208DF85D
:1011500018006A46002104F13800FFF767FA0823F7
:10116000242200216846FFF751FA06946B460022BC
:10117000DFF8881504F17000FFF770FA20460EB012
:10118000BDE8F081FFF736FA0020F8E738B5FFF741
:101190002DFA7449497E31B1DFF868150C68FFF704
:1011A00029FA204632BDFFF725FA00F08FFF10F52F
:1011B0000030DFF8542541F10001A2FB0045DFF8C3
:1011C0000C0502FB015501690020221845EB0103C3
:1011D000184632BD000000000810044020000E0038
:1011E0002DE9F84F04460E4692469B46FFF7FEF95E
:1011F0005C4D8046B5F93400B5F93610401AC0F39D
:101200000B0008286FF0010944DAA88E401CC0F3D7
:101210000B00A886B5F93400ADF80000002046495F
:1012200001EB4017F97F090604D5401CC0B208281D
:10123000F5DB002704F1700000F0F7FABE6087F8D4
:101240001EA0C7F804B02021BDF80000B883FC60E0
:10125000DDE90A23DFF8B40410401940C7E90401AE
:10126000B8340020F87740F6FF76686A00283946DF
:1012700005F1240006D0FFF716FA30B100F05EF851
:1012800040464BE0FFF70FFA40B9A88E3018C0F384
:101290000B00A88600F070F948464AE000F04EF8CE
:1012A000E87F697E084208D0012085F820000020F0
:1012B000E8772877A87E401CA87600F05DF9A86A38
:1012C000002834D1687E18B1192000F0EEFA2EE023
:1012D000687F60BBFFF78AF90446A87F20B1DFF87A
:1012E00000140120887018E0B868FFF734FAA86489
:1012F000B8B100F030F8AA6C121AB2FBF1F2022A6F
:1013000023BFAA6C101AB0FBF1F10121EC3528467D
:10131000FFF780F92846FFF781F92046FFF76AF9C1
:1013200005E02046FFF766F90421FFF723FEBDF92B
:101330000000BDE8F28F0000D8090020BDF80000D1
:101340002080F87F40F08000F877A07810B100206E
:10135000A07028777047A86BDFF81013C068096881
:1013600070470000581D00202DE9F04106460F4649
:1013700014461D46FFF776F980463846FFF7B0F968
:10138000070003D14046FFF771F90AE0F87F072113
:10139000084209D04046FFF769F90721F87F084263
:1013A000FCD10220002116E07968DFF86403814255
:1013B00002D0796831667860C6E916454046FFF785
:1013C00055F94FF0FF3106F13800FFF71BF9002007
:1013D0003066D6E91A01BDE8F081DCB5DDE90667C3
:1013E0000446CDE90067180008BFDFF82433204623
:1013F000FFF7F6FE002803D500204FF00041DCBDCA
:101400000146204602B0BDE8D04002224FF0E04342
:10141000AAE70000581D0020001004400200004010
:10142000BDE87040FFF7E6B801E042F002022DE9A6
:10143000F843DFF8CC42606A0090894603271546DE
:10144000FFF7D4F819F1010F05F0010680460AD123
:10145000A06A002819BFA06AB0F91C90E08E00F1C4
:1014600001090020E0750FFA89F0FFF739F9010052
:1014700070D0A06A814205F0020525D1280003D072
:10148000606A0090002060620122C87FB240104371
:10149000C877FFF7E7F80746002E14BFDFF874029D
:1014A000DFF8740200F0BEFD00F066F825B906E032
:1014B00000F055F800F05BF800980028F8D13846A5
:1014C000FFF7D4F8832747E0009A8A4204F1EC0042
:1014D00016D100F0AAF9280012BF0020606A006847
:1014E000606200F049F8009800F039F800F03FF829
:1014F000009818B32800F6D120E0009A12680092F4
:10150000009AEAB112688A42F7D100F08EF9009889
:1015100000681DB1009A0021116004E00168009A82
:10152000116000210160009003E000F018F800F065
:101530001EF800980028F8D100F01EF8832701E07B
:1015400000F01AF8607F38B9022104F14C0000F075
:1015500096F901E000F010F83846BDE8F283C07F4C
:10156000009940F00400C8776846FFF791B801463B
:1015700004F13000FFF797B84046FFF73BB838B5A5
:1015800000F01AF805465E48407E68B1204600F03B
:1015900049FD044600F04AF804F0FF00012801D19B
:1015A000812032BD022032BD00F040F8012032BD62
:1015B00000000000A41D00200446FFF717B80A46EB
:1015C0004F49896B884201D00320704709E0000031
:1015D000D02108400A464A49896B884201D003203D
:1015E000704700211046CAE770B545498A6B9042A2
:1015F0006FF07F0411D1487E78B1FEF7F7FF054602
:10160000464800F00FFD064600F010F806F0FF0017
:10161000012802D13002001670BD204670BD0000C6
:101620005100070600000460001004402846FEF741
:10163000E1BF70B50E461546FEF7D8FF832430494A
:101640001EB1022E0DD005D30EE08A6A3AB1896A26
:10165000898B02E00A7F12B9898A298005E08024FB
:1016600003E0497E297000E003245BE0F480000081
:1016700080B50846FFF734F800B1806802BD00006D
:101680000100070601010E0438B5FFF795FF1C495C
:10169000CA7D520702D58B7D9C420FD001228B8AD6
:1016A00002FA04F52B438B820C341D4B1D68A240BB
:1016B00025EA02021A601A6802B90A76BDE83240C9
:1016C000FEF798BF681E002004000020681E00205E
:1016D0004F0900004F0800008B090000A10A00001C
:1016E0007B23002000200940347B000051090000CA
:1016F000D1070000890700006709000015090000F4
:10170000581D00200430044000093D00F1EFFF9F08
:101710001909000001000204010001040100030492
:101720000C100440FEF766FF204670BD000000006C
:10173000FFFFFFFFC4090000000000004F09000088
:1017400001001A01DFF800F021B30110DFF800F00A
:1017500095C00110DFF800F00DA80110DFF800F0CF
:10176000BDBE0110FEE7DFF80001007D70476DE0AF
:1017700038B5FFF7FCFFDFF8F8500446A8680021F1
:10178000FFF7E4FF6969081AA969814238BF0020A0
:1017900084F3118832BD2DE9F041FFF7E8FFDFF84F
:1017A000D0500446A8680121FFF7D0FF0121A9838A
:1017B0000021E9836E6929682A68871B801A711ADB
:1017C000884204D20020A88384F311882BE084F39C
:1017D0001188002406E0A61931460120FFF7BAFF60
:1017E0003F1B0446A742F6D2FFF7C1FF8046E88BB5
:1017F000012804D131460020FFF7ACFF0446A96957
:1018000014F1010F08BF084603D0E01B814238BF26
:1018100008468119FFF7A2FF012028840020A88331
:101820002E6088F31188BDE8F08100218182DFF805
:101830003C10C0684969884204D1DFF85C00006848
:10184000FEF7ECBE7047808A70477047DFF84C1097
:101850000968EFF3118081F311887047F6E7DFF82C
:101860004000806870470000A4010020780100203B
:1018700078010020616280F311882046704738B5F6
:1018800004460D46FFF7EAFF616A2943FFF7F2FFBE
:10189000BDE83240FFF756BFF8800000F08000003E
:1018A000C8010020816042607047102804D3DFF82F
:1018B0000C101038C1F8000F7047000000E000E085
:1018C00001F012B9FFF7C2BFDFF89811C20744BF99
:1018D00001220A60820744BF4FF480720A60400709
:1018E00044BF4FF4803008607047DFF87C21C307A5
:1018F00048BF1160830748BF5160400748BF9160EF
:101900007047000010B504460020D4E90A2347F6CA
:10191000906101F095F90123994228BF4FF0FF3003
:1019200010BD10B50C4600F0C7FB011D201AB0F128
:10193000004F05D8081BB0F1004F38BF8C4200D2D1
:101940000C462146BDE810400120CEE72DE9F041CC
:1019500080460A46D8E90A01D8E90C45A0FB02678F
:1019600001FB0277A6196F41340C002244EA0741BB
:101970004046FFF7D6FFC8E90E67BDE8F081F8B52D
:101980000646FFF79FFF0446DFF8E050DFF8E070FF
:101990000120E861FFF798FFF96A096A1420884777
:1019A0003069B0F5802F34BF0421010C0120FFF70E
:1019B0009CFF3A681268232100209047DFF8B4109A
:1019C00001200860DFF8B400016821F4E02141F44F
:1019D000803101600120286084F31188F1BD00008E
:1019E00000F074BB10B5DFF89000446800F006F812
:1019F0006069A169BDE8104008470000012063E765
:101A0000F8B504460D4600F061FBD4E90A6732469A
:101A10003B4601F015F93DB1A6FB002306FB01335F
:101A200007FB0033C4E90C23F2BD10B5DFF83C001E
:101A3000DFF86440002101600121C161216020685C
:101A4000FFF7DCFFDFF860100968096A1420884797
:101A5000206810BD000080B500F038FB000C40EAA3
:101A6000014002BD04200940182009400000244321
:101A70008401001080022443E4010020002009407A
:101A8000DFF8EC14096821B10A898242FAD10846CC
:101A900070470020704700002C200940DFF8D80470
:101AA000C088704700000000B001001000F008F886
:101AB0000EBD00BF08B582B00023009302ABF5E76E
:101AC00077B58DB01C461498ADF8180000250F9816
:101AD00028B92CE10EAA0DA800F070F96D1C00F0D9
:101AE00032F9080000F01D812529F3D100F02BF90F
:101AF0002D2905D10120ADF8060000F024F902E0FF
:101B00000020ADF80600302904D10120049000F037
:101B10001AF901E000200490002000904FF0FF30FF
:101B200002900A202A2918D12168216051F8042B3B
:101B30002160009200F0FDF8009A002A11D50122E0
:101B4000ADF80620009A524200920AE0009A00FB8B
:101B500002113039009100F0ECF8A1F130020A2AAC
:101B6000F4D32E291AD1002100F0F2F82A290F927D
:101B700010D100F0F9F80291002944BF0020029032
:101B800000F0E1F80AE0029A00FB0211303900F09F
:101B9000DFF80F92A1F130020A2AF4D3049808B1B9
:101BA000009804906C2918BF4C2905D10120ADF88C
:101BB000040000F0C8F802E00020ADF8040008A816
:101BC00007900CA805900020642918BF692903908C
:101BD0000DD1BDF818000028FFD000F0BFF86FF05D
:101BE00009030298049A8242B8BF049019E00A23BC
:101BF00075291FBF1023782908236F2903D1BDF849
:101C0000180038B906E0702913D1049320682060C9
:101C1000016814E000F0A2F8049A02988242B8BF6A
:101C20000490049A059800F0A5F807900599081A01
:101C30002FE0632919D12068206001680FE0001DA2
:101C4000206010230598082200F094F8401E0790A9
:101C500040200799087005980799401A19E0001D5F
:101C6000206007980170012013E0732913D100F060
:101C70007BF8079111B90FF244300790079801F0F3
:101C800057F80390029810F1010F1ED00399884273
:101C90001BDA039019E00F98401E0F900E9802284F
:101CA00013D3029810F1010F02D00E99884201D38C
:101CB0000E9800E0401CDFF8C462366802906B4664
:101CC00022460FA90DA8B047451900980399401A5C
:101CD0000090BDF8060038B902E000F030F86D1C45
:101CE0000098401E0090F8D50398411E039150B112
:101CF0000798401C07900EAA10F8011D0DA800F0CF
:101D00005DF86D1CF0E7BDF8060000283FF4E7AE73
:101D10000098401E00903FF5E2AE00F010F86D1CF8
:101D2000F6E70D9810B10D9900200870284610B004
:101D300070BD0F990F9A0978521C0F9270470EAA26
:101D400020210DA83AE00F9810F8011B0F90704762
:101D500002910F990F9A0978521C704720682060F1
:101D60000168001D206070472068206050F8041B47
:101D700020607047F0B500240025002B44BF5B4273
:101D8000002902D54942521E2D25B1FBF3F60FF270
:101D9000342703FB1611641C795C00F8011D3146E1
:101DA0000029F2D19442BEBF302100F8011D641C0D
:101DB000F8DB290018BF00F8015DF0BD10B50C4636
:101DC000116802290BD3491E1160016819B14A1C20
:101DD00002600C7010BD01F001F900B100E010BD0F
:101DE0002046BDE8104001F0F7B86549096808478A
:101DF00064480068004701207047FEE7704770475D
:101E000010B50446606808B9012010BD0B460146B4
:101E1000206852A200F0BCF8A1684118A160616876
:101E20000129A4BF081A6060002010BD2DE9F0410F
:101E300004468846A088164600F021F80746F11BA4
:101E4000002E01D40A2904DB236845A200F083F8A0
:101E5000C719A08980B1F51BA468002E05D42046BF
:101E600000F066FF401D854206DB23460FF2681234
:101E7000294600F070F8C7193846BDE8F0813EB534
:101E80000D463A49098814468142034628BF0FF29D
:101E9000501210D237490988814207D3FFF7F0FD6D
:101EA00021464268284600F073F83EBD2D49098856
:101EB00031B90FF238122146284600F069F83EBDCC
:101EC000314B1B680095002C48BF47F6FF7400217A
:101ED000029101946A462D49984702983EBD2DE92A
:101EE000F843170048BF47F6FF77044688460026A8
:101EF00074B32088010004D03A464146FFF7BFFF83
:101F00000646B91B012922DB208820B116A24046D3
:101F100000F03EF88619A068C8B1656875B128461A
:101F200000F006FFA7EB0609401D814506DB2B46A6
:101F30000FF2CC02494600F00EF88619B91B12299F
:101F400005DBA3680FF2C00200F005F886193046E1
:101F5000BDE8F283000040461AE00000257300004F
:101F6000257000008A0500003A2000005A21000078
:101F7000CC090020B6200000F001002008810000FC
:101F800000810000048100000C810000011E00009F
:101F900008B478B504001ABF2668002E00260D4646
:101FA00005AB3046FFF786FD854238BF681E16B187
:101FB00021680144216072BC5DF808FB286E756CD5
:101FC0006C290000303132333435363738396162AC
:101FD0006364656600000000282725732729000038
:101FE0007B6D6F64756C652325647D007B6D6F640C
:101FF000756C652D726F70653A25787D0000000064
:10200000222573222C2000006C696E652025643A1D
:102010002000000021490868C2430A600A680242A1
:10202000FAD170471E490A68002AFCD1CA610860CB
:10203000C8690028FCD00020C8614868704719486A
:1020400001686FF00202114041F400710160032148
:102050001548816041F2300141610121C160502188
:1020600041610121C1604FF4CA6141610121C16038
:10207000016070470D4802680A6082684A60C26861
:102080008A60406B20F0784040F08050C860704714
:10209000704701461022064800F024B81010044092
:1020A0000010044000000460004104404C13005044
:1020B000180000217047FF7F0948016842680368E3
:1020C0009942FAD1100C40EA0140704710B5044A19
:1020D000136850681468A3421946F9D110BD000076
:1020E0000820094062B38B0708D0521E11F8013B4B
:1020F00000F8013B00F024808B07F6D1830740F005
:10210000208000BF103A07D330B4B1E83810103A3D
:10211000A0E83810F9D230BC530724BFB1E808104A
:10212000A0E8081044BF51F8043B40F8043BD20734
:1021300024BF31F8022B20F8022B44BF0B78037028
:102140007047083A07D3B1E80810083A40F8043B52
:1021500040F804CBF7D25307E4E70040DFF800F083
:10216000F5C00110DFF800F049BA011020B10823D2
:1021700024220021FEF74ABA704780B50120009062
:1021800009234FF400720021DFF8080700F07BFFFD
:1021900001BD80B5002301223421DFF8F80600F0EC
:1021A00085FF00B10120C0B202BDDFF8EC068068F7
:1021B0007047DFF8E416401890F8ED0070470022F1
:1021C000022904D1012806D140F2EE2203E00128C1
:1021D00008BF4FF47A7210467047DFF8BC06D0F89B
:1021E000DC007047DFF8B00690F8E61021B1D0F8B7
:1021F0000C01010018BF004770472DE9F041DFF8DE
:10220000988608F1E1058AB0A879002861D10120FB
:10221000A871DFF88866DFF88876307B68717068AF
:10222000C8F80C0101A8FFF7A1FF00200690ADF847
:102230001400079001AB00220FF2F54108F10C00E9
:10224000FEF70CFA01AB00220FF2A15108F13000A9
:10225000FEF704FA01AB00220FF2D94108F1540055
:10226000FEF7FCF9B16801208847DFF838060078EE
:102270007868C0F38154707B20B1032C02D1012017
:10228000287003E0032C18BF022C16D1022000F0A6
:102290009DF8032CDFF810160CBF4FF47A7042F251
:1022A00010700968B0FBF1F108F15400FEF7B2F9C3
:1022B00008F15400FEF7B2F905E0012C03D100F05B
:1022C00063FAFFF75AFF386840075CBF002000F050
:1022D0007DF80AB0BDE8F08110B508B1140001D155
:1022E000022010BD8160C26003610146DFF8A805CD
:1022F00000F0F6FE002010BD10B50446FEF776F99A
:10230000DFF89415621892F8E8305B1E82F8E83026
:10231000DBB223B98A680123A3409A438A6066E04E
:102320002DE9F0410546FEF761F98046DFF86815B2
:10233000681890F8ED20521E80F8ED20D2B2002AE5
:102340003FD10FF2A050DFF8644500EB85052E78F1
:102350006F88300615D52168096A38468847216894
:10236000896A384688472168096B38468847DFF80C
:10237000401501200860DFF83C0500688007FAD5A9
:1023800012E0700606D501EB87010020D1F800119C
:10239000884709E021688969384688472168496B80
:1023A000384688470228F9D106F03F003F2818BF79
:1023B000FFF7B6FF687800F03F003F2818BFFFF72F
:1023C000AFFF4046BDE8F041FEF714B910B5044632
:1023D000FEF70CF9DFF8C0148A680123A3401A4302
:1023E0008A60611891F8E820521C81F8E820BDE865
:1023F0001040FEF7FFB8F8B50646FEF7F7F80446BA
:10240000DFF89454701990F8ED104A1C002980F8F8
:10241000ED2039D10FF2CC4000EB8607387800F080
:102420003F003F2818BFFFF7E6FF787800F03F0035
:102430003F2818BFFFF7DFFF7E883878DFF86C741D
:1024400001060ED53968C969304688473968496A36
:10245000304688473968C96A3046884700F019F81D
:1024600012E0400606D505EB86010120D1F80011E7
:10247000884709E039684969304688473968496BB7
:10248000304688470128F9D12046BDE8F240FEF7E2
:10249000B1B8DFF81C1401200860DFF818040068E8
:1024A0008007FAD570472DE9F04F002483B04FF034
:1024B000000A0128D04618BF012664D1DFF8D8935E
:1024C000D9F8DC0001285DD10220C9F8DC00FFF753
:1024D00045FE0090012000F062F9060054D1FEF79D
:1024E000C1F8DFF8D81301900C60012000F042FA27
:1024F000012804D1002000F0A7F94FF0010ADFF80D
:10250000C013DFF8B4030C6000681120FFF751FE20
:1025100008B14FF001081020FFF74BFE08B148F05A
:1025200002080F20FFF745FE08B148F004080B2011
:10253000FFF73FFEDFF8746320B13168096B4FF499
:10254000806088470A20FFF734FE20B13168096BAC
:102550004FF481608847DFF85813DFF86873DFF8BD
:1025600068B30120086048F0200031688969884715
:10257000DFF858130120086099F80800C00707D554
:10258000012416E0042673E00120C9F8DC006CE0A9
:10259000584600F0C7FD0546042DF9D0012D04D1A1
:1025A000326A526803215846904738688008800094
:1025B0003860002000F0C2FDBF4800683068806BC2
:1025C000804754B9012D04D1326A5268012158461E
:1025D0009047386840F0030038600120B84908602F
:1025E00040463168496988470B20FFF7E2FD20B17A
:1025F0003168C96A4FF4806088470A20FFF7D9FD27
:1026000020B13168C96A4FF481608847A849012028
:1026100008600020AD4908600320C9F8DC0031687B
:10262000496B404688470128F9D1042000F0B7F8EB
:10263000A24901200860A0480068A54800688006FB
:10264000FBD5BAF1000F1CBF012000F0FDF800F02F
:10265000C1FE082000F0A3F806460120C9F8DC00FE
:102660000198FEF703F800F039FE0098FFF77AFDB5
:102670003046BDE8FE8F38B50446FDF7B7FF054686
:102680002146854800F040FD28464BE030B5002447
:1026900001288BB004D021D303281DD018D31DE00E
:1026A00001A8FFF763FD7C4D8A490694ADF81440FC
:1026B000079401AB012205F17800FDF7CFFF0094EC
:1026C0000023854A2C2105F19C00FDF7B7FF05E0AA
:1026D00000F09CFE044601E000F03EFF20460BB0F7
:1026E00030BD00F054B938B5FDF780FF05466A48A3
:1026F00090F8E000012410B1FFF74BFD0446284696
:10270000FDF778FF204632BD38B5FDF76FFF624D0B
:10271000044695F8E00020B100F080F9002085F82B
:10272000E0002046BDE83240FDF764BF0000000035
:102730007047000010B582B0042000F01BF9022899
:1027400018BF032807D100F01FF8FFF716FDBDE8FA
:1027500016400220D0E56148534900684E4CC0F352
:10276000815003280CBF4FF47A7041F28830096819
:10277000B0FBF1F104F15400FDF74CFF04F15400FB
:10278000BDE81640FDF74ABF032000901C234FF020
:10279000405200213F4800F076BC0020704770B5E1
:1027A00004463D4E304600F091FC002598B9304675
:1027B00000F092FC0646B068204207D03269F36808
:1027C0000021204698470546012D05D0304600F0EF
:1027D00085FC0600EFD1284670BD414901280CBF99
:1027E00040F2FF70002008600020704770B5FDF7D0
:1027F000FDFE294E294D044696F8E00028B100F070
:102800000DF968B1002086F8E0000220AD68A84705
:1028100006461020FFF7C3FF8EB10320A8470EE045
:10282000214909683220B0FBF1F101B9012106F11B
:102830003000FDF7EFFE06F13000FDF7EFFE204619
:10284000BDE87040FDF7D6BE38B501281ED100F0B6
:1028500091F801281CD000F0D7F80F4C1249012044
:1028600084F8E00032200968B0FBF1F505B90125D4
:1028700004F13000FEF7D9FF294604F13000FDF7DE
:10288000C9FE04F13000FDF7C9FE01E000F0E8F8F0
:10289000002032BD00A00C40BC0800208C7A000053
:1028A000B03F00507F230020F4800000B8010010EA
:1028B00028200860282008402C2009400C400940AE
:1028C00000022243242208400040034080010443C8
:1028D000141009409536000065340000B43F0050E4
:1028E000000004608F3F00008F3F01008F3F020017
:1028F0008F3F0300903F00018F3F0101903F000296
:10290000903F00038F3F01048F3F00058F120804A2
:102910008F3F00048F3F0006513F00007F3F0100C2
:102920003F3F04003F3F02003F3F01007F3F020066
:1029300070B50446E00782B00D46624E05D5A8B2D8
:1029400000900023012200F011F8A00705D5A8B2DD
:1029500000900123022200F009F8600705D5ADB20E
:10296000009502230C2200F001F873BD00213046CF
:1029700000F089BB0146042907BF1D234FF0C04268
:102980001C234FF080524F48342100F08FBB38B5E4
:102990000546FFF791FB4C4CA168401A4FF47A7141
:1029A000484305EB104500F04BFF2169401A48BF32
:1029B000404240F6B9318D4207D2062805DAA068B8
:1029C000E168814201D322685AB940494A68D20776
:1029D0004FF4FA6017D4086800F0FF007D214843E7
:1029E00008E0081A3A494843000C00EB9000904276
:1029F00038BF1046C82801D2C82032BDB0F57A6F62
:102A000088BF4FF47A6032BD80B501210320FFF703
:102A10008FFFFFF751FB2C49886001BD80B5012075
:102A2000FFF7A8FF012819D00023012234212548EF
:102A300000F03CFB98B100F026F8FFF73DFB22497F
:102A40008B680A68C860A2EB9202C01A204B5843F8
:102A5000000C0860904238BF10460860012002BD9B
:102A600010B500210320FFF763FF0120FFF782FF6D
:102A700008B100F008F8144CFFF71EFB606000F08E
:102A8000DFFE206110BD1348006800F0EDBE10B5F8
:102A900011490A6811490968140424161B38444373
:102AA000E41004EB2244120600FB00F312160906A0
:102AB0005A435843091604EBA222484302EBA040B4
:102AC00010BD000000A00C405C230020AC3F005073
:102AD00040420F008000001090130050A4100050DE
:102AE000002200F0DDBE000010B54048046814F17B
:102AF000010F08BF002400F055FF3D490020086089
:102B000001203C4908603C49086001F01BF93B4842
:102B1000006820B13A480068204600F01CF83949A6
:102B2000394A00200860394801686FF31B4111439E
:102B3000016037480168C1F30131012906D10168FC
:102B4000344A114041F400320260016032480068AA
:102B50000028FBD110BD70B5054630480121016049
:102B60002F4909680029FBD02E4C2F4AC021216033
:102B700053682E499B075DBF13681B0C43F0F0039D
:102B800072230B70002101639668304600F014FF39
:102B90003146284600F043FF2548816D89B240F256
:102BA0000F22914213D201680068C1F30361C0F3A0
:102BB000034001B1491E072805D006280EBF072093
:102BC000801C00F00F0041EA00101A4908703046DE
:102BD00000F094FF18490968C9680220884740201E
:102BE000206001201549086070BD00001C130050D2
:102BF000840460425C600C40082204438001284346
:102C0000000120438C210840000039014820034086
:102C100004000940FFFFFCFC0C0068421010094052
:102C20009402224300600C40AC3F005056620840C2
:102C3000BC12005002600840A001001094046042E1
:102C40001B4213D1094236D12AB18446B0FBF2F0BF
:102C500002FB10C2704701F0E5B8FCD3002200234C
:102C600070470B000200002100207047904271EB7A
:102C7000030CF6D370B5B1FA81F4B3FA83F52C1BCB
:102C8000A340C4F1200532FA05F63343A2405FF0B9
:102C90000046E64002E05B085FEA3202841A71EB0C
:102CA000030524BF204629467641F4D302000B00D9
:102CB0003000002170BD012ACFD970B5140C20D08E
:102CC000B1FA81F4B2FA82F5C4F120046419B4F1C6
:102CD0002006D6D3B2405FF00044F440002502E065
:102CE00052085FEA3303C61A71EB020E24BF304666
:102CF000714664416D41F3D302000B0020002900AE
:102D000070BD0C46B1FBF2F102FB11452D0445EA02
:102D10001045B5FBF2F402FB145580B240EA0545BC
:102D2000B5FBF2F002FB105240EA044070BD000017
:102D300000F10103810704D010F8011B89B181075C
:102D4000FAD10268B2F10131914311F0803F04BF22
:102D500050F8042FF6E710F8011B11B110F8011B11
:102D6000FBE7C01A70470000DFF800F00DC3011048
:102D7000DFF800F081C60110DFF800F095B7011010
:102D8000DFF800F08DC20110DFF800F03DC2011045
:102D9000DFF800F009C30110DFF800F045C00110B2
:102DA000DFF800F0D1C70110DFF800F067BE0110B6
:102DB000DFF800F011C80110DFF800F021C80110A1
:102DC0000C381F283ED8DFE800F0103D3D3D3D3D6A
:102DD0003D3D3D3D3D3D3D153D3D3D1A3D3D1F24A5
:102DE0003D3D3D293D3D3D2E3338DFF8F40100687F
:102DF00000687047DFF8E801006840687047DFF856
:102E0000E001006880687047DFF8D4010068C0689E
:102E10007047DFF8CC01006800697047DFF8C00137
:102E2000006840697047DFF8B80100688069704742
:102E3000DFF8AC010068C0697047DFF8A4010068E2
:102E4000006A70470020704700B589B009216846C4
:102E5000FFF78AFF09B000BD00B581B0FEF730FD75
:102E6000DFF88001DFF880110068884218BF00F0A9
:102E70009BF8DFF87801B0F5B26F03D001B05DF8D0
:102E800004EB92E001B000BD2DE9F04184B01D4695
:102E90000B6880461446002226681F78002003F144
:102EA000010C242FC1F800C038D15F780CF1010368
:102EB0004C2F0B6006D156F8040BAA684146FEF76A
:102EC000B5FF25E0462F0DD156F8041B0191414670
:102ED00056F8040BADF8002002906846AA68FEF789
:102EE000FEFF15E0532F19D156F8040BE861266058
:102EF0002346288B0090EA69A968D8F80000FEF7FD
:102F0000DFFDD8F8001011B10144C8F800102668A0
:102F10000021E96001222968091A2960662F08D179
:102F2000298B002911BF361DF11D21F0070101F188
:102F300008061AB9E9690F700121E960266004B03A
:102F4000BDE8F0814FF0FF309060704700B581B070
:102F5000FEF7A4FD012818BFFEF704FC0FF21D00C8
:102F6000FFF706FFFFF708FFFFF70AFFFFF70CFF69
:102F700001B05DF804EBFFF70BBF000000B581B0B6
:102F8000FDF770FBFFF7EAF801B05DF804EB0320F2
:102F9000FFF702BF10B504460320FFF7FDFE2046F1
:102FA000BDE81040FFF7FCBEFEE7FEE700B581B0CC
:102FB000FFF7FAFEDFF83800C06801B05DF804EBF7
:102FC000FEF7C0BBDFF82C10DFF82C0088617047DB
:102FD000FFF7EEBEFFF7F0BEFEF707BFFEF708BF34
:102FE000F001002098CA01107047282090050000C9
:102FF00078010020440100200004000070B5044660
:103000000D46164600F0E2F9401E8041C00F1A49F5
:103010000A68002AFCD0012E02D0022E02D003E062
:10302000257002E0258000E0256001220A6000286A
:103030001CBFBDE8704000F0CDB970BD38B5044686
:103040000D4600F0C3F9401E8041C00F0A490A68CE
:10305000002AFCD0012D02D0022D02D003E02478FA
:1030600002E0248800E0246801220A6008B100F030
:10307000B1F9204632BD000000800C400B461146DD
:1030800004221818BAE710B500EB4100102B1446C3
:1030900000F5007002D3103B001D240C02999940EA
:1030A00041EA0441BDE810400422A7E738B51D46B7
:1030B0000818102D144602D3103D801C240C022148
:1030C000FFF7BCFF204080B2E84032BD0068002816
:1030D0000CBF0120002070470068704700687047EF
:1030E00038B504460D4600F09EFE00212960616857
:1030F00069606168002914BF0D6025606560FFE7A5
:10310000BDE8324000F091BE0B684A68002B0CBF4E
:1031100042605A604A680968002A0CBF0160116069
:1031200070470000006801074CBF042000F0030056
:10313000704700001628A8BF203870472DE9F84FC7
:1031400006469348934C0068934D800704D50820A9
:10315000A87192482060BFE000F072FB8046904862
:10316000006800900027001700F101090098800214
:1031700008D4C8F13E00C0100928A8BF0820814526
:10318000B8BF814687480068C0F30460FFF7D2FFEC
:10319000824685480068C0F30440FFF7CBFF09EB87
:1031A0000A011629A8BF152104DA6FF0090291421D
:1031B000B8BF114601F01F027C4B42F4F8521A804E
:1031C0007B4A126812F0030F18BF0127520748BF4D
:1031D00047F002070EB147F0040795F90720A8EB66
:1031E0000202052A02DAAA7997425DD0A8F10F0CF3
:1031F0000026BCF1000FB64607F0010207F00403F9
:10320000DFF8B09123D40CEB0C1C4FEA2C2EBEF14E
:10321000080F28BF4FF0070E7646072E28BF062658
:1032200009EB860A59F82660DAF804A0AAEB060A28
:103230000AF0FF0613B1CAF3072B5E445FEA877BEF
:1032400044BFCAF3074B5E440AB106EB1A6659F84D
:103250002E9009F0FF0A13B1C9F307239A44BB0764
:1032600044BFC9F307439A440AB10AEB196A401AEA
:10327000ACEB0E220099AF71724380320128B8BFC7
:103280000120342301F0FF0158430AEB1222484386
:10329000B0FBF2F0B0F5803F28BF4FF6FF7008F3A7
:1032A0000708A88085F8078043480068A988286037
:1032B00000201F2904D21F21A98004E04908401CD6
:1032C000B1F5007FFAD20F39090940EAC1003B4944
:1032D0000843206000206060BDE8F18F10B53848D9
:1032E000006884B21CB300F0ABFA2B4991F90720B7
:1032F000904205DA6FF07F029042B8BF1046C87165
:103300008888844201D28C8010BD2B4A12680B68D9
:10331000D21A921C202A28BF1F22231A5208D340F7
:103320001818B0F5803F28BF4FF6FF70888010BD99
:103330002448026802B9704710B5234B996801F020
:103340004060B0F1406F21D011480468A4071DD43B
:103350005C68A4071AD404681B68C3F303531C33C6
:103360001B0114F0050F06D09A420FD26FF0050131
:103370002140016010BD934208D20A0158BF44F0B9
:103380000104490158BF44F00404046010BD00006A
:10339000000009403010094070230020FDFDA4000A
:1033A000B43F0050B81200503C1100506E6208400B
:1033B000242208409C1300500820094000E7A48004
:1033C0003410094028500940AC3F0050EFF3108002
:1033D00072B67047EFF3108062B67047DFF800F006
:1033E00099C8011010B50C18FFF7F0FF401E80417E
:1033F000C00FDFF8F0130A68002AFCD0246801220D
:103400000A6008B1FFF7E6FF204610BD38B5DFF8C7
:10341000D843DFF8D8132078897B002508430AD0E9
:10342000FDF7E4F8A178002906BF0121A17001256C
:10343000FDF7E0F80DB1002032BD0220FEF7C6FF17
:103440000E20FEF7D8FFDFF8A803016809B10120BC
:1034500032BDDFF8A023402111600121C1610020AD
:10346000607032BD70B5DFF88C0382B0002101605E
:103470004821C160DFF8800300F1D804A17A002957
:1034800068D00129DFF8742329D110684BF2F521A7
:103490004843050ADFF868030068C0F3814001284B
:1034A00006D100F0CDF9FFF7F2FA684305EB90552D
:1034B000607B10B10020607305E0D2480068000214
:1034C00015EB10204508D0480560290C416001210A
:1034D0008160C648807B00283AD0052039E0022967
:1034E00009D11568284600F0FDF8A5F2FF50032821
:1034F0002ED308202DE003292CD1116800F1B80546
:10350000A1F5C0612868E961002848BF4042002950
:1035100048BF49428842A8BF002018DA6868BB4EFD
:1035200080B2009008234FF47F4230213046FFF7ED
:10353000AAFDA86800F072F904213046FFF7A3FD48
:10354000A86900F071F93046FFF79DFD0120207059
:103550000B202073BDE873402DE9F041A64CDFF845
:10356000AC82AB4FAB4EA34804F1E10582B0E978E1
:103570004A1E0B2A00F28080DFE802F00622334662
:103580005B33465B3346636EA349096809682020B4
:1035900088470F20F860072341F61D5038614FF42B
:1035A000C0720220009000F070F807234FF4C07240
:1035B00000214046FFF77AFD01203060022044E000
:1035C0000120F861287800281DBF00203061032009
:1035D0000620E87003203860002070607068800763
:1035E00034D4E878032804D1022000F04BF80420FA
:1035F00007E0002000F046F8E87806280CBF072016
:103600000A20E87001201AE0042903D12021B961C1
:10361000012105E00122BA610A290CBF0321022120
:103620006970002139600821C160016001203860A3
:1036300026E005290CBF06200920E87000207060F4
:1036400004E00020306070600C20E87004F1780025
:10365000BDE8F641FCF7E2BF0021016001206449AA
:1036600008600E20FEF75CFE0220FEF745FE0120FA
:10367000E8700020A87003E0BDE8F341FFF7AEBE9C
:10368000BDE8F38100900523602200214046FFF74A
:10369000FABC000080B558495E4891F8E410891ED4
:1036A0000A291AD8DFE801F0060A0E190A0E190ACB
:1036B0000E19120001688907FCD510E041688907DE
:1036C000FCD40CE041688907FCD508E00168890753
:1036D000FCD441688907FCD401E0FFF77FFEBDE818
:1036E000014039E7F8B50746484C30212046FFF73E
:1036F00079FE414E06F1B805C0F307206860042149
:103700002046FFF76FFEC0F38440A86020212046CA
:10371000FFF768FEC0F38120A861B7F5C06028609C
:1037200002D186F8D800F1BD296996F8D8202AB9C7
:103730006A68A968EA60E861AA696A61E8690028BC
:103740004CBF6FF00102022200EB40001018421043
:1037500000EB927001EBA0006968E960012810DAC3
:103760006A69032A04D1153001281DDA01201BE003
:103770000B300128B8BF0120491E48BF0021E96075
:1037800007E01F2812DB6A692AB915381F28A8BF6D
:103790001E20032109E00B381F28A8BF1E20491C4A
:1037A0004029A8BF3F21E960002169612861082301
:1037B000E86880B200904FF47F42302100F03CF87E
:1037C0000120009011234FF4003200F034F82869F2
:1037D00000F024F800F02FF8686900F025F800F0F8
:1037E0002BF8F1BD00800C409D0900208C7A000070
:1037F00004800C402C500C40BC08002008400C40B9
:10380000B43F0050102009403C600C4000A00C4028
:1038100000400C4034600C40A001001080B20090C9
:1038200012234FF4F802704780B200900A234FF43D
:1038300040622021704704212046FFF724BC00008D
:103840000748084A81681278006852B2A0F54070B3
:10385000C9035043C913A1EB2010803000127047F8
:10386000285009400C13005070B50446FFF7AEFD18
:10387000451EAD41ED0F074E30680028FCD0A04733
:1038800001203060002D1CBFBDE87040FFF7A2BDD5
:1038900070BD000000800C4062F30F2262F31F42F3
:1038A00000B500BF130096469446103928BFA0E823
:1038B0000C50FAD85FEA417C28BF0CC048BF40F8E2
:1038C000042BC90728BF20F8022B48BF00F8012BA2
:1038D00000BD000030480068000C00F0070005281B
:1038E00028BF4FF0FF3070472C490A68C2F30F32EF
:1038F0004BF69A139A424FF0FF3006D10868000F3A
:103900000B280CBF0420002070474BF6BE118A42E2
:1039100001D1012070474BF641318A4201D1032089
:1039200070474BF620318A4208BF022070470000E2
:103930001A48F8B50068050F1948006800F0FF063E
:10394000802E28BF0026FFF7CFFF04284FF0FF345A
:1039500006F10A071DD8DFE800F003121A1A1B004F
:10396000012D12D0032D06D0072D06D0082D08BF3B
:1039700006F116040DE014240BE0152409E025B12E
:10398000022D08BF06F1140403E00A2401E005B982
:103990003C4660B2F2BD0000941200501813005073
:1039A000A010005080B5FFF79FFF20B9FFF7C0FFC0
:1039B000162800DB01BDFEE7DFF8E8130968C1F354
:1039C00004611629A8BF203901EB2071491C162972
:1039D000A8BF152104DA6FF009029142B8BF114661
:1039E00001F01F01DFF8C02341F4F8511180DFF826
:1039F000BC13096889074FBF40F040600021DFF821
:103A0000B0231160DFF8AC13C0F3C06282F0010292
:103A1000C0F380600A6080F001008860704770B574
:103A2000054682B0084600F0EEF80246DFF888430B
:103A3000182100F060F800F012F980B20090002325
:103A400040F2FF322C212046FFF71DFBDFF86C63AC
:103A5000F068C0F30D021C2100F04DF8706800F012
:103A6000FC32142100F047F83068DFF85413DFF817
:103A7000546301EA0002102100F03DF8284600F0EE
:103A8000F8F802460C2100F036F8284600F01CF940
:103A9000400040F020003072284600F01EF940F04F
:103AA00010003072284600F021F90246282100F06B
:103AB00022F8284600F0FFF8400040F06000F07265
:103AC000284600F02DF9C00040F0800030702846F4
:103AD00000F02FF98000BC4940F47C400880284663
:103AE00000F011F90246082100F005F8B7494FF43B
:103AF0008000086073BD2046FFF7C0BAF8B5810C9E
:103B000001F003010129B24CB04D02D002292AD0A4
:103B100026E0216A8A0323D44FF480422A606FF0A2
:103B20008F06AC4AD2F8023033404E0A06F08006C7
:103B30003343C1F303363343C2F80230C1F30326E3
:103B4000D2F801301B0946EA0313C2F801306FF0C6
:103B5000E7061368334001F0E7011943116002E002
:103B60004FF0004129609C4E9C4AB16809075CBF38
:103B70004021A9624FF400712964800D216AC90CAB
:103B800001F0030141F0300110F00300117003D087
:103B9000022826D008D326E001210420FEF7C8FE23
:103BA0008F4800F0F0F822E00120FEF7E3FE074620
:103BB00039460420FEF7BCFE0420FEF7DBFEB842C7
:103BC000FAD1366826F07F4000F0DDF8854B1B689F
:103BD0001B684FF060220721300E98474FF4806039
:103BE0002860032100E002210420FEF7A1FE2068E6
:103BF0007D4900F03F00087047F618007B490880B7
:103C00007B480068F1BD7B490968C1F38362830387
:103C1000C1F38F2120D4000400164FF6FF7307E094
:103C2000490804D11946520804BF01220121401C51
:103C30000028F5D401280FDB490041F00101B1F55E
:103C4000803F21BF0121520042F00102102A24BF0F
:103C50000F221946401EEDE741EA024070476548D1
:103C6000016800680002C1F3870100F44070084356
:103C7000704730B5604C61490A686568ED07C2F36A
:103C80000351C2F303430AD42468250501EB2571CF
:103C9000240481F3040103EB247383F304031B0462
:103CA00043EA015193B21943222824BF02F0804015
:103CB0000143084630BD0021202803D35048006846
:103CC000C0F30151084670470121222803D34D4813
:103CD0000068C0F30071084670470121222803D311
:103CE00048480068C0F3407108467047002120280A
:103CF00007D343480068C10C01F44071C0F38450FD
:103D000001430846704720283F4907D33C483F4AB3
:103D10000068810A02EA003040EA81510846704793
:103D20000021222803D337480068C0F3C061084649
:103D300070470021222803D332480068C0F3455160
:103D400008467047324800680028FBD13148324AA3
:103D5000416812688908890041F0005141F004016E
:103D6000520748BF41F001010BD4026812F0030F63
:103D700007D041F003024260026802F00302032A06
:103D8000FAD141607047254982B20A60C0F307400A
:103D9000486001208860224800680028FBD000208D
:103DA00088607047B81200506E62084000000940F9
:103DB00094042A430000204300A00C4070130050DC
:103DC000FFFFFC0041A10C40DCA10C4040A00C40D6
:103DD0006C1300500A600840A83F005008A10C4036
:103DE000BD378600B40100100BB00C4070B00C4021
:103DF0002C20094050130050AC3F00507813005065
:103E0000981300508C13005000803F4000F03F009A
:103E10000C00684200400340B03F00503C600C4042
:103E200084088C437047FCF7E1BBFCF7E3BB000060
:103E3000DFF800F0D9C10110DFF800F025B1011062
:103E4000DFF800F013C10110DFF800F0B9C2011073
:103E500000B583B000F00DF8032114E0E0B500F0E8
:103E600008F8042100F012F808B100200EBD0298F5
:103E70000EBD0821ADF800100190704700B583B069
:103E8000FFF7F7FF052100F001F807BDADF80210BC
:103E90006846DFF8E01A0968084700B58FB00823C4
:103EA0003C2200216846FFF7C3FFDFF8CC0A00F18F
:103EB0005001079100234FF4587108916A4601217F
:103EC00006910FF24D11FFF7B7FF0FB000BD10B50F
:103ED00086B00820ADF800000120DFF8981ADFF85E
:103EE0009C4A0968ADF80200684688479DF80400BE
:103EF00020700298606204F1500000F0A5FEA062FC
:103F000000230020019000904FF47A720FF61521E3
:103F100004F12C0000F054FE0FF6192000F000FF11
:103F200000214FF0004000F097FF20626A464FF6F4
:103F3000FF70E08101210020206108208DF8000041
:103F400040F2044000F0EEFF4FF47A61022001F0ED
:103F5000E6FB4FF47A61032001F0E1FB0FF6144217
:103F60001521002001F0E6FA44F6C740019001AAAD
:103F700001208DF80300042100208DF802008DF847
:103F8000010001208DF800004FF4816001F016FC63
:103F90000DF1030201214FF4806001F00FFC0DF1DF
:103FA0000202012140F2024001F008FC0DF1010281
:103FB000012140F2034001F001FC6A46012140F278
:103FC000064001F0FBFB01F07FFA207801F08EFA49
:103FD0004FF0FF3001F0ABFA4FF0FF3001F06BFA19
:103FE00004F15C0000F08CFF04F1600001F015FAB0
:103FF000207801F00FFA207801F063FA00F0F8FA67
:10400000206A0FF68413002100F051FF06B010BDA6
:1040100070B586B0FFF75BFFDFF86049DFF85459F1
:1040200024E0A06A00F03BFE060004D000F07EF819
:104030003046FFF723FFA06AFFF702FF0028F0D009
:10404000A08AC10712D54FF6FE710840A082002059
:10405000A083608320830120607105A9E08B227812
:10406000001FADF81400E08A01F0CEFA0820ADF888
:1040700000000A20ADF802004FF0FF3001906846C2
:10408000296888470028D6D10820ADF80800092003
:10409000ADF80A0002A8296888479DF80E10049E12
:1040A0000028C8D1BDF80C00102801BF207881423B
:1040B000304600F006F8002EBDD03046FFF7C8FEAF
:1040C000B9E700B585B0017891290BD0B02905D0AA
:1040D000D02929D105B05DF804EB84E005B05DF886
:1040E00004EB8DE241780E2902D0102915D01BE097
:1040F000818841F20542914216D100F072FA80683F
:104100000FF6C81390F90300404200900421DFF835
:104110006C08006A00F0CBFE06E005B05DF804EB29
:104120000021082001F032BD05B000BD2DE9F041AD
:10413000044686B02088022829D004282DD00828DB
:1041400011D0102809D020284CD16068FFF7B9FFA2
:10415000606806B0BDE8F0417AE6A17806B0BDE837
:10416000F04100201FE1646860884FF6FF718842CB
:1041700038D0012101F0EDFAA0B32188606800F089
:1041800045FD608806B0BDE8F04101F017BC6068ED
:104190000178A07800F0C7FA1FE06068DFF8DC67FC
:1041A0000578F78A01F0B4FCDFF8D417DFF8D027E0
:1041B000B0FBF1F102FB110855B100F0DEF8CDF8CB
:1041C00000800022306A0FF68413042100F06FFE95
:1041D00042460021384601F029F9606806B0BDE882
:1041E000F0414BE6EEE170B5DFF8905786B004463B
:1041F000286AA2780FF2E8764FF6FE7162B1012AC2
:1042000046D0052A5CD0062A00F08B80072A00F0F1
:10421000A8800D2A11D0ADE06089E883E01C00F091
:104220004BFD00F0D6F9286A0022012100F03FFE84
:1042300000F0B0F80FF25C7399E02069217B014433
:10424000491E00E010448842E5D210F8012B002AF4
:10425000F9D00378022B18BF032BF3D1401C521E58
:1042600001E0801C921ED2B2022A01DB884203D3F5
:10427000012AE8D1401CE6E70378F02B04BF43781D
:10428000FF2BEED12179601D06B0BDE87040FAE247
:104290000021E97004910391029101910022697853
:1042A0000FF2FC6300F091F9687830B100F072F819
:1042B0000FF20073032100F0FAFD6878A87059E04E
:1042C0006278C2B9022028716089E88201202872D0
:1042D000A88B18B905F12C0000F096FC00F05AF8F4
:1042E0000FF2E06300F072F9201D00F0E5FC0346D8
:1042F00000F043F810E00022E9822A716A7104920A
:10430000039202920192009202210FF2C46300F024
:10431000CEFD00F038F8607800900022286A032172
:1043200026E0002028716871A8832872E982A0889D
:1043300000F0D4F900F02EF80FF2B06300F046F967
:1043400000F021F8A07900900022286A032100F0F3
:10435000AEFD286A06B0BDE870400022042100F0DE
:10436000A1BD00F03EF9E1780FF2906300910221C7
:1043700000F09DFD06B070BD002200200490039067
:1043800002900190704700200490039002900190E9
:1043900033467047002004900390029001900090F3
:1043A0000022286A70472DE9F041DFF8D045DFF898
:1043B000D465206AA3786278E7780D0786B01CD5AB
:1043C000002F38D1110036D0591CCBB2934228BFF0
:1043D0000021A17000F005F9A1780FF23463491CA7
:1043E00000F0F3F8A07806EBC000801C00F064FC3D
:1043F000034600F0FDF80321E2E094F804C0E58AEA
:104400005FEA817853D5BCF1020F18D0A7B901211A
:10441000E1700021617000F0B9F90FF2006300F063
:10442000D5F8206A0422032100F03CFD002201217E
:10443000032000F0E0FDC5E000F0F3FDC2E0A08B3A
:104440000100FBD0217A0029F8D1E179F9B10023EC
:1044500001221221284601F0F1F900280190EDD047
:10446000A08B0199ADF800000120ADF80200A07901
:1044700008700020ADF8080069462278E08A01F053
:10448000E5F868B11221684601F0E7F99AE0ADF865
:10449000000069462278284601F0D4F8002805D1AA
:1044A00001202072E07980F00100E0718AE0C80606
:1044B0000ED5BCF1020FF9D14FF416700090002315
:1044C0004FF448724FF4C871284600F084FD79E03B
:1044D000C80736D5BCF1000F1BD1002A72D00121CC
:1044E000217106EBC300851C42782B460021002079
:1044F00000F056FD00F07CF8206A0FF2305300F017
:1045000065F8284600F0D8FB00F063F8002203218C
:104510000FE0BCF1010F18BFBCF1020F52D1032014
:104520002071284600F036FD00F062F80FF20853C3
:10453000022100F0A5F9206A0022042100F0B2FC5B
:1045400040E048073ED5BCF1020F3BD1284600F0C1
:10455000E1F868BB0121284601F0FBF8002831D0C2
:10456000284600F0D7F807004FF47A7604D0786830
:1045700000F061FB3E8016E0E0894FF6FF71884253
:1045800020D12420FFF76AFC2061D8B100210191DD
:104590000091002300220FF2A53100F011FBE5810C
:1045A00004F10C07A6813146786800F02FFB09E082
:1045B000284600F093F800F01BF80FF28C4304211A
:1045C00000F05EF906B0BDE8F0810091022100F034
:1045D0006EBC002104910391029101910091034668
:1045E00070470021049103910291019100227047CC
:1045F00000200490039002900190009000227047E8
:1046000030B5DFF8785304462879022885B04FD1B9
:104610006278286A2179162A05D100F051F80091B4
:104620000FF234433BE00B2909D001290FD1217A45
:104630000A291CD100F04AF80FF2304305E0FFF7D9
:10464000D0FFE1680FF234430978009109E01329A3
:1046500014D1A9790FF2444300914A1CAA7100F0C9
:104660002FF8042100F023FC0020287220E01229FA
:1046700019D100F02BF80FF21443E6E77E2905D19B
:1046800000F08CF80FF22443217A06E07F290AD14A
:1046900000F084F80FF224432189009100220421C4
:1046A00000F005FC04E0687910B1204600F07CF8C9
:1046B000217904F1080005B0BDE8304001F0CDB823
:1046C0000022049203920292019270470021049109
:1046D0000391029101910022217B704738B5044675
:1046E00000F018F8A0B14068A44D00F0A4FAE889E1
:1046F000A0420BD1286930B1FFF7A6FB2869FFF76C
:10470000BDFB002028614FF6FF70E881002032BD1C
:10471000122032BD9949CA89824202D101F10C00AE
:104720007047002070470200944800B5006A85B0C9
:1047300005D100F033F800910FF2A03321E0012AF7
:104740000B460AD121B900F021F80FF2A03319E08D
:1047500000F023F80FF2A43313E0022A05D199B92F
:1047600000F014F80FF2A8330CE0032A0CD121B9A1
:1047700000F00CF80FF2A83304E000F00EF80FF28E
:10478000B4330022FFF722FF05B000BD049103916E
:104790000291019100910022704700930021049141
:1047A000039102910191704710B5744C6179012910
:1047B00086B019D10079032860D10FF2A0300FF232
:1047C000FC230088ADF81400FFF7D6FD0421172064
:1047D000009000F055F80220607102222378E08AF0
:1047E00005A900F018FF49E002292ED10179072917
:1047F00028D1018951B1C1680A784B7802EB0322B4
:1048000022838A78C97802EB0121618340781A28D3
:1048100034D1208B010031D0ADF800000321608B32
:104820002278ADF80200617102208DF8040069461B
:10483000F1208DF80500FF208DF80600E08A00F0D9
:1048400003FF1BE0012919D1E3E7032916D1017900
:10485000092911D1018979B1C1680FF204330878AF
:10486000497800EB0120A083FFF786FD009002212C
:1048700000F006F8002020720020607106B010BD24
:10488000206A00F014BB2DE9F0473C4E7778082FE2
:1048900080468A461DDA0025DFF8E89000E06D1CAE
:1048A000E8B2B8420AD2EDB209EBC500811C06227B
:1048B000404601F02BFA0028F1D10AE009EBC704C9
:1048C00006224146A01CFDF70DFC84F801A0781CCF
:1048D0007070BDE8F08780B502460021202000F00E
:1048E00035F8401E8041C00F02BD38B50C46154654
:1048F0000120FFF7B3FA020005D015702146BDE88C
:104900003840022022E031BD10B51C460120FFF7DF
:10491000A5FA30B104700246BDE810400021042021
:1049200014E010BD1548818A41F001018182406A7E
:10493000FBF764BE01460022102007E00F4901EB9F
:10494000C00000F10C0200215FF0080070B50446C1
:104950000D4616460820FFF781FA50B10480857095
:1049600046600246BDE87040044B596A986A00F000
:1049700072B970BD540600207C1E002090060020F5
:1049800040420F002C220020424C452043656E74AB
:1049900072616C00496E697469616C697A65640062
:1049A0004465766963657320466F756E642025647F
:1049B000000000003C2D20546F2053656C6563742B
:1049C00000000000436F6E6E656374656400000054
:1049D000436F6E6E656374204661696C65640000A8
:1049E000526561736F6E3A202564000044697363F9
:1049F0006F6E6E65637465640000000050617261E3
:104A00006D205570646174653A20256400000000D3
:104A1000446576696365202564000000446973631A
:104A20006F766572696E672E2E2E0000436F6E6E74
:104A3000656374696E670000446973636F6E6E65C9
:104A40006374696E67000000525353492043616EDE
:104A500063656C6C6564000041545420527370208F
:104A600064726F7070656420256400005265616433
:104A7000204572726F7220256400000052656164E7
:104A8000207273703A202564000000005772697428
:104A900065204572726F7220256400005772697438
:104AA000652073656E743A202564000046432056E5
:104AB000696F6C617465643A202564004D5455201B
:104AC00053697A653A202564000000005253534927
:104AD000202D64423A202564000000005061697274
:104AE000696E6720737461727465640050616972E5
:104AF000696E6720737563636573730050616972D3
:104B0000696E67206661696C3A20256400000000C8
:104B1000426F6E64696E67207375636365737300BB
:104B2000426F6E642073617665207375636365738D
:104B300073000000426F6E642073617665206661C9
:104B4000696C65643A20256400000000506173734D
:104B5000636F64653A20256400000000F0FF0000E8
:104B600053696D706C652053766320466F756E6473
:104B70000000000053696D706C6520424C45204375
:104B8000656E7472616C000000000000DFF800F0D8
:104B9000F5B80110DFF800F02DBF0110DFF800F0CC
:104BA00011BF011000B583B00821ADF800100190CD
:104BB0000521ADF80210684651490968884707BDCC
:104BC000F0B589B004460D4616461F460823242238
:104BD00000216846FBF71AFD0F984A4909680690BC
:104BE0006B464FF47A70B0FBF1F101FB07F00590D2
:104BF00001FB06F20E98ADF8100029462046FBF79F
:104C00002DFD204609B0F0BDFBF708BD38B50446C0
:104C10000D46FCF718FE10B12046FCF706FE00F02A
:104C20000CF800FB05F12046FBF7F4FC2046BDE83C
:104C30003240FBF7F3BCFCF7F8BD324909684FF48A
:104C40007A70B0FBF1F0704710B504460021FFF711
:104C50009DFF204610BD70B584B004460820ADF815
:104C600000000D460420ADF802000C20244909681C
:104C7000019016466846884758B9029949B18E6036
:104C80002046FFF787FF15B12846FBF7B7FC012048
:104C900003E03046FFF786FF002004B070BD10B57A
:104CA0000446FFF77BFFA04204D08468FFF77AFF39
:104CB000204610BD002010BD30B585B004466846C2
:104CC0000FF248011422FDF71DFA0F483021017040
:104CD000A21D782141700623811C12F8015D2D0967
:104CE0005B1E1DF8055001F8015B157805F00F05F6
:104CF0001DF8055001F8015BEFD105B030BD000093
:104D000054060020F48000006C2200203031323341
:104D100034353637383941424344454600000000B7
:104D200030B50446414D83B005F1300105F148002E
:104D300001F088F9A8600FF2810101F053FAA86828
:104D40003B4A00F035F8A8683A4A00F031F8A86804
:104D5000394A00F02DF8A868384A00F029F8A86808
:104D6000374A00F025F8A868364A00F01DF8A86810
:104D7000354A00F019F8A868344A00F015F8A86818
:104D8000334A00F011F8A868324A00F00DF800200C
:104D9000019000900023C8220FF2810105F10C0060
:104DA000FFF70EFF6C6037BD4FF0C05101F02ABA1B
:104DB0004FF4E02101F026BA10B51C4C0020207001
:104DC0000B2001F0DDF918B9207840F001002070C7
:104DD000132001F0D5F918B9207840F002002070B6
:104DE0000C2001F0CDF918B9207840F004002070B3
:104DF0000F2001F0C5F918B9207840F008002070A4
:104E0000122001F0BDF918B9207840F01000207090
:104E100004F10C00BDE81040FFF7F6BE03484168FE
:104E20000A001CBF0078084770470000C405002036
:104E30000B000580130005800C0005800F00058025
:104E4000120005800B000010130000100C00001071
:104E50000F000010120000102DE9F8430D0008BFEC
:104E60000FF2700504460027DFF8349000E07F1C45
:104E70000C2000FB07F859F8086076B1BC4203D05B
:104E8000B06980472042F2D0C84432682946404683
:104E900090470028EBD0404600E00020BDE8F283B8
:104EA000407B000010B103689B681847704700B949
:104EB000704710B586B00C9C04940B9C03940A9C1C
:104EC0000294099C0194089C00940468E468A0473B
:104ED00006B010BD0300000000B583B0ADF80000BF
:104EE0008DF806100020DFF80C130968ADF80200F9
:104EF0006846884710B99DF807000EBDFF200EBD1B
:104F00001CB5BD4C00B1606004F10800019004F1D3
:104F10001C00009004F10C03A2786078082100F0D6
:104F2000A1FB16BD70B5034600244FF48066104601
:104F30009B1B0A46B04D08D05B1E0CD05B1E12D0E6
:104F40009B1E15D05B1E1AD021E0102915D10146F9
:104F500005F10C0004E010290FD1014605F11C00F9
:104F6000FDF7C0F814E0042907D10068A8600FE03D
:104F7000012902D10078A8700AE0182408E038B1AD
:104F8000012905D10078032802DAE87000E0022444
:104F9000204670BD014698484078132200F090BB2F
:104FA000FEB5064694480F46417814461D465020EB
:104FB000FFF792FF8DF800008DF801608DF8027008
:104FC0008DF803400622294601A8FDF78BF86846B4
:104FD00000F069FBFEBDE0B5ADF80000ADF80210D1
:104FE000ADF80420ADF806300498ADF80800684626
:104FF00000F05DFB0EBD70B504467F480D4641785C
:1050000082B016465020FFF767FF8DF800008DF83C
:1050100001408DF802508DF80360684600F06BFB8C
:1050200076BD7548407800F06ABB00B58FB00823A4
:105030003C2200216846FEF7FBFE704800F150015B
:10504000079100234FF4DC7108916A460321069111
:105050000FF20901FEF7F0FE0FB000BDF0B585B00C
:105060000820ADF808000120624C634D2168ADF8BE
:105070000A0002A888479DF80C00687000F083FBC6
:10508000287005F10C021021022000F0F1FC05F15E
:105090001C021021032000F0EBFC05F108020421A2
:1050A000042000F0E5FC14E03078D02803D130462D
:1050B00000F042F80746002E18BF002F09D0082044
:1050C000ADF800000320ADF80200019668462168A3
:1050D00088470820ADF800000A20ADF802004FF024
:1050E000FF3001906846216888470028F1D10820E8
:1050F000ADF808000920ADF80A0002A82168884729
:10510000BDF80C109DF80E20049E0028E1D1012767
:10511000102904BF68788242CDD130884FF6FF71E4
:105120008842C1D170884004C5D505F10802042128
:10513000042000F0B2FCBEE73EB504462E4DA07838
:1051400040B105281CD0062823D00C2825D01128D2
:1051500028D045E06078002842D105F10C021021EA
:10516000022000F09AFC05F11C021021032000F03F
:1051700094FC0622E11C05F12C00FCF7B3FF2FE0A4
:10518000607868BB6289E0780823211D00F060F92F
:1051900026E0A08800F073F922E0217BA08800F0CF
:1051A00079F91DE0E878012810D1A088ADF8000059
:1051B000E088ADF802002089ADF804006089ADF800
:1051C0000600A089ADF80800012004E040B9A088DD
:1051D000ADF8000000208DF80A00684600F06CFA77
:1051E000686828B10168080002D0204688473EBDA3
:1051F00001203EBD5406002018060020B8190020EA
:10520000E0B50821ADF800100190022100F00FF880
:1052100008B100200EBD02980EBD00B583B0082174
:10522000ADF800100190032100F001F807BDADF8C2
:1052300002106846DFF8A813096808471FB5ADF8E3
:1052400006108DF804000824DFF894138DF8082068
:105250000393ADF80040ADF80240684609688847FE
:1052600004B010BD30B585B0144608220291ADF8E7
:1052700000201922DFF8681309680190ADF80220B8
:105280001D466846884714B1BDF80C10218015B141
:105290009DF80E102970089A0499116005B030BD70
:1052A00000B583B00820ADF800001A2000F015F812
:1052B00010B99DF804000EBDFF200EBD00B583B0EF
:1052C000ADF800008DF80610002000F006F810B9C7
:1052D0009DF807000EBDFF200EBDDFF8041309681E
:1052E000ADF802006846084750B110F1040F01D133
:1052F0000420704710F1030F01D1022070470120F4
:1053000070478123037042EAC111002341F47C41BC
:10531000C370818070478223037081800023C37033
:10532000827170473EB504460820ADF800000D4676
:105330002020ADF802001020DFF8A4120968ADF8B3
:1053400004006846884720B9029810B16FF0040045
:105350003EBD00950023002221464FF0FF30FFF7AD
:1053600081FF3EBD10B582B01446CA78012A03D130
:105370008A88DFF8F8341A8000F010F858B90090E5
:1053800069462046FFF7CEFF28B900984478FFF71A
:1053900044FF204616BDFFF7A7FF16BD0B460222AD
:1053A00010214BE738B51C461546FFF7F7FFC0B98B
:1053B000009069462846FFF7B5FF90B900984578F8
:1053C000280002BF0098C079A04205D100988168EA
:1053D00004982246FCF786FE0098FFF71EFF284639
:1053E00032BDFFF781FF32BDF8B500F04DFA00F095
:1053F000ADF907000DD032462946FFF78CFF00F0CB
:1054000076F93872FFF74CFF3B4601B0BDE8F0403B
:105410008AE0F1BD10220121E6E738B500F0ECF991
:10542000050002D00422012175E031BDF8B500F07D
:10543000DAF907000AD0132200F03BF800F045FB30
:105440003946BDE8F840DFF828248BE70420F2BD98
:105450002DE9F04100F059F907000FD0142200F0B7
:1054600028F83C72FD603E8287F81280FFF718FF33
:105470003946BDE8F041DFF8FC2373E71EE038B59C
:1054800000F041F8050004D0152200F012F82C813C
:1054900044E031BD70B500F0BAF8060008D016221D
:1054A00000F007F800F032F83346BDE870403BE00A
:1054B00070BD01212FE7002204217CE00420BDE81B
:1054C000F081102202218FE710B500F088FA040065
:1054D0000AD0112200F01DF8FFF7E2FE2146BDE8D8
:1054E0001040DFF894233DE7042010BD38B500F0EC
:1054F0000AF8050006D0122200F00BF800F0F7F8C9
:1055000028720BE031BD04460A2079E63481B57279
:10551000C6E60221FFE6FFF7FEFEAC60FFF7C0FE25
:105520002B4601B0BDE830400222102186E6002261
:10553000032140E000B583B00FF249030193062335
:105540000093032300F04EF80EBD1078802802BFB0
:10555000508840F27F61884208D19088984202BF0B
:1055600091790098814201D1012070470020704755
:1055700010B582B00624FFE70094FFF7E6FF16BDE2
:10558000000000000323F3E71078802802BF508852
:1055900040F27F6188420CD19088032818BF04280C
:1055A00007D1907901001CBF1028112801D10120DA
:1055B000704700207047F8B500F008FA07000CD0DB
:1055C00032462946FFF7A7FEBC60FFF769FE394661
:1055D000BDE8F840DFF8A422C4E60420F2BD0000D4
:1055E000540600202DE9F04100F035F807000AD0FC
:1055F000069A4146FFF78FFE3C817D8100F067FAF5
:10560000079A00F010BA59E7022300F0FFB80446E9
:105610000D460C20F4E52DE9F04100F076F8070086
:105620000FD0062200F015F83C81BE72FD6000F03C
:105630001BFA00F0DEF83946BDE8F0410FF25D32AA
:1056400090E63BE70A23E1E03423DFE01223DDE0CC
:105650004246032155E604460D461646984610205C
:10566000FFF7CEBD2DE9F04180460D4616461F4698
:105670001820FFF7C5FD040014D0002200F04CF8FC
:1056800000F0F2F920726572A672E7600698206158
:1056900007986061FFF704FE2146BDE8F0410FF274
:1056A00061225FE60AE70FF25D23092202E00FF2B2
:1056B000592311220021EBE00FF251231222F9E7C6
:1056C000F8B500F09DF807000FD00A2200F024F88A
:1056D00000F00DF838727D813E73FFF7E1FD394629
:1056E000BDE8F8400FF229223CE60420F2BD214635
:1056F0005020FFF7E3BD0FF21D230422DAE70FF27B
:1057000019230522FFE70021D3E004460D46164683
:1057100098461420FFF774BD0421FFF7F2BD70B561
:10572000FFF775FF06000BD03022FFF7F5FF00F002
:1057300009F83146BDE870400FF2E112FFF712BEE2
:10574000042070BD34817581FFF7AABD0A20FFF7E0
:1057500057BD7CB5044600208DF804000D460C2092
:10576000FFF74EFD06000BD01122FFF7A2FEFFF758
:10577000CDFE00F019F80FF2A9123146FFF712FE24
:105780009DF8040076BD1CB500F026F904000AD08F
:105790001222FFF78EFEFFF783FD00F005F80FF2EF
:1057A000891200F008F803E001A900910123704775
:1057B0009DF8040016BD2146FFF7F4BDF8B500F0D2
:1057C00012F807000DD03622FFF7A6FF3C817D813D
:1057D00000F07DF93946BDE8F8400FF25D12FFF7A1
:1057E000C1BD0420F2BD04460D4616461020FFF749
:1057F00007BD3874FFF754BD04460C20FFF700BD09
:1058000004460D4616460E20FFF7FABC2DE9F0417E
:10581000FFF77BFF07000FD0FFF71AFF3C81FD6009
:10582000314600F022F9FFF7E4FF3946BDE8F041C8
:105830000FF20912FFF796BDFFF740BE38B51446C8
:105840000F4A15682A0006D0009302460B462146EF
:105850000120A84732BD002032BD0A4A13681A0051
:1058600003D00A460146012018477047D40900209A
:10587000A1590000A7590000AD590000895500004A
:10588000401C0020441C002004460D46164670476C
:105890002DE9F041FFF7DFFE070004D000F005F826
:1058A000BC60FD60BCE0FFF709BE32460421FFF793
:1058B00028BD2DE9F041FFF7CEFE070006D0FFF727
:1058C000F4FFFFF714FF3872FD60A9E0FFF7F6BDA3
:1058D0001078802802BF508840F27F6188420CD146
:1058E00090884FF680710140B1F57E4F04BF00F003
:1058F0007F00984201D101207047002070470000CE
:105900000023E5E70923E3E71123E1E71223DFE7BB
:105910000A23DDE70423DBE70523D9E73023D7E7B4
:1059200080B5112302E0000080B51223009301230B
:10593000FFF70BFE02BD00003623C9E71078802870
:1059400002BF508840F27F6188420DD190884FF6A7
:10595000807101404FF68052914205D100F07F00E6
:10596000012801DB01207047002070471078802853
:1059700002BF508840F27F6188420DD190884FF677
:10598000807101404FF68052914204BF00F07F00C9
:10599000984201D101207047002070470623E5E7B7
:1059A00080B51323C2E780B51423BFE780B5112368
:1059B00000930223BCE700F015F802BD80B50FF29A
:1059C000910100F049F841F20540F4E704460D4624
:1059D00016460C20FFF714BC00208DF804000820A8
:1059E000FFF70EBC2DE9F041FFF74EFF98460E2061
:1059F000FFF706FC070009D000F00AF83D817E8120
:105A0000A7F80C80FFF74CFC069A0CE0FFF756BD98
:105A1000812038700120F870BC8070473D81FE60A5
:105A2000FFF73EFC42463946BDE8F041FFF79ABC1D
:105A30001078802802BF508840F27F61884204BFFE
:105A40009088984201D101207047002070470000E3
:105A500041F20543ECE700000091002301460022DB
:105A600070473C817D81BE8141465020FFF726BCB6
:105A7000F8B5FFF7B8FE07000DD0012200F022F8BC
:105A80003C727D7200F023F83946BDE8F8400FF211
:105A90007902FFF767BC0420F2BDF8B5FFF7A3FE5B
:105AA00007000DD0022200F00DF83C727D7200F06C
:105AB0000EF83946BDE8F8400FF25102FFF752BC2C
:105AC0000420F2BD0521FFF71CBC3C81BD72FE60C5
:105AD000FFF7E6BB1078802802BF508840F27F6154
:105AE00088420DD190884FF6807101404FF6806258
:105AF000914204BF00F07F00984201D1012070471D
:105B000000207047000000000123E3E70223E1E7E3
:105B10001CB500200190FFF762FF04000BD00522A6
:105B2000FFF7D0FFFFF7BCFB01A9009104230FF2A0
:105B30000D02FFF740FE019816BD00000523C9E7DE
:105B4000DFF800F055C0011038B50FF24100394CB4
:105B5000394D00F0BDFB394800F0B5F923681B68EA
:105B600001220121284698472268526801212846CF
:105B7000904700F001FD00F01DFDFFF756FAFEF71B
:105B80008CF9FFF7DDFF002032BD000070B52C4E10
:105B90000446306886B00D4628B900214FF0004019
:105BA000FFF75AF9306000F05CF80FF2DC030021D7
:105BB000FFF77DF930680FF2E003022C0BD0042CC4
:105BC00002D0052C1CD027E000F054F800F042F879
:105BD0000FF2D0030EE0012D06D100F04BF800F0DB
:105BE00039F80FF2D40305E000F044F800F032F881
:105BF0000FF2DC03306800220221FFF758F916E0AB
:105C000000F038F800F02DF80FF2D8030221FFF76A
:105C10004EF900F017F80AE000F02CF800F021F837
:105C20000FF2D0030221FFF742F900F00BF806B0A3
:105C300070BD0000D801001000400340387A000019
:105C4000B006002001208DF800009DF8000000281B
:105C5000FBD17047002004900390029001900090C7
:105C60007047002004900390029001900090002261
:105C700030687047002104910391029101910091D5
:105C80000022FFF714B900003E3E3E535441434BFF
:105C900020415353455254002A2A2A4552524F520A
:105CA0002A2A2A003E3E204F5554204F46204D457B
:105CB0004D4F5259210000003E3E20494E5445525E
:105CC0004E414C204657204552524F522100000071
:105CD0003E3E20494E5445524E414C204552524F73
:105CE000522100003E3E204943414C4C2041424F4E
:105CF000525421003E3E2044454641554C542053C9
:105D000050494E4C4F434B2100000000030000203F
:105D100013F0030F09D0521E22BF13F8010B11F824
:105D200001CBB0EB0C00F3D07047121F22BF53F829
:105D3000040B51F804CB6045F7D0121D0AD200BA0B
:105D40009CFA8CFCB0EB0C0038BF6FF0000088BFF1
:105D500001207047521E22BF13F8010B11F801CB2E
:105D6000B0EB0C00F6D0521C08BF10467047000084
:105D700070B5FBF774FD04460026DFF808550DE00A
:105D800024FA06F0C00708D505EB8600406820B16C
:105D9000026811001CBF31469047761C2868F6B295
:105DA0008642EDD370BDDFF8E0040168DFF8DC0463
:105DB0000160DFF8DC04FBF762BD2DE9F0470E005F
:105DC000F5B2044644BF86F0204686F4C046A800DB
:105DD00000F1804000F5012004EA06030168DFF8C5
:105DE000B4743B4086EA0102A1431943224004F403
:105DF000E023120EB3F5E02F02F0010202D1CA0136
:105E000005D411E014F4E02F08BF002A0CD001F4EF
:105E1000E022B2F5A02F04D0B2F5C02F04D10522A4
:105E200000E0062262F31241DFF86C74016038680A
:105E3000E84000F0010805F1804000F50839B00D98
:105E4000B8F1000F00F0010A03D1600248BF89F8E1
:105E500000A020020DD5FAF7C9FB0122AA4039683B
:105E600033024CBF13460023914319433960FAF7BC
:105E7000C1FBB8F1000F03D0600248BF89F800A051
:105E8000BDE8F087002948BF0021800000F1804074
:105E900000F5012001F03F010268920941EA8211F8
:105EA0000160704710B5DFF8F403006800F07F046C
:105EB000FDF71AFD012804D1FDF70CFD022808BFEB
:105EC000641C204610BD2DE9F04FA1B00546FCF73B
:105ED00094F9FDF709FD0026012804D1FDF7FAFC2D
:105EE000022808BF0126DFF8B803C168C1F3815159
:105EF00001294FF0010A04D10068000E0AFA00F0EF
:105F00000643DFF8A003DFF87C930078DFF898738E
:105F1000FFF7C8FF5FEA000BC9F800B004D0FF220A
:105F200059463846FDF7B8FC4FF00008002405E05C
:105F30000AFA00F07C5440EA0808641C55F8240072
:105F400000F0FF01FE2909D0FF29F6D0594503D200
:105F500026FA00F2D207EBD5022070E00920FCF708
:105F60004AFAC9F8805008232422002117A8FAF71A
:105F700059FB8DF874A017AA012109F1D400FAF792
:105F800055FB0024DFF824A30BE05046FFF715FF74
:105F90004FF0FF31E0B2FFF775FF0020CBF80400AF
:105FA000641CD9F80000844213D226FA04F0C0071A
:105FB00009EB840B48BF0420F0D428FA04F0C00792
:105FC00047BF385D55F8201004F0FF0040F4C04191
:105FD000DBE70823302200210BA8FAF72BFBDFF8C0
:105FE000D052DFF8D022287813900BAB002000901D
:105FF000102109F18400FAF721FB0823282200214F
:1060000001A8FAF71FFB6868DFF8AC1207900023BD
:106010000020089001AA09F1A000FAF717FBDFF8A9
:106020009C02016821F47C5141F40051016001207F
:10603000DFF88C120860DFF88C120860002021B0B5
:10604000BDE8F08F2DE9F0418E4E04460D4606F175
:10605000D40800F05EF8002035B9002020606060B0
:10606000A06085B125E0401C15F82010FE29F4D071
:10607000FF29F8D03268914204D206EB81014968C9
:106080000029F0D000244046FAF7B8FA2046BDE8CF
:10609000F08106EB81020123546003FA01F162688A
:1060A0001143616055F820208049204600F0AAF88D
:1060B000384615F82010FE29E5D0471CFF29E8D105
:1060C000F6E72DE9F04105000E46F7B203D06D4C1E
:1060D0002068874201D3022019E004F1D40800F0BF
:1060E00018F804EB8700416809B101250BE0456011
:1060F00001216868B9400843686032466B49284608
:1061000000F080F800254046FAF778FA2846BDE806
:10611000F0814FF0FF314046FAF774BA10B50C46E3
:10612000F0B1416821FA04F2D20719D50122A24048
:10613000914341600020534901EB840250605A486A
:10614000025D5A48FF2A0EBF44F02041D1F880106A
:1061500051F82210FFF731FE4FF0FF3120468DE05D
:10616000022010BD10B5044606E090FAA0F0B0FA87
:1061700080F12046FFF7D2FF60680028F5D110BDFE
:10618000514915E010B53F4B1C68A14204D203EB06
:1061900081035B68834201D0022010BD01F1804180
:1061A000100001F5083118BF01200870002010BD53
:1061B0000968C14001F00100704710B5314B1C68FF
:1061C00001F0FF02A24204D203EB82025268824233
:1061D00001D0022010BD0A464FF4E02100F012F871
:1061E000002010BD10B101600020704702207047F0
:1061F00080B500F01CF880F0005080F4C04040F002
:10620000004002BD38B51F4C25680B46114601F011
:10621000FF02AA4204D204EB82025268824201D0F9
:10622000022032BD1846FFF7C8FD002032BD8100B4
:1062300001F1804101F50121164A09681140234A04
:1062400013680143C340DB07126D48BF41F480016E
:10625000C240D00748BF41F40001084670470B46D2
:1062600010B51146074A1468A34204D202EB830218
:106270005268824201D0022010BD1846FFF702FE8C
:10628000002010BD481C0020E0200240E0200260F9
:10629000E81C0020007F077FD020024044130050FC
:1062A000A83F00507F230020381D0020007FC767D3
:1062B000847A0000A75D0000715D00000030094095
:1062C0000C40094008000940C020024080200240E4
:1062D0000149086070470000C005002081B001201E
:1062E0008DF800009DF800000028FBD101B0704738
:1062F00070470000DFF800F0ADB50110DFF800F0E6
:1063000019AE0110DFF800F0E5C10110DFF800F070
:1063100085C20110DFF800F081C20110DFF800F043
:1063200055C10110DFF800F043C20110DFF800F0A2
:1063300079AB0110DFF800F0D9B60110DFF800F0FA
:10634000EDB3011020B108232C22002118F05CBE0F
:10635000704720B108233C220021FDF769BD70473A
:1063600080B5FBF7FBFEADF80000FAF73FF9ADF89A
:106370000200009802BD01B5BDF80200FAF73AF933
:10638000BDF80000BDE80240FBF7ECBE38B5DFF811
:10639000A008DFF8A018DFF8A04880088000091ADC
:1063A0002161E060034602E0002523F8025B0D183E
:1063B000AB42F9D38B0800EB8303002223F8042CB3
:1063C000E82202804FF6FC721140EC39A0F8E81088
:1063D000E8306060002000F004F8A060E0686060D1
:1063E00031BDF8B500240025061D16F003001CBFC2
:1063F000311D0E1AFFF7B4FFDFF83C28B6B210606B
:10640000112EB4BF576897683A88130403D582F4F5
:10641000004200251AE02B0014D0238839880B4451
:1064200023809BB2B34211D327461A46B7B1921BC1
:1064300092B2042AA7BFBA5346F40041398841F406
:10644000004109E0B242F1DA01253C4617443A889E
:10645000002ADAD1002701E027F8041BFFF78BFFA1
:106460003846F2BD10B50446FFF77AFFDFF8C817CB
:10647000086034F8042CC2F30E0224F8042C221F06
:106480004B689A4238BF4A60BDE8104073E738B5A0
:106490000446FFF765FF00210C23DFF8A0274B43DC
:1064A000D518AA6C4AB1944204D1FFF764FF05F1F4
:1064B000480032BD491C0329EED3FFF75CFF0020E2
:1064C00032BD70B50546FFF74BFF044600200C2295
:1064D000DFF8681742438E18B16C49B90020306567
:1064E000B5640022FFF706FFF06418B918F096FDB6
:1064F0008D4205D12046FFF73EFF06F1480070BDF2
:10650000401C0328E3D32046FFF735FF002070BD71
:1065100038B50446FFF724FF0025DFF820170C22CA
:106520006A438A5A130008D0944203D1FFF723FF2D
:10653000E8B232BD6D1C062DF1D3FFF71CFFFF2022
:1065400032BD10B504462088FFF7E2FFFF2800D1D6
:106550006BE10C22DFF8E416504308448168080020
:1065600002D16FF0010010BD2046BDE81040084781
:1065700002460FF23870104710B500200C21DFF8EA
:10658000BC26002401FB00F31344401C03289C6438
:106590001C65F7D30020002301FB00F4401C1353BB
:1065A0000628F9D3082010800FF2E9609060BDE85A
:1065B0001040EBE670B590B0FBF7D0FD044668469E
:1065C000FFF7C7FE05200690002240F2B630089083
:1065D00069464DF651200490DFF864060590DFF817
:1065E0006406FFF78BFE050006D0FFF7B9FE0646EE
:1065F0002846FFF766FF08B918F010FD3046FFF790
:10660000BAFE2046FBF7AEFD10B070BDF8B500F045
:10661000E6F8FFF756FF05006FF0020616D0FFF709
:106620009FFEA28800210C27DFF810364F433B4421
:106630001F883FB91A805D60A2689A6021736968FB
:106640002161C4E2BA4203D1FFF795FE3046F2BDA4
:10665000491C0629E7D318F0E1FC00BF38B500F06B
:10666000BEF8FFF72EFF050016D0FFF779FE0021D8
:106670000C23DFF8C8254B431A4413884BB94FF657
:10668000F873138055600023936021716968A160DD
:1066900013E7491C0629EBD318F0C0FC00BF10B566
:1066A000044660680C3080B2FFF79BFE00B91AE028
:1066B0006168018100210160FF2181720C30A060BE
:1066C000002010BD80B540680C3811E080B288E62B
:1066D00010B50446606880B2FFF783FEA06000B981
:1066E00001E0002010BD6FF0030010BD80B54068D0
:1066F000FFF7B8FE002002BD38B504460D46FFF78F
:106700002FFE002145F80C1C216811B9256006E018
:10671000114651F80C2C002AFAD141F80C5CBDE866
:10672000324028E62DE9F04104466FF00206E068A9
:10673000A0F10C05A0790628BCBF207906280BDA49
:10674000FFF70EFEA179DFF8F4840C27794341446A
:10675000496819B9FFF70FFE304617E0FFF70BFE47
:1067600020792871A0796871207AA871A079E168F0
:106770007843404440680830FFF7BEFFA079784373
:10678000404440684068F9F739FF0020BDE8F081D7
:1067900070B500F024F8FFF77AFE060002D16FF022
:1067A000040070BDFFF7DCFDB168002541B10D4666
:1067B000A5F10C010A68B26000220A60FF228A7209
:1067C000FFF7D9FD2800A56001D1022070BDA5F119
:1067D0000C00017921714079A071002070BD044640
:1067E000FFF790BD06280ADA0C23DFF8502458433F
:1067F000105A02001CBF4FF6F872904202D14FF0BF
:10680000FF307047088000207047811D0079E9E75C
:1068100010B50446E088FFF77BFEFF2800D104E0B6
:10682000A0712046BDE810407CE74FF0FF3010BD5E
:106830003EB50446FFF7ACFF050017D12079694645
:10684000FFF7D0FF78B10820ADF804000320ADF8C1
:106850000600DFF8F413A0688968029001A8884751
:106860006FF005003EBDBDF80000A08028463EBD8B
:1068700010B5DFF8D82312680C464FF47A71A1FBEB
:1068800000010023FCF7DCF9002399424FF000429D
:1068900001D8904202D36FF0020010BD20600020AA
:1068A00010BD38B5FFF79BFFFFF7F1FD0546FAF77E
:1068B0005AFF002818BF012800D015B96FF0040056
:1068C00032BD606840B9009000996868F9F79AFE97
:1068D000401E8041C00F32BD10F1010F08BF4FF0C4
:1068E000FF30F0D06946FFF7C3FF0028ECD032BD7F
:1068F00080B54068F9F782FE002002BD18F08EFBDB
:1069000000BF80B54068FFF701FD002002BD80B5E3
:106910004068FFF7FFFC002002BD80B5FFF7FEFCDA
:10692000FFF700FD002002BD80B5FBF717FCF9F76B
:106930005DFE002002BD10B58CB004466846FFF72E
:1069400001FDE02000F013F808B918F067FB0BE038
:1069500010B58CB004466846FFF7F4FCE06800F020
:1069600006F808B918F05AFB00200CB010BD0890CA
:106970000023A16860686A46FFF7D8BC10B50446DA
:10698000FFF7D8FC6060002010BD014688684968A8
:106990000847F0B507468BB0BC68AB4D6CBB0C200C
:1069A000FFF71FFD04006FF003061ED0082324220A
:1069B000002101A8F9F72AFE0020ADF81400069086
:1069C000079400237968A24801AAFFF7B7FC20606A
:1069D00068B90820ADF800000C20ADF80200684648
:1069E000A96888472046FFF73DFD304618E0F86863
:1069F00060603869A060BC600AE02868804706468D
:106A00002068FAF712FF3869A06030466968884745
:106A100079682068F9F7FEFD2068F9F7FFFD00208E
:106A20000BB0F0BD10B5044682B060686946FFF750
:106A30001FFF20B9009860602046FFF7AAFF16BD2F
:106A400080B5406810B96FF0020002BD0068FAF727
:106A5000ECFE002002BD7D490968416000207047BE
:106A600050B50446794802686FF00046A6FB020163
:106A700000234FF47A72FCF7E3F8002399424FF0B9
:106A8000004201D8904200D330466060002050BDE3
:106A90002DE9F04186B00646FFF734FCFFF7F7FC1E
:106AA0000446002002900025FAF75DFE002818BF7A
:106AB000012800D014B96FF0040063E0706820B1C1
:106AC00010F1010F03D14FF0FF30009004E0694650
:106AD000FFF7CEFE070054D1FFF72CFC00990127E9
:106AE00001EB000800E0009000996068F9F78AFD6A
:106AF00078B303A8FFF74CFE07001AD19DF81000E9
:106B000001A9FFF76FFE80B9059A9DF81210BDF834
:106B10000400B368984740B1BDF80400B0819DF807
:106B20001200B0730598306113E0059902A8FFF7D1
:106B3000E3FD009801276D1C10F1010F18BF00281C
:106B4000D2D0FFF7F7FBB8EB000002D000998142EA
:106B5000C9D2029EFFF704FC56B1314600E011464F
:106B600051F80C2C002AFAD1A26841F80C2CA6602E
:106B7000FFF701FC002D03E06068F9F73FFD6D1E93
:106B8000FAD1384606B0BDE8F081F8B5FFF727FE28
:106B90000546FAF7E8FD002818BF01286FF0040643
:106BA00013D0FFF7DDFB0021244A0C234B43D75AB7
:106BB0004FB113445B681B68AB4201D1217106E001
:106BC000491C0629F1D3FFF7D6FB3046F2BDFFF78B
:106BD000D2FB0020F2BDF8B50446FAF7C4FD002848
:106BE00018BF012802D16FF00400F2BDFFF78AFB45
:106BF0000546FFF7B5FB0021104A0C234B43D65A3C
:106C000037000ED0A788BE4208D1D118496809685C
:106C1000A9420CBF01210021A160D8E7491C062927
:106C2000EBD3FFF7A8FB4FF0FF30F2BD00000000F0
:106C300084230020183F00202C1C0020C01B0020B3
:106C400060060020716500004C060020F480000002
:106C50008B69000070B504463C20FFF7C2FB0500BD
:106C60006FF0030611D0FFF774FB207AA8610022B1
:106C7000608928622946E06828616068FFF73EFB6A
:106C800004462846FFF7EEFB0CB9304670BD0020E5
:106C900070BD000041882D2902D36FF001007047BC
:106CA0000FF2140252F8211008470000436500005B
:106CB00061630000776300000D6600005D66000000
:106CC0009F660000C5660000D1660000ED6600000A
:106CD000256700009167000011680000316800001E
:106CE000A3680000F1680000FD680000036900006F
:106CF0000F6900001B690000296900003769000066
:106D00007D690000256A0000576A0000616A000082
:106D10000B680000677700003B780000916A000074
:106D20008B6B000093690000416A0000D57700007A
:106D30000D78000021780000D76B00006D7800000E
:106D400085780000556C0000000000000000000085
:106D50007B7800009378000051690000000000007B
:106D60000000000000000000000000004068006813
:106D7000012140F84C1F7047F0B52A4C6568266821
:106D80008DB02879FBF737FBF9F730FC07463078F0
:106D9000A8B908233022002101A8F9F74BFC06947A
:106DA00001ABA879204A099000200090301D697934
:106DB000F9F744FC01203070204600F024F83846F2
:106DC000F9F718FC20460DB0F0BD70B544680568B1
:106DD000F9F70CFC0646287880B12079FBF7E9F931
:106DE000012808D12168002041F8040F281D18F05F
:106DF00019F9002028702079FBF792FA3046BDE897
:106E00007040F9F7F7BB40680268002142F82C1F78
:106E10000068064900F108021160012140F8041FD2
:106E200070470000A47A00006D6D0000000400208F
:106E3000DFF800F06DA9011070B50568AE6A002496
:106E400006E0242000FB0460083018F0F3F8641C0E
:106E500095F82C00E4B28442F3D3686800F0E8FAB5
:106E6000DFF868020068FFF77DF90020288070BD18
:106E70004FF0FF310160DFF85C12416000210172C8
:106E800070472DE9F043DFF8489299B0D9F80050E7
:106E9000D9F80470044688461646F9F7A7FB2988F6
:106EA000012902D1F9F7A6FB0DE001212980F9F7AC
:106EB000A1FB1EB904A8FFF7DBFF04AE002C18BF2E
:106EC000B8F1000F01D100205BE010A800F0C8FA73
:106ED0007068149010A9307A8DF85800F87900F095
:106EE000AAFA00284DD0686008233068A860AC6218
:106EF00085F82C802422002107A8F9F793FB0026AF
:106F000008E0242000FB064007AA01210830F9F719
:106F10008DFB761CF6B24645F3D301208DF8340084
:106F200007AA012105F10C00F9F780FB3979DFF898
:106F3000A801DFF89841014300916946BA791043EE
:106F40004860DFF89821787910438860FE20C86097
:106F5000201DFFF777F8206098B1DFF88411DFF883
:106F600084010968B0FBF1F0FFF762FF79792068CE
:106F70000122FFF707F939681122484600F078F836
:106F8000484619B0BDE8F083026892F82C2091427F
:106F90003CBF012200F0DBB87047006890F82C205D
:106FA000914200D3704770B508302423026A5943D8
:106FB0008B188D5801685C6803F108063046F9F7B4
:106FC00021FB48B11CB12146284600F061FA304649
:106FD000BDE87040F9F712BB70BD2DE9F8430068B9
:106FE000154690F82C20914228D200F10802242462
:106FF000106A614351F80080089C081800F10809E4
:10700000099811685E1B071B00F01DF9F6B2FFB26C
:10701000A0B10020844607E05A185B1C02F808C0A3
:10702000DBB29E42F8DA401CC0B2874205DB011990
:1070300005EBC11189B20023F2E714E0BDE8F1834A
:107040001CB500F00BF803D200F003F800F0B2F822
:1070500013BD01240194049C00947047046894F8C3
:107060002C40A14270474846BDE8F243F9F7C6BA42
:107070002DE9F04100F022F800F01DF800F019F8B9
:1070800000F013F800B12FE0BDE8F0812DE9F041E8
:1070900000F014F80122FFF775F800F00AF800F08C
:1070A00004F800B120E0BDE8F081424629462046C0
:1070B0003DE0B97930680022FFF764B80446034E1A
:1070C000676830680D469046397970474C23002038
:1070D0002C7B000040420F000000C0800000808038
:1070E000F4800000A0860100B9793068BDE8F04165
:1070F0000122FFF747B838B50FF2581425680095FC
:1071000001F00F049DF80030D2189DF802308DF880
:107110000020E3188DF8023003229DF8013003EBC4
:1071200011118DF801106946FFF7A2FF31BD00B5BE
:1071300085B0002303930092029301916946006891
:10714000406800F092F900B1012005B000BD2DE9C2
:10715000F84381461500D9F800600F4605D0B168A4
:1071600006F10C00F9F74EFA10B3B06A2421794306
:107170000F58081800F1080825B1B1684046F9F722
:1071800041FA90B10024224600214846FFF7B3FFA0
:10719000802207EBC4114846FFF778FF641C082CD7
:1071A000F1DB2DB14046F9F729FA06F10C005BE757
:1071B000BDE8F1832DE9F84F064615460C461F46FB
:1071C000284600F069F980460A9807EBC0101FFABC
:1071D00080FA3068826A242161438E580B9C89189A
:1071E00001F108091CB1816800F02DF830B30027C7
:1071F0000FF2640B12E0213A02EB820292B20023FA
:1072000003EB020C03EB010E1CF80BC00EF806C0DA
:107210005B1C052BF4DB002141717F1C47450ADA1A
:10722000062000FB07A17A5D8819202AE3D10621F8
:1072300000F02EF9F1E70CB1484607E0BDE8F18F08
:1072400001F1080901684846F9F7DCB9BDE8F24FD9
:10725000F9F7D4B9B010000000005F00000007008B
:107260000700147F147F14242A7F2A122313086432
:107270006236495522500005030000001C224100DF
:107280000041221C00082A1C2A0808083E080800A1
:107290005030000008080808080060600000201056
:1072A0000804023E5149453E00427F400042615180
:1072B00049462141454B311814127F102745454559
:1072C000393C4A4949300171090503364949493673
:1072D000064949291E0036360000005636000000D7
:1072E0000814224114141414144122140800020139
:1072F000510906324979413E7E1111117E7F49497B
:1073000049363E414141227F4141221C7F49494942
:10731000417F090901013E414151327F0808087F40
:1073200000417F41002040413F017F081422417FFE
:10733000404040407F0204027F7F0408107F3E41AE
:1073400041413E7F090909063E4151215E7F0919ED
:107350002946464949493101017F01013F404040EA
:107360003F1F2040201F7F2018207F6314081463D4
:107370000304780403615149454300007F41410201
:107380000408102041417F00000402010204404033
:10739000404040000102040020545454787F484487
:1073A00044383844444420384444487F3854545482
:1073B00018087E090102081454543C7F080404781C
:1073C00000447D40002040443D00007F10284400E0
:1073D000417F40007C041804787C08040478384419
:1073E0004444387C14141408081414187C7C0804D1
:1073F00004084854545420043F4440203C4040205A
:107400007C1C2040201C3C4030403C442810284438
:107410000C5050503C4464544C4400083641000029
:10742000007F00000041360800003E1C08000000FC
:10743000016809680847084A1268904201D3002091
:10744000704709B90FF228010C224243034B9818E8
:107450009A58D26810470000F8060020EC7A000025
:107460000FF20C012022FAF74DBE02681269104794
:1074700000000000FFFFFFFF000000000000000010
:1074800040420F0008000000000000000000000063
:10749000002200F00BB80000002100E0491CC9B236
:1074A0000A5C002AFAD1084670470000401810F024
:1074B000030308D0C91A1FD3DB0748BF00F8012D0A
:1074C00028BF20F8022D130030B414461546103999
:1074D00028BF20E93C00FAD8490728BF20E90C0062
:1074E00048BF40F8042D890028BF20F8022D48BF6E
:1074F00000F8012D30BC7047C91818BF00F8012DE5
:10750000CB0728BF00F8012D704701680A680A44BC
:1075100082604B681A44C26008310160704781681C
:10752000C268914208D101680A680A4482604B68C7
:107530001A44C260083101608168491C816011F8F9
:10754000010D704738B504460D46A068E1688842D1
:1075500012D120686168884208BF17F05FFD20687B
:10756000227C016802B14944A16042680A44E26099
:10757000083091422060ECD0A068401CA06000F868
:10758000015D31BD2DE9F0418AB000F1080105919E
:107590000268520801EBC20106910021079108918F
:1075A0000168490800EBC10108310091017901F03F
:1075B00001018DF8101040680099400801EBC000EF
:1075C000019000200290039006E005A8FFF79DFFC0
:1075D00007980899884207D1059806998842F4D1FE
:1075E00001980AB0BDE8F08105A8FFF798FF0446AE
:1075F00014F0030603D105A8FFF791FFC61C250967
:107600000F2D14D105A8FFF78AFF00F10F050EE03A
:1076100007980899884204BF05A8FFF776FF0798E6
:10762000401C079010F8011D6846FFF78BFF761E7F
:10763000EED1002DCCD005A8FFF771FF0646A008BB
:1076400000F00300032804BF05A8FFF768FFDDF87A
:1076500000800299039F06EB002008E0A8F10808CB
:10766000A8F10801801A0A6849685718394658F87D
:10767000082C8A1A8242F1D340420C18AE1CA7D0C3
:10768000BC4206D158F8044B58F8040B2718BC42EA
:10769000F8D00298039914F8015B884217D100983A
:1076A0000199884208BF17F0B9FC009800689DF85E
:1076B0001010029009B1484402900099029849685C
:1076C000009A01440832884203910092E7D0029860
:1076D000401C0290761E00F8015D3FF479AFCFE7C1
:1076E00080B501280CD002280CD0042802D008282C
:1076F0000AD00BE00020114612689047002002BD1E
:107700000220F8E70420F6E70520F4E717F086FCEE
:1077100000BF10B5044601E0FAF758FEB4FA84F051
:10772000202800D110BD00F016F8F5DB401FFAF755
:1077300062FEF3E710B5044601E0FAF7DDFDB4FAA6
:1077400084F0202800D110BD00F005F8F5DB401FC3
:10775000FAF7E6FDF3E7C0F11F00C0B20121814056
:107760004C400528704738B50546012068713D4CEE
:107770002879A8B1FEF7F4FD05462078FF2805D149
:107780002846FEF7F8FD6FF0060032BD401C207061
:10779000C0B2012804BF6068FFF7BBFF284615E0B0
:1077A000FEF7DEFD21780A0004D1FEF7E4FD6FF05C
:1077B000070032BD491E2170C9B239B9FEF7DBFDA1
:1077C0006068FFF7B7FF0020687101E0FEF7D3FDA6
:1077D000002032BD70B50446606810F07F4F02D0C3
:1077E0006FF0020070BDFEF7BBFD1E4E05463078FF
:1077F00028B17068FFF79EFF6068FFF78AFF606836
:1078000070602846FEF7B7FD002070BD80B5406867
:1078100010F07F4F00D00DE0FFF77BFF002002BD8E
:1078200080B5406810F07F4F00D003E0FFF782FF83
:10783000002002BD6FF0020002BD10B5044682B008
:10784000A168606808601420FEF740FF009010B93E
:107850006FF0030016BDA368034A0F21FAF73CFD41
:10786000002016BD58060020E176000010B5044641
:10787000FAF739FF2071002010BD80B5FAF744FFF8
:10788000002002BD10B50446FAF7A7FC6060002096
:1078900010BD10B504466068FAF723FFA060002011
:1078A00010BD0000F0B5044685B0A0686568007999
:1078B0000E460021FE2803D01C49084300900421F5
:1078C000FE204DF8010069462846FEF7BBFB05F196
:1078D0000C07386038B33078387205F2344605F159
:1078E0003400306005F118014FF4806070601C2294
:1078F00005F23C40FAF706FC02A8FFF7B9FA02AA23
:1079000001213046FFF7BDFA786040B10021FFF752
:1079100044FB78680021FFF737FB204603E0386816
:10792000FEF720FC002005B0F0BD00000008C0807C
:1079300010B54468206930B10021FFF72EFB2069A3
:10794000BDE8104012E010BD1CB544682069134624
:107950008B4238BF0B4630B1019300917F23002248
:107960000021FFF73AFB2069BDE81C400021FFF72A
:107970000BBBF0B58BB047680D4614461E4604A8F5
:107980001821FBF7ADF806204443387D2346012833
:107990001A4605D005D303282AD038BF7F2300E03C
:1079A0000022D0B2D9B2884207D001950095DBB24F
:1079B0003869D2B20021FFF710FB1498109B039096
:1079C0003246139802901621129801901198009057
:1079D00004A800F024F80095E3B2386904AA002155
:1079E000FFF72EFB38690021FFF7CEFA0BB0F0BD90
:1079F00000227F23D9E710B54468E06840B1FEF764
:107A0000B1FB0020E0602069FFF716FA002020613A
:107A100010BD6FF0010070474FF0004070470CB48C
:107A200080B502AF3A6827F003031B1DFAF741F84F
:107A3000BDE8804002B07047190880801B08808034
:107A400007088080060880800B2000C0132000C03B
:107A50000C2000C00F2000C0122000C00D0080804C
:107A60000400C0800500C0800E00C0801A00808025
:107A7000140080801800C0801E00C0800300C080F9
:107A8000FE000000FF0000000000000000000000F9
:107A9000AD7C00008D2600000101010000000240C5
:107AA0000A29FF00581300209C7A00000000000003
:107AB000000000000000004017FF00000000000070
:107AC00004000000080000001000000009080AFF80
:107AD0000080004018FF00000000000005000000CA
:107AE000000001000000020017181EFF6480000063
:107AF00078130020B47A0000648000005414002041
:107B0000D07A00000000000000000000000000002B
:107B100040A1C0A6A22FF800278116AC00AFB0107C
:107B200000000000107B000004050E00301500204E
:107B3000247B0000FFFF05052C7B00000D000000EA
:107B40004880000060150020387B00000000000025
:107B50000000000000000000080000007A23002060
:107B6000587B0000000000000000000080B5F8F71E
:107B70003DFD36490A7822B9354B1B681A7001223F
:107B80000A7080B2BDE80240F8F734BD38B5F8F7A6
:107B90002DFD04462E4D284600F064F8A0B2F8F7FB
:107BA00029FD284632BD70B50E461446F8F71EFD75
:107BB00085B227480168097809B900F053F826B959
:107BC0004FF480710122084612E0304600F027F899
:107BD00058B114B14FF0FF3020700820FAF7A0FB25
:107BE0002846F8F707FD002070BDB268716830685C
:107BF00000F042F817490120086017480068C007E4
:107C0000FBD50220154909684968884706460CB12A
:107C1000002020702846F8F7EDFC304670BD4FF08C
:107C2000FF3180B102681AB1403AB2F57F5F0AD2E3
:107C3000426822B1A2F58072094B9A4203D2806851
:107C4000102838BF00210846704700007E2300201E
:107C50005C7B0000A802504208800240CC0100106A
:107C600000FFFF0001680A782AB901220A70406803
:107C70000068FAF7C0BB704710B50A4B1C6824F4C3
:107C800080641C6009021202090CA4B202F4706242
:107C900044EA014442EA0141C0F387101C600843F2
:107CA000586010BD1480024030BF704738B5FBF7F4
:107CB0008DFBFBF73DFBFAF778FA044604F00C0065
:107CC0000C2849D0600721D4F9F752FD054601215F
:107CD0000120FAF774FA2349096801FB05F2904282
:107CE00014D28220B0FBF1F01F4C291A04F10C00D1
:107CF000F8F790FC04F10C00F8F790FC0120FAF77B
:107D0000D2FB04F10C00F9F790FD27E0200723D403
:107D10001648FBF707FA0428FAD0E206144900D403
:107D200018B9086840F0010002E008684008400007
:107D30000860104C1048114D016841F003010160CA
:107D4000202021688969884728682068806B8047DF
:107D500001202860286801E0FFF7A6FFBDE8314058
:107D6000FBF738BBF4800000BC0800200040034053
:107D70008C210840B8010010242208402C20094022
:107D8000EBC70CEEC90CF1CB0CF44B14F74E19FAFF
:107D9000521DFD582500613101144202184E031C8A
:107DA0005A04249305309300807D00000D070000E5
:107DB000C7100000DD620000E1110000DD6200007C
:107DC000DB130000291400002B140000DD6200000A
:107DD000DD620000BF150000D5150000DD62000067
:107DE000DD620000DD620000DD6200008D11000038
:107DF000E915000033160000711600006D7B0000CD
:107E00008D7B0000A77B00007B756E6B6E6F776EBD
:107E10002D696E7374616E63652D6E616D657D0095
:107E20007B656D7074792D696E7374616E63652DF9
:107E30006E616D657D0000007B7374617469632DF4
:107E4000696E7374616E63652D6E616D657D000092
:107E500019E050F8041BCB0744BFA9F101035918DE
:107E6000121F0023042A41F8043BF9D25FEA827C06
:107E70000B4604D54FF0000CA1F800C09B1CD107A5
:107E800044BF0021197050F8042B002AE1D170473B
:107E900010B5074979441831064C7C44163404E087
:107EA0000A68081D114488470146A142F8D110BD57
:107EB0002C0000006C0100007FC80110C9BC01103B
:107EC00051B2011037C20110BDAD0110C1B1011096
:107ED00071BA011069BB011021C0011075FFFFFFCD
:107EE000A8190000D80900200000000099F6FFFF43
:107EF0000200000002000000100400001800000052
:107F0000780100202C0000007DF6FFFF0200000039
:107F1000020000004104000003000000EC0100200A
:107F20000400000061F6FFFF0200000002000000F4
:107F30001F04000003000000F00100200800000002
:107F400045F6FFFF0200000002000000D40300001D
:107F50001A000000A40100202400000029F6FFFF01
:107F60000200000002000000D20300000C0000002C
:107F7000C80100201C0000000DF6FFFF02000000F9
:107F800002000000470300001B0000000001002069
:107F900044000000F1F5FFFF0200000002000000B5
:107FA000B8030000060000000002002004000000EA
:107FB000D5F5FFFF0200000002000000960300005C
:107FC00003000000F801002008000000B9F5FFFFE1
:107FD00002000000020000000E030000220000006A
:107FE00044010020340000009DF5FFFF0200000066
:107FF000020000005203000009000000E40100201C
:108000000800000081F5FFFF0200000002000000F0
:1080100000010000BB01000020050020B6040000A4
:10802000DFF800F059C501100548012808BFFAF72C
:1080300013BF70470348012808BFFFF7F1BF70471F
:108040000100000001000000A57800003179000067
:108050004979000073790000F7790000137A000075
:10806000197A0000B3F001000BF1010093F3010055
:108070009FF30100D1F4010081F501005FF30100DD
:1080800000F00BF8002803D0FFF702FFFFF7D2FF44
:108090000020FDF759FDFAF783FE0120704700B577
:1080A00081B0FFF7C1FFAFF3008001B05DF804EBD2
:1080B000FFF7E6BF44F21830C2F20000854648F2EE
:1080C0009F00C0F200008047FEE7000001000000B2
:1080D000000000000000000000000100000000009F
:1080E00045B50110C52F000099A6011019B801105F
:1080F000200000000A00000094070020E521000095
:10810000FF1D0000F71D0000892E0000452F000014
:108110001200018301000143C5A70D63AD2F15B007
:1081200007010004070020C5A700016110610810C5
:108130000F07100000384035002D400140028460D8
:10814000005D08101700F80118A384070083057E5E
:10815000A40306E0EA2306010003040102351C1013
:108160002308047F176304003888604500C3003883
:1081700001AC526003A302AD0163026801438AFFB0
:108180000043022804FF01F00120F1620001100306
:108190000B2000801304120C04120F04121204F2BC
:1081A00001FE47F21F015A10036163000077044388
:1081B00043653A120607800C01051B006805002084
:1081C000A87D0000B07D5212FC0C12C018100703ED
:1081D000030000401C00204404F2082C72F001321D
:1081E000FEFF00011007D748000009490000EB0816
:1081F000253C2002FC06002004615C1002E5190009
:10820000008F300200FF001413161CD821045224E2
:10821000048340028641AB200101004018F1061C96
:10822000125C182104526404526C0412CC2112080E
:108230002443D80A7C43800610128C1C2104439CE2
:108240000104C7010085434B180D12B424210452C8
:10825000BC0452C40452CC0452D4048397173D1278
:10826000050BD62045432C08131204082104520C98
:1082700004521404521C04522404522C0452340498
:10828000523C04830000A862046415104358111C7A
:10829000D0030BC201100001E5EB12884821045203
:1082A000900452980452A00452A80452B004617879
:1082B000F1C7016520FE0A0186038008DB27000064
:1082C000492800009B27242BFF7FDC83010001A1AC
:1082D0000CD00388080020000152B8142002340199
:1082E000002004523C0412000110037823002044B3
:1082F00004124804211043183F08110170052001A1
:108300000100007C221031015200011007200500FD
:1083100020D40700200111C3010001129418210488
:1083200022000150026CDC020001500348070020CB
:10833000030D10034D2F00009504F30101000120EF
:10834000020408002017120001000220050020523C
:0E8350000001520001120001000208000000AE
:10DA500038B504460D4610F07DF90848216801608C
:10DA600061684160A16881600EF0A1FD0EF091FD3A
:10DA70002846BDE8324008F028B900BF80470020A2
:10DA80002B6D0100E39C010013870100E39E010060
:10DA90004D52010049A101001D090100872A010022
:10DAA0000101010021DC00000A006E1902000000E3
:10DAB000DCCC010002000000D8CC01000061310084
:10DAC000BCDA0000010000000000D0020A050000DE
:10DAD0000000000002010000000000001000000033
:10DAE00000000000EC000021000000000000000029
:10DAF000E4DA0000C8DA000000000000CCDA000020
:10DB0000D0DA0000D4DA0000D8DA0000DCDA000055
:10DB1000E0DA000060460020DFF800F041950010D8
:10DB2000DFF800F071950010DFF800F0D1950010DB
:10DB3000DFF800F03D970010DFF800F06597001067
:10DB4000DFF800F029980010DFF800F0C999001004
:10DB5000DFF800F0F9990010DFF800F0159A0010D6
:10DB6000DFF800F0319A0010DFF800F0859A00101D
:10DB7000DFF800F0A19A0010DFF800F0F59A00102D
:10DB8000DFF800F0159C0010DFF800F08D9C00100D
:10DB9000DFF800F0099D0010DFF800F0459D00104F
:10DBA000DFF800F0D19D0010DFF800F02D9E00108E
:10DBB000DFF800F08D9E0010DFF800F0AD9E001041
:10DBC000DFF800F0CD9E0010DFF800F0ED9E0010B1
:10DBD000DFF800F00D9F0010DFF800F0499F001003
:10DBE000DFF800F0699F0010DFF800F0D19F00100F
:10DBF000DFF800F011A00010DFF800F031A00010F5
:10DC0000DFF800F075A00010DFF800F009A10010A7
:10DC1000DFF800F0B5A10010DFF8141A08707047A3
:10DC20002DE9FE430C46200454D5DFF8040A0078A1
:10DC300000F013FE05004AD0DFF8F87939680126B4
:10DC4000002918BF11F1010F07D0DFF8EC090078A7
:10DC500000F0A5FD4FF0FF3038602878812802D011
:10DC600082282CD02FE000208DF808608DF8090064
:10DC7000AE88AF7995F80280B00A3F2807D1C6F385
:10DC8000C21020B100F029F800F02EF803E000F0F7
:10DC900024F800F078F88146284600F071FD9DF8E0
:10DCA0000800A0B1DFF8940901904B469DF80900E7
:10DCB00000903A463146404600F096F907E0284683
:10DCC00000F0C0FB064616B1284600F059FD84F46A
:10DCD000004000E00020BDE8FE8302AB0DF1090228
:10DCE000294630467047000038B500F07F04C0096F
:10DCF00000F00700401E04280D4642D8DFE800F07F
:10DD0000030C32373C00122C3BD12A7CE96828896D
:10DD1000BDE8384001F04DB82889E968012C1DD0D4
:10DD20000B2C17D00D2C11D0132C0BD0192C05D087
:10DD30001E2C26D1BDE8324001F046B9BDE8324084
:10DD400001F013BABDE8324001F0FCB9BDE834403F
:10DD500001F0CAB9BDE8344001F0B8B9BDE83440BB
:10DD600001F061B91A462046BDE83840F5E1204689
:10DD700001B0BDE83040A5E2204601B0BDE830402A
:10DD800076E1012032BD0B4640F21D41401A00F001
:10DD90008F8040F2E471401A00F08D80801E00F008
:10DDA00090802A3800F08F80363800F0878040F26B
:10DDB0009E31401A00F08C80401E00F08B80401E87
:10DDC00000F08A80801F00F089804FF47F71401A34
:10DDD00000F0868040F6FC31401A00F08480801EFE
:10DDE00000F084800C3800F08380401E00F08280B8
:10DDF000401E00F08180401E00F08380801E00F0F5
:10DE00008580401E00F08580401E00F08580401E09
:10DE100000F08580401F00F08680401E00F08A8060
:10DE2000401E00F08280401E00F088804DF6E231F6
:10DE3000401A00F08580401E00F08680C01E00F071
:10DE40008780401E00F08880801E00F08880401E81
:10DE500000F08B80401E00F08A80401E00F08B8016
:10DE6000401E00F08A80401E00F08A80401E00F0B4
:10DE70008A80C01E00F08980801E00F08A80401ECB
:10DE800000F08A80401E00F08C80C01E00F08D8063
:10DE9000C01E00F09080401E00F09280401E00F0F6
:10DEA0009280801E00F09380401E00F0968099E0E2
:10DEB0001889FFF731BE9868FFF732BE986801F005
:10DEC000A4BA01F0D1B959891889C9B2FFF72CBE9B
:10DED00001F004BB01F0D9B9FFF72ABEFFF72CBE51
:10DEE000188901F027BB986801F0DBBAFFF728BE5C
:10DEF000FFF72ABEFFF72CBE1889D968C0B2FFF71A
:10DF00002BBE1889D968C0B2FFF72ABE9868FFF700
:10DF10002BBE1889FFF72CBE188901F04FBAD968BB
:10DF20009868FFF729BEFFF72BBE9A7A597A187ABC
:10DF300001F059BA1889C0B201F05EBAFFF724BEE9
:10DF40001889C0B2FFF724BE1889C0B2FFF724BEFB
:10DF5000D9689868FFF724BE9868FFF725BE5989ED
:10DF60001889C9B2C0B2FFF723BEFFF725BE1889D2
:10DF7000C0B2FFF725BEFFF727BE9868FFF728BE9F
:10DF80001889FFF729BEFFF72BBE1889C0B2FFF72B
:10DF90002BBE1889FFF72CBE59891889C9B2FFF723
:10DFA0002BBED9681889FFF72BBE59899A89188921
:10DFB000C9B201F074BA18895989C0B2FFF724BEFA
:10DFC000188901F05ABA1889C0B201F043BA5989C8
:10DFD0001889C9B2C0B2FFF71BBE1A69D968986820
:10DFE00001F05DB9012070472DE9F843089C804697
:10DFF00004F10C000F461546994680B200F0AEFBC6
:10E00000060016D08020307086F8019040F27F60C4
:10E010007080B780B57106F10C00F471B0602246D3
:10E02000099900F04CFB31464046BDE8F44300F04E
:10E03000B6BBBDE8F18310B502460020941E012C4A
:10E0400002D9A41E02D004E0102900E004290ED059
:10E050000CE0A2F12004402C04D2BDE81040104690
:10E0600002F0E6B8A2F18001102900D3022010BD11
:10E0700070B5401E04280D46144643D8DFE800F072
:10E08000030D171A2C0000F03FF818BBEA68314660
:10E090002046BDE8704002F0D7BB00F035F8C8B9A3
:10E0A000EA6831462046BDE8704002F0DDBB02F070
:10E0B00002FC0FE0A86868B1DFF884150160DFF8A2
:10E0C000841509888180912181717C210181182129
:10E0D000418115E0022070BDDFF86C351B68083304
:10E0E00000221B68002100209847DFF86015887126
:10E0F000020ACA71020C000E48720A7204202070D3
:10E10000002070BD012070BD2C7A6E7A3146204609
:10E1100091E738B5012815461C4602D0022809D0DF
:10E120000DE0049B0A462146284601B0BDE8304078
:10E1300002F0F8BC0846BDE8324003F01FB80846BC
:10E14000BDE8324003F028B80B46012811461846B6
:10E1500008BF02F023BD03F036B838B50C460346BD
:10E16000E168227C2089022B1D462ED0042B4FD043
:10E17000062B33D0082B47D00A2B51D00C2B57D06D
:10E180000E2B59D0102B24D0122B61D0162B63D01C
:10E190001B2B00F085801D2B00F08680302B18BFD4
:10E1A000322B22D0342B3FD0362B49D0382B4BD0BA
:10E1B0003A2B5BD03C2B67D03E2B69D0402B6BD0E9
:10E1C000422B49D0432B75D07AE0BDE8384003F0AC
:10E1D0008EB8A17ABDE8344003F09FB81346A27A06
:10E1E00001B0BDE8304003F0BEB86189A289A37BCD
:10E1F000302D04D101B0BDE8304003F0E5B801B0E6
:10E20000BDE8304003F0EDB8BDE8384003F001B997
:10E2100013464A88098801B0BDE8304003F0FCB8D5
:10E22000BDE8384003F016B9BDE8384003F013B933
:10E23000BDE8384003F012B9BDE8384003F00FB92B
:10E24000BDE8344003F021B9BDE8344003F02BB9F8
:10E25000BDE8384003F03FB9162D03D1BDE8384082
:10E2600003F03AB9BDE8384003F081B9E17A0B0018
:10E2700008D0062906DA009201230A46E16803F075
:10E280002CF932BD022032BDBDE8384003F06CB934
:10E29000BDE8384003F069B9BDE8384003F066B91D
:10E2A000BDE8384004F098B8637C01B0BDE8304068
:10E2B00004F05CB8A289618905F071FB002032BDD1
:10E2C000012032BD2DE9FC410F4614460026DFF83F
:10E2D0007C5310B3032837D0042829D005282BD02D
:10E2E00009282DD00A2834D00B2840D00C2857D02C
:10E2F0000E284FD00F2844D010283DD011282ED002
:10E30000122830D0302855D031285CD032284CD05B
:10E31000362873D0372879D090E078690190386931
:10E320000090FB68BA7A797A387A05F05BFB6BE08B
:10E33000B86805F081FB67E0387A05F0C2FB63E05E
:10E34000B86805F023FE5FE0F968387A05F097FFBA
:10E350005AE03A7B7989387A06F0EEF854E0B868EA
:10E3600006F027F950E0B86806F057F94CE0F96874
:10E37000B86806F0BFF947E0B97A388906F008FABC
:10E3800042E0387C0090FB68FA7AB97A388906F066
:10E390004EFA39E0FA68B97A388906F087F933E03D
:10E3A0003989F86806F003FA2EE0F968B86806F0D3
:10E3B00071FD29E03889798926281DD028281BDAA3
:10E3C00005F012FF20E04FF6FF78ADF800803889A5
:10E3D000FF2811DA26280FD028280DDA05F011FFC2
:10E3E0004045ADF8000007D00220207002226946A7
:10E3F000A81D00F064F922E0022620E07989FA687D
:10E400003889C9B201F0CEF8064618E03F89A91D47
:10E41000384601F09BF9064640F201403F1A04D00D
:10E420003F1F04D0FF1E04D005E0022004E01020AE
:10E4300002E0042000E00120207000E001263046C8
:10E44000BDE8F6812DE9F04184B0044600208DF846
:10E45000090001208DF80800A588A079A778042D6F
:10E4600080460ED8DFE805F06F030A2F4B0002AAA2
:10E470000DF10901204600F082F862E00026103814
:10E48000052860D8DFE800F01916120D0903E268CC
:10E49000A17A208903F010FF53E0A06802F01BFA74
:10E4A0000EE0A17A208902F010FA09E0207A02F049
:10E4B0001AFF05E002F0D6FE43E0207A02F002FAED
:10E4C0008DF8086040E00026A8B1042804D0052893
:10E4D00006D006280AD036E0A06806F087FD33E0B3
:10E4E0002089E168C0B206F061FD2AE000F041F841
:10E4F00006F028FD25E0A06806F06CFD21E0062866
:10E5000021D8DFE800F01B20140F20040A00208926
:10E51000E168C0B204F052FB13E000F02AF804F006
:10E520001EFB0EE0E168208904F0F7FA09E0236998
:10E53000A27BA189A06804F0C5FA02E0A06804F0FB
:10E540009AFB064600E00126204600F019F99DF8E6
:10E55000080050B13948019033469DF809000090F9
:10E56000424629463846FFF73FFD002004B0BDE88B
:10E57000F08161892089E268C9B2C0B27047F8B5FC
:10E580000E468179314F00240429154628D01029E0
:10E5900012D0112914D0122917D0132924D01429EC
:10E5A00028D015292ED0162930D0172934D0182973
:10E5B0000ED019290FD038E0007A06F039FE29E094
:10E5C000817A008907F08DF82BE007F0B5F828E094
:10E5D00007F09EF825E0C168008907F034F80FE0E5
:10E5E000806801F073FA15E0C268817A008901F051
:10E5F0007AFA05E0837C028AC168007A01F0FAF8B1
:10E60000044613E0008901F06FF903E0817A008984
:10E6100001F092F92C7009E00269C168007A01F0FA
:10E62000CEF9B8710120307000E001242046F2BD1F
:10E63000D448002038430020DB480020BE4600209C
:10E6400002020200AADA000030430020B84600208F
:10E6500000B583B00821ADF8001001900B21ADF892
:10E6600002106846DFF87416096888470EBD1FB5AA
:10E670008DF806100824ADF800408DF8040006243B
:10E68000DFF858168DF808200393ADF8024068466D
:10E690000968884704B010BD80B5052007F0A5F8CB
:10E6A00000F0EDF90C2000F001F802BDDFF82C16A7
:10E6B0000968ADF802006846084707F0A5B803E00E
:10E6C00011F8013B00F8013B13465A1E002BF7D10D
:10E6D00070471144491E03E011F8013900F8013B6D
:10E6E00013465A1E002BF7D1704770B504460D46ED
:10E6F000A8B207F0A5F8060003D02A462146FFF786
:10E70000DEFF304670BD10B513465A1E3BB110F8FF
:10E71000013B11F8014BA342F6D0002010BD0120AF
:10E7200010BD10B5044610460A460146204607F0C3
:10E73000A7F8204610BD02F0B5B8DFF8A425DFF831
:10E74000A435126A11541B7805E0DFF89835DFF81C
:10E7500090251B78126AC0181154704710B5040038
:10E7600001D1002010BD04F10C0080B207F068F860
:10E7700028B1002101600481FF2181720C3010BD9D
:10E7800080B508B9052002BD10F8021CFF2901D090
:10E79000042002BD0C3807F060F8002002BD38B537
:10E7A0000C46010622D5DFF838150A78FF2A08BF83
:10E7B0004D7805D0DFF82C351B78096A9A188D5CE6
:10E7C000FF2D02D1FFF768FF0EE000F09BF9014634
:10E7D000FF2004F8020C234600222846FFF747FFDB
:10E7E00048B12046FFF7CCFF012032BD2146BDE8ED
:10E7F0003840002200E032BD70B50D0004461646D8
:10E8000018D0200648BFFFF747FFDFF8D814097873
:10E810008C4204D32846FFF7B3FF032070BDA5F157
:10E820000C000168002904BF817AFF2904D0284622
:10E83000FFF7A6FF052070BD8472012EDFF8A0044B
:10E84000294603D1001D00F055F802E0001D00F03C
:10E8500039F800F033F8002070BD2DE9F04104468E
:10E86000DFF88404DFF878740068804780467868B1
:10E870000026002503E005B9064650F80C0C50B1FF
:10E8800010F8021CA142F6D1002D08BF0546F4D0B5
:10E8900000F014F805E04FF40041204600F0A4F821
:10E8A00025B132462946381D00F031F8DFF83C1416
:10E8B0000968404688472846BDE8F0814FF400418A
:10E8C000204642E038B500F00FF8002145F80C1C56
:10E8D000216811B9256006E0114651F80C2C002A78
:10E8E000FAD141F80C5C27E10446DFF8FC0300682C
:10E8F0000D46004738B5FFF7F7FF216845F80C1CB7
:10E900002560DFF8E8130968BDE83440084770B5B2
:10E91000044600F014F8A5F10C0123680A689D4232
:10E920000CBF226046F80C2C00220A60FF228A727B
:10E93000BDE8704002E1DFF8B41309680847DFF86A
:10E94000A80300680D46164600472DE9F04104462D
:10E95000DFF89003DFF8885390F8008020060E4619
:10E960002CD50420FFF7FAFE070008BF042039D099
:10E970004FF6FF7038807E80A7F10C062878FF28BC
:10E980000FBF6D78296A40440D5CFF2D05D13846D4
:10E99000FFF7F6FEFFF780FE0EE0204600F0B2F82B
:10E9A000FF21B1723B46014600222846FFF75FFE79
:10E9B000C0B13846FFF7E4FE012013E0444510D211
:10E9C00000F028F8DFF82813096831F814203243E2
:10E9D00021F81420FFF7AFFFE868FFF739FE0020A9
:10E9E00000E00320BDE8F08138B50C46BD49097848
:10E9F000884205460CD200F00DF8BD49096831F88F
:10EA00001520A24321F81520FFF795FF002032BD05
:10EA1000032032BDB4480068004730B5B04C002038
:10EA2000606083B006F06EFF07F0BBF8AD48057874
:10EA3000680006F005FF20626A00FF21FFF771FE03
:10EA40000222FF21A01CFFF76CFE07F001F900F085
:10EA500016F81420A14D2968ADF8020068468847D1
:10EA60000198206100F00BF81520ADF8020068460F
:10EA7000296888470198801E606100203EBD0820FB
:10EA8000ADF80000704730B587B00820ADF8080039
:10EA90001B20ADF80A0001200390914D0FF27D007C
:10EAA0008E4C21680590E8690690A869049002A838
:10EAB00088470499A96108B1FFF7EEFD00F053F80B
:10EAC000FFF7DDFF0A20ADF802004FF0FF300190A4
:10EAD000684621688847F1E780B50021804A0A44EA
:10EAE0009378FF2B01D1907001E0834203D141F074
:10EAF0008000C0B202BD491C0229EFD3FFF7CCFD54
:10EB0000FF2002BD10B580F08004022CA8BFFFF7E3
:10EB1000C3FD73482044807810BD000038B504461A
:10EB2000FFF778FF05466E48C1698C4204BFC06894
:10EB3000FFF78EFD4FEA0500BDE834406B490968D8
:10EB4000084710B50446608850B9A079FFF7C4FFA4
:10EB5000FF28E07102D16FF0030010BD002010BD4E
:10EB60006FF0010010BD2DE9F04F8BB006F0EDFF06
:10EB700000245FEA000B03D006F0F9FE4FF0FF3BE4
:10EB8000574DA868010003D0804701E0FFF784FDDE
:10EB90000820ADF808000720504E3168ADF80A0093
:10EBA00002A888474F499DF80E20049F0978E8B9CC
:10EBB000002600E0761C8E42E8D2286A805D9042F2
:10EBC000F8D1F6B2FF2EE1D017F8080CFFF784FF5A
:10EBD00017F8061C012908BF387002D0022908BFA7
:10EBE000B87039463046FFF7DAFDD1E7404F386854
:10EBF000E4B230F8140018B9641CE0B28842F5D3CE
:10EC0000E0B28842DFF8E480DFF8DC901DD2D9F86A
:10EC1000000080473968E4B231F814A0002200F007
:10EC200047F8344A2C70514652F824202046904729
:10EC30008246FF202870D9F800008047396831F8F3
:10EC400014204AEA020200F033F806F07EFF07467D
:10EC50005F452AD007B9284F6869B84238BF0746D0
:10EC6000D9F8000080470446FFF709FF1C20ADF8E3
:10EC70000200A86931680190684688470821E86960
:10EC8000ADF81410401C1321E861ADF8161009907E
:10EC900006971A49A8690891079005A8316888471E
:10ECA0000798A861204600F005F80BB0BDE8F08F8A
:10ECB00021F81420D8F80010084710B548B10023F7
:10ECC00000E05B1CDCB2944205D2DBB2C45C8C4237
:10ECD000F7D0002010BD012010BD000080470020AB
:10ECE0009C440020A8DA00008447002088470020C8
:10ECF0009847002080DA00008EC2F5281DEB000046
:10ED0000DFF800F0F5950010DFF800F03196001004
:10ED1000DFF800F05D9600100A4610B5052A18BF0E
:10ED2000042A03D0062A18BF072A08D10C244B4B0B
:10ED300062431A4422F8301D9070002010BD02205A
:10ED400010BD38B50D4604462888052818BF04288C
:10ED500003D0062818BF072801D1686808B9022027
:10ED600032BD0121204606F0BCFC08B9142032BD9A
:10ED70004FF6FE70844207D0204606F0EEFC29894B
:10ED8000884201D21B2032BD354800780028294630
:10ED9000204603D0BDE8344001F0D0BFBDE8344088
:10EDA00001F082BF80B52F4B009313460A46012124
:10EDB00020E070B50D4684B004461646EB88AA885C
:10EDC0006988288800F032FA58B100200290019634
:10EDD000042000902A46244B1221204601F0FAFE1E
:10EDE00000E0182004B070BD80B5204B009313469E
:10EDF0000A46132101F020FF02BD38B504461C4825
:10EE00000129017011D11B480088051DADB20120F8
:10EE1000FFF776FF94FBF5F082B2284601B0BDE81B
:10EE2000304000230021FFF76FBFBDE832400020D3
:10EE3000FFF766BF03B50E480078012881B003D103
:10EE400002AA01A9FFF764FF07BD0A4A001F10804C
:10EE500003480170704707480088704758480020F1
:10EE60008E4600203D0E0100BB0E0100210F010067
:10EE7000D9480020A4460020704700005D49086082
:10EE8000704738B50D460446288817280ADBFFF777
:10EE9000E2FF2988884205D3002000902B460222F9
:10EEA000554987E0022032BD80B500F031F80422D8
:10EEB000524900E0524907F051F902BD38B50D46FC
:10EEC00004462879022809D1E86810B1072102F028
:10EED0009FF900902B4606224A496BE0022032BD82
:10EEE00080B50A79102A18BF022A03D100F010F861
:10EEF0000822DFE7022002BD80B500F009F80A22EF
:10EF00004149D8E780B500F003F80C223F49D2E729
:10EF1000002200920B46704738B50D460446A8887B
:10EF2000022809DB286838B1012102F071F900904C
:10EF30002B460E2236493DE0022032BD80B50A79CB
:10EF4000102A18BF022A03D1FFF7E2FF1022B1E70F
:10EF5000022002BD70B50D4682B00446287A122602
:10EF6000012809D1204607F08DF969880F388842B9
:10EF700001DA022076BD9226687A0128686808BF07
:10EF800046F0400610B1032102F042F900902B46F2
:10EF900032462049204607F0E1F876BD38B50D46E7
:10EFA0000446A86810B1052102F032F900902B4602
:10EFB00016221949204607F0D1F832BD80B5FFF777
:10EFC000A7FF1822154976E738B5044600200090BF
:10EFD00000231E220021204607F0C0F8050006D1BC
:10EFE00004480268100002D01E212046904728469F
:10EFF00032BD0000B4470020C35D0100F55D010093
:10F00000DB5E01005D5E01006B5F0100C35F01001C
:10F0100013600100B75F01007F600100F96001002B
:10F020006E490860704780B5002200920B460122AD
:10F030006B4900F0BAF802BD80B50A88172A05DBD3
:10F04000002200920B4603226649F2E7022002BD2D
:10F0500038B50D460446A878012818BF02280DD1FE
:10F06000288800281CBF6868002807D0022102F009
:10F07000CFF800902B4605225B4931E0022032BDDB
:10F0800038B500F01EF81CBF6868002806D000F0F4
:10F0900036F800902B460722544921E0022032BD69
:10F0A00038B500F00EF81CBF6868002807D00221B0
:10F0B00002F0AEF800902B4609224D4910E00220E4
:10F0C00032BD0D46044628880028704738B500F048
:10F0D00024F808B100F013F800902B460B224549A4
:10F0E000204600F062F832BD38B500F016F808B1DD
:10F0F00000F005F800902B460D223F49F0E7012172
:10F1000002F086B838B500F008F808B1FFF7F7FF4D
:10F1100000902B460F223949E2E70D460446686805
:10F12000704738B5FFF7CDFF1CBF6868002807D0CF
:10F13000022102F06DF800902B4611223049CFE7F2
:10F14000022032BD80B5002100910023132270E718
:10F1500038B50D460446A86810B1052102F058F8EC
:10F1600000902B4617222749BAE780B5002100916D
:10F17000002319225DE738B5FFF7CFFF10B1032157
:10F1800002F046F800902B461B2209E038B5FFF745
:10F19000C4FF10B1032102F03BF800902B461D2262
:10F1A0001949204606F0DAFF32BDF8B50446069844
:10F1B000009015461E46204606F0D0FF07000AD1F3
:10F1C00006480268100006D0012D04BF3078451CA7
:10F1D000E9B2204690473846F2BD0000B047002013
:10F1E000935D0100CF5D0100015E0100B95E010089
:10F1F000475F0100875F0100016001003B60010083
:10F2000041600100A96001001D610100DFF800F00C
:10F21000DD8A0010DFF800F0A18B0010DFF800F0AD
:10F22000D5700010DFF800F09D58001030B540F6A2
:10F230007B44851FA5423CBF8D1FA54212D281424F
:10F2400010D3B2F5FA7F0DDAA3F10A0040F6774445
:10F25000A04207D2501C49004843B0EBC30F804185
:10F26000C00F30BD002030BD80B507F0E5FD8DF842
:10F27000000008F061FE9349002008706A46924938
:10F280000880012140F6034067E080B50FF2D022EC
:10F29000412141F20200FFF7B9FF002002BD7CB519
:10F2A000002808BF00294FF620442DD162BB01A8D9
:10F2B00008F094FD9DF8040000EBC000451DEDB280
:10F2C000284606F0BDFA060018D020203070042031
:10F2D00070700020B0709DF8040000280CBF002260
:10F2E000721D311DF01C07F00DFE324629462046E6
:10F2F00009F0D3F8304606F0B0FA15E004218DF895
:10F3000001102020072106E007F0FCFD04218DF804
:10F310000110202000218DF800008DF802106A46AF
:10F320000321204609F0B9F8002076BDFFF76EFFF3
:10F33000002016BD80B500208DF800006A466348A5
:10F3400000788DF80100042100208DF8020060484B
:10F3500000788DF8030042F20200FFF757FF00200B
:10F3600002BD1FB5044608980290079801900698C0
:10F370000090204608F0F0F98DF80C008DF80D4053
:10F38000200A8DF80E0003AA032142F22000FFF7A5
:10F390003DFF5CE010B582B0044608F029FA00F0A9
:10F3A00003F842F22100C1E78DF800008DF801401A
:10F3B000200A8DF802006A460321704738B50446DA
:10F3C00042F2160529460020FFF724FF204607F0E9
:10F3D00066FE8DF8000020B16A4601212846FFF73D
:10F3E00015FF002032BD80B5012308F02FF800F092
:10F3F0001BF842F21E00B0E780B5012108F0F2F8D8
:10F4000000F012F842F21D00A7E780B530B10146C6
:10F4100008223048FFF753F9002000E0122000F0E6
:10F4200003F840F6634098E78DF800006A46012132
:10F43000704710B584B0089C0294079C0194069C08
:10F44000009408F0FDF942F21301FFF7E3FE0020FB
:10F4500004B010BD80B51D218DF8001004218DF879
:10F46000011010B9FFF7DAFE00E011208DF802005C
:10F470006A4603214FF61D400DE080B51C208DF833
:10F4800000006A4604208DF8010003210C208DF84D
:10F4900002004FF61C4009F000F8002002BD08F001
:10F4A000CFBC80B530B10C4902780A704078487002
:10F4B000002000E01220FFF7B7FF42F201004CE706
:10F4C00000000000244F0020264F00201843002099
:10F4D0001A430020904800208848002000B585B0DD
:10F4E0006A460DF1020101A8FFF79CFE8DF80800A5
:10F4F000222107208DF8090002AA02A881700221AA
:10F500008DF80B109DF804108DF80C10BDF802104A
:10F510008DF80D10090A8DF80E10BDF80010C1719C
:10F52000090A017241F201000921FFF76FFE002074
:10F5300005B000BD10B582B004460DF1030108F01E
:10F5400053FC00F004F8042141F20540EEE68DF88A
:10F5500000008DF80140200A8DF802006A467047CD
:10F56000002000800000C000000000E4000000282F
:10F570002200000000000004000017FCFF790000DA
:10F58000003030000000000000000000000000001B
:10F59000000000000000000000000000000000006B
:10F5A000000000007CB5164600244FF48063C21AA8
:10F5B000DFF8745C26D0521E2BD0521E2ED0521E65
:10F5C00033D0521E38D0521E3DD0521E44D0521E4F
:10F5D00049D0521E4CD0521E53D0521E00F079809A
:10F5E000521E00F07D80521E00F08180521E00F0FD
:10F5F0008680921E00F08F80521E4DD0083A00F097
:10F60000918097E0012918D13078032811DA6873C6
:10F610009AE0022911D13088288595E001290CD182
:10F620003078022805DAA8738EE0012905D13078F8
:10F6300005287DDAE87387E0012979D1307802283E
:10F6400076DA287480E0102972D11022314605F153
:10F650003C00FFF734F877E0012969D130780228BF
:10F6600066DA687470E0012962D1307828756BE041
:10F6700004295DD13068DFF8B41B884258D2E862B3
:10F6800062E0002954D105F045FE10B900F0AAFC53
:10F6900017E00120287657E0072949D10622711C7E
:10F6A0006846FFF716F830780022694600F087F9BF
:10F6B00006460A2E47DA05F02DFE30B9304600F036
:10F6C0009DFC502001F0DEF822E0A9190120087706
:10F6D0003AE001292CD13078022829DAA87433E0E5
:10F6E000012925D130780A2822DAE8742CE0012992
:10F6F0001ED13078C11F0A291AD2687524E0012969
:10F7000016D1E97D3078E875002908BF01281BD1A2
:10F7100000F00CFC18E001290AD13078042807DA3F
:10F72000A87511E0012903D116B13078A8760BE055
:10F73000182409E0282806DA022904D1318804F0C7
:10F7400053FD044600E00224204676BD38B500246F
:10F750004FF480630D46C21ADFF8CC1A1CD0521E3B
:10F760001CD0521E1CD0521E1CD0521E1CD0521E29
:10F770001CD0521E20D0521E20D0521E20D0921ECD
:10F7800021D0521E21D0521E21D0521E21D0521EF5
:10F7900021D00A3A22D024E0487B20E0088D24E0E2
:10F7A000887B1CE0C87B1AE0087C18E010223C3102
:10F7B0002846FEF784FF1BE0487C10E0087D0EE041
:10F7C000C86A286014E0887C09E0C87C07E0487DAE
:10F7D00005E0C87D03E000F0F2FB00E0887E2870C1
:10F7E00006E0282803DA04F00CFD288000E002245B
:10F7F000204632BD2DE9F0428CB0814614460AA85D
:10F800000022C0E900221E460AAA484600F0D7F8A6
:10F8100005460A2DDFF8107A4FDA00F04FFB8146DB
:10F82000787B02280CBF01200020009033464A4616
:10F830002946204600F08FFD1422002101A8FEF782
:10F8400070FF062000FB05F606F1240001AA102136
:10F8500000F089FA88B91022FF2101A8FFF72DFADC
:10F8600058B906F1250005AA042100F07CFA01AA86
:10F8700009F00101204604F019FF05F1700006AA05
:10F88000102100F070FAA0B906A800F07DFA002659
:10F8900006AF304637F8201041B106A901EB8001D0
:10F8A0008A7837F82010204604F040F8761C042EA1
:10F8B000EFDB284600F05EFB12E0082E04BF787BE9
:10F8C00002280DD100224946204600F0DBFC386BAF
:10F8D00030B14368180003D0002200212046984729
:10F8E00000200CB0BDE8F08270B505F013FD10BB30
:10F8F000DFF83449207E01280AD100F073FB002094
:10F9000020760A22002104F11C00FEF70AFF0CE019
:10F9100000256619307F012804D1284600F06EFBCF
:10F92000002030776D1C0A2DF3DB502000F0AAFF79
:10F93000BDE87040FAE270BD2DE9F04184B00446A4
:10F94000884601A80021C0E90011204605F09BFE71
:10F9500006001EBFDFF8D078787B02282DD07079A2
:10F9600001AAB11D00F02BF805460A2D19DA00F0A6
:10F97000A5FA00F0040108F004029142A2BF00F0D1
:10F98000080008F0080188420BDB284600F096FAD0
:10F9900002460120009008232946204600F0DBFCA7
:10F9A0000BE0787B28B171790022204600F06AFCD8
:10F9B00018B10521204604F0EBFEBDE8FF812DE9DA
:10F9C000FF4116460D460A246A79022102F0C00260
:10F9D000C02A08BF002102D0402A08BF012102002E
:10F9E00018BF022803D0032818BF00290DD12846CC
:10F9F00000F087FA04460A2C3DDA002E3BD006229E
:10FA000029463046FEF75BFE35E0022910D100277B
:10FA1000DFF8DC890E207843404406222946C01DC9
:10FA2000FEF771FEF8B97F1CFFB20A2FF2DB22E06D
:10FA3000012920D100270620784323306A4610216F
:10FA400000F091F950B91022FF216846FFF735F90F
:10FA500020B92946684605F01DFA20B17F1CFFB287
:10FA60000A2FE8DB07E00A2F3C4604DA1EB13146D4
:10FA7000204600F030FA204604B0BDE8F081F8B529
:10FA80000C4615264FF6FF71884215460BD100270C
:10FA90002A462146384600F01AF900B100267F1C9C
:10FAA0000A2FF5DB10E005F0EEFD60B1811D407915
:10FAB0000022FFF784FF0A2806DA2A46214600F0D2
:10FAC00006F9002600E014263046F2BD10B5DFF836
:10FAD0005847217B2063262004F086FB207BBDE86D
:10FAE000104002F0A5BF38B50446002508000DD12E
:10FAF000DFF83807DFF83437B2FBF0F0214603FBBC
:10FB0000102004F06EFE050003D00121204604F011
:10FB10003FFE284632BDF0B5044685B0A078DFF838
:10FB20000857062800F0C580092800F0AE800A2892
:10FB300023D00B2805D00C2800F0B6800E2879D0F1
:10FB4000BAE0286B50B10668300007D020690090F9
:10FB5000637B227B6189E01CB047ADE0206961894D
:10FB6000002814BF0120E86A04F03BFE002803D0FF
:10FB70006089012104F00CFE9EE0607800260028D8
:10FB800046D1A079C00743D5686B002840D10E222A
:10FB900000F099F8A08805F076FD0600ECD06769C2
:10FBA000CFB1387C8DF80600062207F111016846B6
:10FBB000FEF785FD0622B11D06F10C00FEF77FFD64
:10FBC000062207F11101B01DFEF779FD387C40F0E7
:10FBD0000200707107E070798DF806000622B11DF1
:10FBE0006846FEF76CFDA1799DF80D00890801F0CB
:10FBF000010108438DF80D002146684600F0D3F856
:10FC000028B9287B0221FEF7A0FE002055E015262A
:10FC1000286B002850D0436818004DD06278A08827
:10FC200001219847300047D02B6BA0885B68324693
:10FC3000032128E0607806281DD1A08805F023FD67
:10FC4000060018D0A87D012804D014D3032807D0BB
:10FC50000CD310E07179A088002200F013FB0AE0B9
:10FC60000022002140F20940FFF79CFCA188307877
:10FC7000052204F061FC286BF0B1436818001BD02A
:10FC80006278A0880221984716E0E0780022211DC2
:10FC9000FFF795FE0A280FDA06235843253004F1B2
:10FCA0000C0200F00CF807E0217BA088FFF744FE6F
:10FCB00002E0A088FFF718FE012005B0F0BD042186
:10FCC000C0B200F0D1BD00216846FEF72ABD70B574
:10FCD00006460620704388B00C461546203004AA1C
:10FCE00000F040F8002838D10622FF2104A8FEF7D2
:10FCF000E4FF90BB70366A461021F0B200F0A4FD1C
:10FD000048BB684600F040F8200009D110220021CD
:10FD10006846FEF7D2FFF0B91022FFF7D4FF12E0D9
:10FD2000694600F023F838B9280016D0694600204B
:10FD300000F01CF888B104808178A9420BD085704E
:10FD40000DB900210180684600F01EF86A461021B6
:10FD5000F0B200F089FD012000E0002008B070BD85
:10FD600020306A460E21C0B200F06EBD002231F88C
:10FD70002230834202D101EB82007047521CD2B282
:10FD8000042AF4DB00207047002130F82120D24300
:10FD900020F8212000EB8102491C9378DB430429E1
:10FDA0009370F2DB70472DE9F043DFF87C44DFF815
:10FDB00040968046606B85B00F460E26E8B9B8F1D4
:10FDC000000F18BF002F70D0404600F09AF80A28A4
:10FDD000607612DB002506FB05F00622FF21484471
:10FDE000FEF76BFF40B96D1CEDB20A2DF3DBA07E70
:10FDF000002814BF25780A256576607E0A2854DA23
:10FE00000625616B6843C9B9203042460E21FFF7D1
:10FE100057FF607E00F0AEF81022FF21FFF754FF7D
:10FE2000607E703000F045F8607E70430E224146DF
:10FE30004844FEF744FC6763002037E08A683AB123
:10FE400021301C21FFF73CFF616B00208860F3E745
:10FE50000A693AB122301C21FFF732FF616B0020A2
:10FE60000861E9E74A693AB123301021FFF728FF1A
:10FE7000616B00204861DFE7CA6882B1243010213D
:10FE8000FFF71EFF606BC06800F11002607E6843E0
:10FE90002530FFF714FF616B0020C860CCE7E07DE0
:10FEA00008B100F082FA00F0DEF9012005B0BDE8EB
:10FEB000F0836A461021C0B200F0D6BC00B506231C
:10FEC000584385B0FFF74CFF00280CBF9DF80D008C
:10FED000002005B000BD30B50A2885B00C4600DA18
:10FEE0000CB902200BE006235843FFF739FF050049
:10FEF00004D1062269462046FEF7E1FB284605B0FC
:10FF000030BD70B504460025DFF8E4640E20684378
:10FF1000062221463044FEF7F6FB08B1284670BDA4
:10FF20006D1CEDB20A2DF1DB0A2070BD38B500243E
:10FF300000F04EFA0620604320302A460E21C0B25F
:10FF400000F082FC58B10622FF212846FEF7E9FBAB
:10FF50000622FF21E81DFEF7E4FB00206873641C05
:10FF60000A2CE5DBB048C07D08B100F01EFABDE800
:10FF7000314078E138B50A210A23AB4A5C1EDBB276
:10FF8000134413F8013C834201D1214603E0234688
:10FF9000E4B2002CF2D1C9B2084605E01418135C93
:10FFA000657815546370401C0928F7DB092905DAC8
:10FFB000BDE838400A21052000F056BC31BD70B5BF
:10FFC00000240025DFF828640E2068430622FF2164
:10FFD0003044FEF772FE00B9641C6D1C0A2DF3DB81
:10FFE000E0B270BD10B50024204600F007F8641C94
:10FFF000E4B20A2C01DA0100F6D010BD2DE9F04779
:020000040001F9
:10000000894D697E884290B0814609D1287B0121C3
:10001000FEF7EAFC287B0221FEF7E6FC00F0DDF9A2
:10002000062000FB09F505F1200607AA0E21F0B213
:1000300000F00AFC002843D10622FF2107A8FEF7A2
:100040003CFE00283CD11C22FF21FFF73DFE102280
:10005000FF210BA8FEF765FB0E22FF2107A8FEF784
:1000600060FB07AA0E21F0B200F0FEFB064605F188
:10007000210000F029F8824605F1220000F024F862
:10008000804605F12300FFF714FF044605F1240024
:10009000FFF70FFF074605F125006A460421C0B2AD
:1000A00000F0E2FB48EA0A012143394340EA010536
:1000B00009F170000BAAFFF7FDFE2843304300E072
:1000C000002010B0BDE8F0876A461C21C0B200F0E5
:1000D000CBBB10B5C74C207304F14C0005F007FAF8
:1000E000FFF724FF22460A21052000F0ADFB30B1C6
:1000F0000020C0F109012154401C0A28F9DB10BD81
:10010000F0B50D46280485B0474C25D5207BFEF779
:10011000A4FB04001DD021780120B0290FD0B12903
:1001200005D0D02904BF2046FFF7F5FC0DE020796B
:1001300060B92289E1886088FFF7A1FC06E0217997
:1001400004F1080000F02AFD00E010B12046FEF79F
:1001500017FB85F4004065E0A80709D500210020C1
:10016000FFF721FE002885F0020550D102214FE063
:10017000E80752D5606B8688A06B4FF6FF7748B9C9
:1001800004F12A00009002239B4A3946012001F025
:10019000EEFFA06385F00105A16B21B3FF20039062
:1001A00002200290002001900DF11200009004AB9B
:1001B000628D304603F07AFA68B99DF810009DF818
:1001C000111000EB012290B228B1A06B418992B2CC
:1001D0003046FFF754FC628DA06B0023394602F0D5
:1001E0001BF8A06398B9206B70B1436818000BD05E
:1001F000606B8088002201219847606B236B8088A8
:100200005B6800220321984700F0E7F803E0012132
:10021000207BFEF79AFB284604E068074CBF85F078
:100220000400002005B0F0BD4044002040420F0013
:1002300010B52038062390FBF3F30624012204FBBB
:10024000130005280DD8DFE800F0030505070709AE
:100250000E2904E01C2902E0102900E0042908BF4F
:100260000022104610BD80B5FFF7A9FE0228ACBFE2
:1002700002200A208DF800006A460121052004F0C2
:1002800061FE01BD70B5AAB006460C46154605F0E4
:10029000FAF908B914205CE0A422FFF714FDADF8C8
:1002A0000060544EF07B317D8DF8040001F00102B6
:1002B000707D8DF8A0002798400842EA400020F0A9
:1002C0000202480800F0010042EA400020F4807277
:1002D000080900F0010042EA002020F400724809F9
:1002E00000F0010042EA402020F48062880900F01A
:1002F000010042EA8020890820F0040001F0010199
:1003000040EA8100279001A9307C020008D04870A3
:10031000102206F13C010DF10600FEF7D0F901E0D4
:1003200000204870707C28B11CB1279840F0020072
:10033000279001209DF899100843B17B8DF8990012
:1003400001B1042108438DF899002946684604F05C
:10035000D1F92AB070BD70B5044606204843082B79
:1003600088B0154604D1290758BF00F1220601D5EF
:1003700000F121061C22002101A8FEF7D2F901AAF2
:100380001C21F0B200F060FA68B99DF81E00C01F91
:100390000A2808D20C98009001AB002205F0010158
:1003A000204604F044FA08B070BD38B5FDF7D0FB24
:1003B000002400F00DF80622FF212846FEF77DFC00
:1003C00010B92946FDF7C8FB641C0A2CF1DB31BDCE
:1003D0000E21074861434518704710B5054C606B06
:1003E00018B1FEF7CDF9002060630A20607610BDD9
:1003F000F046002040440020F0CC0100002010B561
:10040000DFF828446070207082B000F004F9002109
:1004100000F0FEF80098B0F5801F02D100F0E3F87C
:100420000BE020B900F0DFF800F01DF905E000F066
:10043000BDF800F0ABF804206080607816BD38B5D8
:10044000DFF8E8432578290001D0012032BD61881A
:10045000C1F5805189B2814200D350B900F09EF8B5
:100460000020607000F0FFF818B96578280008BF18
:100470000125284632BD13B5DFF8B003BDF80210E0
:1004800040881C46C9B200F0CBF8010009D0DFF863
:10049000A003049A0003A3B2000E08F077F800202E
:1004A00016BD012016BD2DE9FB43DFF8806382B045
:1004B000002070701746BDF80A90708898465FFA61
:1004C00089F100F0ADF80446B8B1002501E0641CE4
:1004D0006D1CEDB2B9B28D420CD2D5480003012398
:1004E00001AAA1B200F094F89DF8040018F80510D4
:1004F0008842ECD0B8B285423ED0BFB2F81C411061
:1005000000EB9170801087007088BFB23818001D12
:10051000B0F5805F03DD00F041F800F0A4F87488C6
:100520004FF6FF70ADF800003D1947F4004000F0B1
:1005300027F8BDF80200C0F30E0000F021F8BA055C
:10054000120E4146204600F016F95FFA89F141F497
:100550000040ADF8000000F015F8BDF80000C0F351
:100560000E00ADF8000000F00DF87078010004D125
:100570007088391D08187080002005B0BDE8F08330
:10058000ADF8020001226946A8B2F4E080B54FF44C
:100590008010009001226946002004E080B5002010
:1005A00000900122694600F0E6F801BD70B5A1484F
:1005B00000688047044600F023F905469C48000384
:1005C0000021000E08F003F808F00CF80646284653
:1005D00000F00EF90EB100F006F92046BDE87040BB
:1005E00095490968084710B582B040F6FC7400F0E0
:1005F00012F8214600F00CF8009810F1010F03D119
:10060000241FA4B2042CF2DA8849201D488013BDAF
:10061000000E07F0BBBF8648000304236A467047FC
:1006200038B50C46051F00E02D1FADB2042D18DBB8
:10063000FFF7F1FF2946FFF7EBFFBDF80010BDF80B
:100640000200A14203D1C0B2281A80B232BD010417
:10065000EAD4011D8D42A8BF281AE3DA002005F074
:10066000C4F8002032BD2DE9F04F83B000F0C8F887
:100670006E4FDFF8BC9183467888041F4FF0FF0867
:100680000025A4B24FEA193A2DE04FF088508119A5
:10069000042201A807F0BCFFBDF804005FFA88F14E
:1006A00088421BD0BDF80600301A061FB6B2301FB4
:1006B00040F6FC718842E8D3BDF802004FF0885143
:1006C0004A19031D211A9BB289B25FFA8AF007F01A
:1006D0005DFFBDF802004019051DADB2BDF8020076
:1006E000201A041FA4B2042C2ADB04236A462146E4
:1006F0005FFA8AF007F04AFFBDF800004FF6FF717D
:10070000884218BF002810D1BDF80200010448BF7C
:10071000241FE7D4001D8442E0DA002005F065F8CC
:10072000584600F065F8002023E00004D6D4BDF858
:1007300000005FFA88F18842D0D080462E1FB5E7CE
:10074000FFF734FF45B12A464FF0885109F1040004
:1007500007F038FFFFF71AFF584600F049F878789D
:1007600028B9281D7880C5F5805080B201E00020AE
:100770007880BDE8FE8F2DE9F04705462C480E46EF
:10078000040B82B017462946E0B207F020FF8146ED
:10079000284800688047804600F032F88246BA0058
:1007A0003146484607F00EFF504600F021F801E0C0
:1007B0002D1D361D3846471EC0B270B104236A464F
:1007C000A9B2E0B207F0E2FE04223146684607F023
:1007D0005BFF0028ECD000F006F840461649096897
:1007E0008847BDE8F38711480121417001707047C7
:1007F00028B1124A12481268526801211047704706
:1008000038B50F4C204607F071FF0546C0B250B115
:100810000A4A12685268002120469047204607F095
:1008200065FF0028FAD1E8B232BD0000A0460020E2
:1008300000E001008447002088470020D801001014
:10084000004003400020D9E5E0B5ADF806000B46B6
:100850000020ADF808008DF804000092DDE90101E8
:100860000022FFF708FE0EBD82B01346ADF802006D
:100870000A460020ADF804008DF80000DDE9000113
:1008800002B010E6652807DA0003642190FBF1F05E
:10089000C0F5805080B2D2E504207047DFF800F048
:1008A0000158001080B502216846FFF7F7FFBDF838
:1008B000000002BD70477047824908607047814957
:1008C00048607047804908707047032290FBF2F03F
:1008D00080B2FEF792BA0178B02904BF41780029AE
:1008E0000CD10179122903D1417C012906D101E003
:1008F0001B2903D140880121FEF79CBA704710B52F
:10090000724C607004F018FF401C20700421607865
:10091000FEF702FABDE8104001F03EBB38B50C46C8
:10092000200411D569484078FDF797FF050008D0ED
:100930002878A02804BF284600F008F82846FDF7CC
:100940001FFF84F4004032BD002032BD30B587B0B7
:10095000044601208DF8000001A9204605F0ECF9BD
:1009600005002AD19DF806105648C9070AD54368E4
:10097000180005D060886A4601A9984705461CE022
:1009800006251AE00368180006D060886A4601A9A7
:100990009847050001D110E006259DF8050060B9D3
:1009A0009DF806008DF810008DF814500020ADF869
:1009B000120004A96088FEF736FB9DF800000028AD
:1009C0001EBFA068002800F0FEFB45B99DF8060098
:1009D000122806BF9DF8051001291B2803D0608846
:1009E0000121FEF727FA07B030BD2DE9F04104469A
:1009F000FF2C0D46164698461FD02020FDF7AEFE70
:100A0000070018D0B02038707E707D8087F8048091
:100A1000069929B1182207F10800FDF750FE04E0FD
:100A2000182207F10800FDF77CFE39462046FDF745
:100A3000B6FE002002E0132000E00220BDE8F081B5
:100A400010B54FF47A746243BDE8104007F09DBEC4
:100A500010B504001EBF2078FF28FE2803D007F041
:100A6000CEFEFF20207010BD80B5009313460A46CD
:100A7000014615480078FFF7B8FF02BD30B583B0D6
:100A800004460D4605F0E9FB50B901A80090ADF809
:100A900004507F230C48007800222146FFF7A5FF71
:100AA00037BD00B583B07E238DF804108DF8052086
:100AB00001A900910022014603480078FFF795FF45
:100AC00007BD0000F0470020A7460020D7480020BF
:100AD000052923D006291BD0072918BF09291DD0B5
:100AE0000B2918BF0D2919D00E2913D00F291CBFAF
:100AF0001129122912D0162918BF17290CD01B2929
:100B000018BF1D290AD0522918BFD22906D007E0E4
:100B1000C0687047006870478068704740687047D9
:100B20000020704770B5052914461D4616D00629C9
:100B300012D0092918BF112910D0122912D0162954
:100B400018BF17290CD01B2918BF1D290AD05229FC
:100B500018BFD22906D007E0072606E0022604E0E7
:100B6000052602E0032600E001264FF6FF729442BC
:100B700003D105F087FB841B02E0D22908BF0C34A7
:100B8000301980B200F0FAFA38B105B12C80714208
:100B9000BDE8704009B200F03BBB70BD80B5FFF707
:100BA00097FF18B1BDE8024000F00DBB01BD000089
:100BB000DFF800F0E9940010DFF800F0A1940010D5
:100BC0000A7802704A7842708A78C97802EB01216B
:100BD000418070472DE9FC410D4616461F460A9A92
:100BE0000999044601AB00F0F8F9804608BB019969
:100BF000089808703346DFF868050178491CCAB2C6
:100C0000002A06BF012101220A46017029460198E7
:100C10000271009701980279204600F00DF8804695
:100C200020B901981E2100F01DFA02E0019800F0A1
:100C3000FDF94046BDE8F6812DE9F041044684B057
:100C40000E4617469846172000F098FA050026D061
:100C50000A9A100003D04146281D904700E000206A
:100C6000010A2E70E9706F70A8700521001DADF8A3
:100C70000800ADF8001001956946DFF8E804007837
:100C80000028204602D000F059F801E000F00CF8EE
:100C90000446200004D0284600F095FA00E0132412
:100CA000204604B0BDE8F08110B50B88DFF8B82409
:100CB0000C2463431A44303A536833B94B68536089
:100CC000098950811181002010BD162010BD80B50A
:100CD000052000F00FF858B9062000F00BF838B9DD
:100CE000042000F007F818B9072000F003F800B15D
:100CF000012002BD0C2210B5DFF86C1442431144F0
:100D0000A1F1300484B06168A9B1DFF858241278E9
:100D10007AB1ADF80000019169462089ADF808006C
:100D2000608900F00BF810B1606800F04CFA002008
:100D30006060012000E0002004B010BD70B50D46D9
:100D400004462889010004D0DFF820140988814274
:100D500001D21B2070BD6868042100F059FA0646D4
:100D6000288930702889000A70702888B070288817
:100D7000000AF0702889051D4FF6FE70844213D1D9
:100D80000C20FDF7EBFC01000CD0902008704C808B
:100D900002200871CD808E60DFF8D4030078FDF763
:100DA000FEFC18E0132070BD3346AAB20021204695
:100DB000FFF7FEFE010007D002280ED0072810D052
:100DC00012280CD01F280DD1DFF8980301780A00F3
:100DD0001CBF491E0170002070BD142070BD022090
:100DE00070BD042070BD38B50446002060600879ED
:100DF000022821D1CA88042A1EDB8868017843783A
:100E0000C57801EB0321837889B203EB05230D1D1F
:100E100095429BB210D1052B18BF042B03D0062B93
:100E200018BF072B08D1218123806FF0030100F048
:100E3000EFF96060002032BD012032BD0B880370E5
:100E400002220B881B0A43700B88012B06D14A88AB
:100E5000827004224988090AC1700CE0022B0AD171
:100E60004A8882704A88120AC2708A8802710622F1
:100E70008988090A417110467047022A1BDB0A78EB
:100E80004B7802EB032202800288012A05D18A787E
:100E9000C97802EB012141800BE0022A09D18A784E
:100EA000CB7802EB032242800A79497902EB0121D7
:100EB000818000207047012070470A8802700A88EC
:100EC000120A42704A8882704A88120AC2708A885E
:100ED00002718A88120A4271CA888271C988090A15
:100EE000C17108207047082A18D10A784B7802EBA4
:100EF0000322028011F8022F4B7802EB032242807A
:100F000011F8022F4B7802EB0322828011F8022F96
:100F1000497802EB0121C180002070470120704711
:100F200004E0022A00D108E0012070470A8802701C
:100F30000988090A4170022070470A78497802EB53
:100F40000121018000207047F8B504460D46164681
:100F50001020FDF703FC070016D0A02038707D801C
:100F6000002078702EB10C223146381DFDF7A7FB0A
:100F700004E00C220021381DFDF7D3FB3946204642
:100F8000FDF70DFC0020F2BD0120F2BD2DE9F0417E
:100F900080460D4616461F462020FDF7DFFB040065
:100FA00019D0A22020706670658006982071677144
:100FB000079929B1182204F10800FDF780FB04E02D
:100FC000182204F10800FDF7ACFB21464046BDE8BD
:100FD000F041FDF7E4BBBDE8F08170B51E000446AA
:100FE0000D4621D0012104F07CFBD8B16148007886
:100FF000002100E0491CC9B2814211DA5E4B1B6836
:1010000003EB01125388002BF4D10020107001F182
:101010004000508022B1D48015723260002070BD33
:10102000152070BD142070BD012070BD10B50446A0
:1010300010220021FDF775FB23E0002200E0521C86
:101040004C4909788A420BDA4B49096801EB0211D5
:101050004B88002BF3D00B798342F0D108467047C0
:10106000002070474FF47A724A4300F109030146A9
:101070000FF2190007F089BB10B50446607A07F03B
:10108000BEFBFF20607210BD0000000010B5040020
:101090001CBF6088002807D01721204600F005F803
:1010A0002046BDE81040C1E710BD1CB504462078BD
:1010B00004280FD10020019000900A46E188207A90
:1010C0001323FFF763FFE18802B0BDE8104012224E
:1010D00005202EE013BD072170B50446002539BB5D
:1010E00018E025480068EDB200EB051630780028BE
:1010F0001CBF707AFF280CD0F088A04209D130467E
:10110000FFF7BAFF14213046FFF7CFFF3046FFF755
:101110008DFF6D1C17490978E8B28842E1D3042598
:10112000FF222146284600F004F86D1C082DF7DB4D
:1011300070BD10B50C240C4B60431844A0F1300472
:10114000608988420AD1606840B1FF2A1CBF0178DB
:10115000914203D100F037F80020606010BD00001C
:10116000DA4800208E46002058480020A44600207F
:101170008C4600208D4600209046002080B5001D42
:1011800080B2FFF719FD28B1BDE804406FF00301FC
:1011900000F03EB802BD000070B500F035F805461D
:1011A00004F1080080B204F04BFB060005D02A4889
:1011B000B48001683160066008362849096828460D
:1011C0008847304670BD38B500F01EF8224A054603
:1011D0001068002101E00146006878B100F10803C1
:1011E0009C4221BF8388C3180833A342F3D303680A
:1011F00000290CBF13600B6004F02FFB2846BDE8EC
:1012000034401649096808470446154800680047F5
:1012100038B504460D4600F00FF801000AD06842C8
:10122000204401F10803984221BF8B88C918083176
:10123000814200D2204632BD0749096841B101F11F
:101240000802904221BF8A888A1808328242F4D369
:1012500008467047000000008C47002088470020A7
:10126000844700202DE9F041DFF8945BDFF8948B90
:1012700028782824604304F0E3FAC8F8000008B98D
:1012800013202EE00027FF260FE0188018220020F0
:1012900098705E721E72987283F82400002103F128
:1012A0000C00FDF73EFA7F1CFFB2287887420BDA6C
:1012B000D8F8000004FB07F14318002F0CBF4FF6CD
:1012C000FE704FF6FF70E0E70FF2D140FFF7F7FA3C
:1012D0000FF6E930FDF7D2FD0FF63D4004F043F97B
:1012E0000020BDE8F081DFF8201B08707047F0B5E2
:1012F00083B000F0BDF907000DD129462046FDF767
:10130000C0FD070007D10198DFF8003B00960322DB
:10131000294600F02CFD3846FEBD70B588B0044665
:101320000120ADF808000D464FF6FF70ADF80A0039
:1013300001A902208DF80C00002000F07CF900F0DB
:1013400036FD06000CD102A92046FDF7F7FD060088
:1013500006D10198DFF8B83A0095112200F069F93A
:10136000304608B070BD2DE9F0411646022E18BF78
:10137000102E88B080460D461F4622D10DB301A91C
:1013800000F015FD0446E8B90120ADF808008DF81D
:101390000C604FF6FF70ADF80A00324629460DF199
:1013A0000D00FDF78CF902A9404600F0E1F8044673
:1013B00040B90198DFF85C3A0097072200F039F94C
:1013C00000E00224204631E100B587B000F01BF8B0
:1013D0008DF80510ADF8022028218DF806100022A6
:1013E0000CE000B587B000F00EF8ADF80220032144
:1013F0008DF80510002228218DF80610694600F0AE
:10140000E0F807B000BDADF8001002218DF804101F
:10141000704713460122D4E070B584B00446ADF89D
:101420000410ADF806201D4602A900F0C0FC06001D
:101430000DD101A92046FDF737FD060007D102981E
:10144000DFF8D4390095052201A900F090FC304660
:1014500004B070BDF6E013460022B2E00DE1F0B535
:1014600083B000F005F907000DD129462046FDF7AD
:1014700053FD070007D10198DFF8A03900960F222D
:10148000002100F074FC3846FEBD38B500F019F8B4
:10149000172807D0287A002804BF687A012800D1CD
:1014A00014E0022032BD38B500F00BF8172807D041
:1014B000287A012804BF687A012800D106E00220BA
:1014C00032BD0D460446694600F071BC29462046EF
:1014D000FDF740FD32BDE6E008E12DE9F0410E00E8
:1014E00086B0804617461D4639D0380037D0404672
:1014F00004F0C8FEC0B20021C9B20C234B433344F0
:10150000421F9B889A4201DA1B202AE0491CCAB27A
:10151000BA42F1D301A9404600F049FC04001FD1B2
:10152000B0680090B38872883188404600F012F9A4
:10153000040015D100208DF811008DF810700120E5
:101540008DF8080003968DF8125017220C98DFF8DA
:10155000D038009002A9019800F009FC00E00224B4
:10156000204606B0BDE8F0816CE086E09BE0BDE07F
:1015700030B50D4685B02A79044600230621FFF7D1
:10158000D1FA0390C8B12888ADF80000691D6888B9
:1015900000F056FB002000F04DFB2A790398ADF8CF
:1015A0000820FDF78CF869462046FDF787FC04000B
:1015B00004D00398FFF707FE00E01324204605B08F
:1015C00030BD2DE9F04188B00D46044690461F46D7
:1015D00001A900F0ECFB064638BB5FEA08000FD01B
:1015E0002888ADF8080002A96888ADF80A00022032
:1015F0008DF80C00032000F01EF8FDF771FC03E0ED
:1016000029462046FDF76CFC06000ED1162229461D
:101610000DF10A00FDF753F80198DFF808388DF84E
:1016200008800097092200F004F8304608B0BDE8B1
:10163000F08102A99BE38DF80D0028208DF80E00A3
:1016400020467047F0B583B000F012F807000DD1C6
:1016500029462046FDF750FC070007D10198DFF826
:10166000C83700960B22002100F081FB3846FEBDF2
:101670000D460446164601A999E3F0B583B0FFF77D
:10168000F7FF07000DD129462046FDF73BFC070078
:1016900007D10198DFF8943700960D22294600F013
:1016A00066FB3846FEBDF0B50D4683B00446287A89
:1016B000002804BF687A0028164614D101A92046E4
:1016C00000F075FB07000FD129462046FDF742FCCC
:1016D000070009D10198DFF858370096132200213E
:1016E00000F045FB00E002273846FEBDF0B587B0AC
:1016F0000D460746144601A900F059FB060026D105
:10170000384604F0BFFDAB88401F834203DB3846F8
:1017100004F0B8FD431FA86800906A8829889BB22E
:10172000384600F017F8060011D100208DF80800A7
:101730000C22294603A8FCF7C2FF6888DFF8E036D0
:10174000ADF81800009417220198FFF772FF304699
:1017500007B0F0BDFEB50D4616461F4604460023F1
:101760003A461621FFF7DEF9029098B10899ADF8D4
:101770000050ADF80260ADF804703A46FCF79FFFE8
:1017800069462046FDF70AFC040004D00298FFF7E2
:101790001AFD00E013242046FEBD00002DE9F043B1
:1017A0000E4687B0804630781746002460B97078BE
:1017B000012809D0B0781B2818BF1D283CD1DFF8BC
:1017C00048562978FF2901D1062091E01D2812D121
:1017D000404600F000FB04000DD0A27A10000AD0B1
:1017E00010062ED4B1784046FFF75BF9A07A40F09E
:1017F0008000A07225E001A80090B388B2687178DB
:10180000307804F095FC0028814670D101A8009042
:101810000022B37828784146FFF7E7F80028814690
:1018200065D1029808B100203870B0781D285ED1CB
:10183000002C5CD0A0725AE0404600F0CCFA0400C4
:1018400001D1002054E0B07801281DD1B188B068E2
:1018500001AA04F0A7FA5FEA000948D1A078052898
:1018600018BF072808D009281CBF0D28112803D04D
:10187000172817D12069A8B1B27801AB214640469C
:1018800000F037F8387032E0A178884207D16368F9
:10189000180004D0B188B06801AA9847DBE74FF080
:1018A000040924E0DFF88C25607A127890420FD08A
:1018B00001A900910022B3784146FFF796F88146CE
:1018C00030B9B17801A8FFF703F908B100203870EA
:1018D000A078032808D1A189BDF80400814288BFFF
:1018E00001464046FFF7CAF8204600F0AFFA4846E6
:1018F00092E12DE9F8450D468246A878052816465E
:101900001F464FF0010847F230540BD007280FD084
:10191000092834D00D2839D011285AD0172800F0C2
:1019200080808DE03A463146284600F0B0F82BE042
:10193000072E19D195F82400EA89401C85F8240067
:101940003988786800EB810010F8041D407801EBBD
:10195000002081B2914210D2401CA88105F10C01F7
:101960002888FFF705FE56E038790A2828D195F82F
:101970002400441EA441E40F23E0002421E03A4661
:101980003146284600F0B3F804461AE00D2E14D173
:1019900095F82400401C85F82400288804F072FC87
:1019A0003988401E8142E8DBE8890818E88105F1A2
:1019B0000C012888FDF7A6FA2DE038790728D6D043
:1019C0000124002C08BF012E3BD138790A283DD1D3
:1019D0004CE0112EC8D138887988401E484395F8CC
:1019E0002410491C85F8241080B279680844817855
:1019F000C07801EB002080B24FF6FF718842BCD066
:101A0000401CA88180B2E9898142B6D3288805F1BB
:101A10000C01FDF793FA287A214606F0BEFE162443
:101A200014E0287B01283A463146284602D100F0CE
:101A30004AF901E000F00FF90446012CC1D023E07F
:101A40000124092E04BF388800280ED000973346A1
:101A5000687A00225146FEF7C8FF30B93146384651
:101A6000FFF736F808B14FF0000844B900200090A5
:101A70001A22AB78687A5146FEF7B7FF01E0162CC0
:101A800002D0284600F0E2F94046BDE8F28510B5E4
:101A90000529044621D100F0C2F8516810889278D7
:101AA000012A03D101EB8000001F03E01222504302
:101AB0000844123801784078E28901EB002080B2B6
:101AC000904212D2401CA08104F10C012088FDF745
:101AD000EBF900F0AAF8162010BD10790A2802D1FF
:101AE00094F8240008B9012010BD002010BD2DE994
:101AF000F043092987B0044615463CD128886988F7
:101B0000401E484394F82410491C84F8241080B2E5
:101B100069680A5C0844407802EB0026207B0128B3
:101B200054D128886988002748431FFA80F82F80FD
:101B3000B946C1454ADA6888A17C431F68684844B1
:101B4000421D9BB204F1130004F04BFB70B1B94588
:101B500006D068686A8800EB09013844FCF7AFFDDD
:101B60006888C7192888401CBFB228806888484404
:101B70005FFA80F9DDE728790A2803D194F8240078
:101B8000002848D1A37CAC4800F060F8002837D189
:101B9000A37CAA4800F05AF8002831D1A37CA848B9
:101BA00000F054F800282BD1A37CA64800F04EF892
:101BB00030BB2879022818BF052804D008281CBF8C
:101BC0000F280C281CD100F02AF86E88B6B24FF608
:101BD000FF7086421FD0218A8E421CD2217B701C4E
:101BE0000129E0810ED1ADF800006946208A00F09D
:101BF00027F8032000F01EF82088FDF771F906E0B1
:101C0000012009E0208804F10E01FDF769F900F0D8
:101C10000CF8162000E0002007B0BDE8F08394F82F
:101C20002400401C84F824007047207A47F2305189
:101C300006F0B3BD8DF8050028208DF8060070472A
:101C4000ADF8020002208DF80400704704F1130281
:101C5000022104F0C6BAF0B50E46172E83B0044632
:101C600047F2305522D1208804F00CFBA18BA38AC7
:101C7000421F5118A183A28B618A511A89B29942DD
:101C800012DAA0F1050C5F1ABC45B4BF431F5B1A02
:101C9000A069084400909BB2218A2088FFF75AFD72
:101CA00020B900F060F80CE0012000E0002000F016
:101CB00054F8012E01D10120FEBD00F054F800F0CF
:101CC00047F81620FEBDF0B50E460446172E83B029
:101CD000104647F230552ED1627D21690C277A4398
:101CE0008B1802881988914202BF59884288914214
:101CF00002BF8288998891421DD181689868FCF75B
:101D000002FDC0B1607D227D401CC1B29142607570
:101D10000FD22169C0B278430F18B8680090BB8811
:101D20007A8839882088FFF715FD20B900F01BF864
:101D30000CE0A07D00E0002000F00FF8012E01D1A2
:101D40000120FEBD00F00FF800F002F81620FEBDE5
:101D50001920A0703C48606070478DF8040001A90C
:101D60002088FDF72BB9207A294606F016BD2DE90B
:101D7000F041069CFF2C05460E461746984614D0A7
:101D800005F108031E2229460FF24D10FEF758FEFA
:101D90006C72AF70C5F804803EB1314605F10C009D
:101DA000BDE8F0411822FCF78ABCBDE8F08110B50F
:101DB0000C4600F010F860B104B12060007AFE28F3
:101DC00001D1172010BDFF2801D1002010BD162021
:101DD00010BD022010BD10B50A4A1268002100E0B3
:101DE000491C074C2478CBB2A34207D2C9B228239E
:101DF0004B43D45A8442F3D1D01810BD002010BDFB
:101E0000D7480020F8470020A8460020DF5D0100E9
:101E100053600100C15E0100195E01003F600100D6
:101E2000C7600100495F01008B5F01000560010090
:101E3000B95F0100D8480020E0CC0100E4CC0100EB
:101E4000E8CC0100ECCC010013610100F8B50446B8
:101E500004F10800FEF7FCFDA51C04F1100628782B
:101E6000172818BF19281AD1A87A012813D1306869
:101E7000A8B1002708E00C2179430844806808B124
:101E8000FFF7A1F97F1CFFB2317930688F42F2DB96
:101E900003F0E3FC03E0B06808B1FFF794F9002019
:101EA00028701822FF20E87100210020307504F10D
:101EB0000C00BDE8F840FCF734BC000010B50C463F
:101EC000FFF789FF30B1817A4A1C944204BF01F0C8
:101ED0008001817210BD000010B582B004001CBFEB
:101EE000207AFF2816D000200090A3782188607AFD
:101EF0001722FEF77AFDA078182806D100208DF869
:101F0000000069462088FDF759F8FE20207220461F
:101F1000FFF79CFF13BD000070B504464FF6FE703E
:101F2000844282B037D008004FF6FF760AD12046AF
:101F3000FFF751FF78BB3046FFF74DFF05002AD071
:101F4000048073BD012906D12046FFF744FF050038
:101F500021D02E800BE002291DD10121204603F063
:101F6000C0FBC0B92046FFF736FF050013D0287A22
:101F7000FF280ED0FE2807D0002000901422AB7856
:101F8000687A2146FEF731FD2846FFF75FFFFF2004
:101F900028720020A87273BD70B5DFF8305A287817
:101FA0000624604303F04CFCDFF8241A086008B9EB
:101FB000132070BD0020FF2206E03380401C002368
:101FC000F270B2703371C0B22B7898420ADA0B68A3
:101FD00004FB00F61E4400280CBF4FF6FE734FF6BC
:101FE000FF73EAE70FF25140FEF766FC0FF615109B
:101FF000FDF716F80FF6551003F0B5FA002070BD86
:1020000070B50446208868B160680378426800F0C3
:1020100040F948B9606803784268DFF8B80900F011
:102020003AF908B9022070BDA078C01F0A2801D370
:10203000182070BDDFF8A0592888010004D021883D
:10204000C0F58030884201DA012070BD0C2003F019
:10205000F7FB060001D1132070BD002008E0626884
:10206000298880B202EB0012401C5181491C298052
:1020700081B222889142F2D30020306008222146AA
:10208000301DFCF71CFB686810B96E6004E0084660
:1020900001680029FBD10660002070BD38B50246FA
:1020A0000846DFF834194C68002301E02346246811
:1020B00094B1A5686D899542F8D12268002B0CBFB8
:1020C0004A601A6018B10822211DFCF7F8FA204670
:1020D00003F0C3FB002032BD012032BDDFF8FC1845
:1020E0000870704710B5044610461422114203D000
:1020F00000F0DAF8012204E04A0608D500F0D4F82E
:10210000002201462046BDE8104003F02CBBC80762
:1021100001D4022010BD002010BD70B505460E464A
:10212000B0061C4609D5104600F0BEF80146284608
:10213000BDE87040012203F016BB8820064210D093
:10214000104600F0B1F8014606F00802284603F0F8
:102150000AFB010009D0617A41B1217A012904D03A
:1021600070BDB00701D4032070BD002070BD2DE903
:10217000F0478146DFF8600844688A4690461E466C
:1021800000E02468FCB1002700E07F1CA188B8B201
:102190008842F6D2A068BFB200EB071568894845AF
:1021A00028BF8245F1D33EB129786868334642465C
:1021B00004F017F80028E8D0089810B1A168498900
:1021C0000180284600E00020BDE8F087F0B5DFF888
:1021D0000828546800E02468E4B1A5686E89B0421C
:1021E000F9DBA788BA199042F5DA4FF0000C01E04C
:1021F00003F1010C1FFA8CF2BA42ECD21FFA8CF3F5
:1022000005EB0312B2F80AE08645F1D101B10E8068
:102210001046F0BD0020F0BD2DE9FC41044600272A
:10222000ADF804704FF6FF786089404515461E46AC
:1022300008D001AA0092401C2378626880B2FFF7A0
:1022400096FF07462378626800F023F830B92378B8
:102250006268DFF8800700F01EF808B160890CE0C2
:1022600023786268DFF8780700F015F858B11FB1DD
:10227000BDF80400A84203D0284600F0D2F803E0DD
:102280007889404400E0608906B130803846BDE876
:10229000F681DFF85007022103F0A3BF80B500F0FC
:1022A000F3FA00B1008802BD80B500F0EDFA08B184
:1022B000807802BD102002BD70B5012982B00446AD
:1022C000154616D0032918D0052925D0072927D06F
:1022D000092929D00B292BD00D292DD00F292FD03A
:1022E000112931D0132933D0172934D0192936D0E8
:1022F00039E02946FCF797FE33E0FCF7ACFDADF87A
:10230000000069462046FCF797FE06002CD129887C
:102310002046FEF7B3FB27E02946FCF799FE20E0B4
:102320002946FCF7ADFE1CE02946FCF7B9FE18E093
:102330002946FCF7CBFE14E02946FCF7D5FE10E059
:102340002946FCF7DFFE0CE02946FCF7EAFE08E030
:10235000FCF7F8FE05E02946FCF7FAFE01E0FCF781
:1023600004FF064600E00226304676BD2DE9FC411A
:102370000E46054617461C4601A900F092FA804613
:1023800038BB380014D00020ADF800006946308812
:10239000FFF71CFF012FBDF8000018BF0027FFF753
:1023A00083FF01463A46284603F0DDF9804680B9AE
:1023B00031462846FCF7EAFE804650B9019DFF2CC5
:1023C00007D0AB1C1E2229460FF25550FEF738FBF2
:1023D000EC704046BDE8F6817CB50D4604461646D5
:1023E00001A900F05EFA17281AD0300014D000209E
:1023F000ADF8000069462888FFF7E8FE012EBDF819
:10240000000018BF0026FFF74FFF01463246204666
:1024100003F0A9F9010003D129462046FCF7ABFEE1
:1024200076BD10B50446FFF739FF01001CBF611EE1
:102430000C18A0B210BD00002DE9F0430D4689B084
:102440008146A87800261E28174614D1484600F079
:102450003CFA06001EBFB078FE28FF2822D00020DC
:1024600000900022AB78F0784946FEF7BEFA30467D
:1024700000F040FA16E0122804BF6878012813D053
:10248000484600F022FA06000ED0327910000BD038
:10249000100607D4A9784846FEF703FB307940F0D0
:1024A00080003071002069E0DFF830452078FF2897
:1024B00012D0A878811E17290ED200F08AF958B1DF
:1024C000A87800F0B3F938B1287810B968780128F5
:1024D00004D1A878122801D006204FE0A87800F097
:1024E00078F9844602A80090AB88AA6869782878B1
:1024F000E0470028804640D1A87800F097F90246CE
:1025000002A9484690478046D8B9AB78042B34D00E
:1025100002A80090002220784946FEF766FA80461D
:1025200058BBA97802A8FEF7D3FA08B1002038708A
:10253000A878122804BF697801291ED0EEB1307145
:102540001BE06878C8B9A8788DF800008DF8048081
:102550006946A878042818BF0628BDF80800ADF819
:1025600002004846FCF75FFD28B16B4601221621A8
:102570004846FEF779FA4FF00008404609B0BDE83A
:10258000F083002070472DE9FE430D4680462888E1
:102590006988814201D3010001D101206DE0002151
:1025A000ADF8041002914FF6FF7900E0401C0021C5
:1025B000009100236988002280B2FFF7D8FD070050
:1025C00037D0BDF80400002838D16B464A460521B3
:1025D0004046FEF7A7FA040001D111204DE0029415
:1025E0003878022806D101208DF80600BDF80000D9
:1025F000860827E002208DF806001221BDF80000B1
:1026000090FBF1F63878102813D1788904F8010B83
:10261000102200F034F81034BDF80400401CADF86E
:102620000400B1B2BDF80400884202D2788948455E
:10263000BCD1BDF8040080B90A201EE09DF8060058
:102640000128DFD138780228F3D1788904F8010B0A
:10265000022200F014F8A41CDEE701A94046FCF7B2
:10266000F7FC48B101AB052216214046FEF7FCF904
:1026700010B10298FEF7A7FD0020BDE8FE8378891F
:10268000000A04F8010B20467968FCF718B810B569
:1026900082B04C880888844201D3020001D1012015
:1026A00016BD00F016F808B90A2016BD002016BDA8
:1026B00010B582B04C880888844201D3020001D151
:1026C000012016BD00F005F808B90A2016BD00204B
:1026D00016BD002200924A1D0B79214647E510B530
:1026E000044682B0084669460088FFF76FFD08B9C6
:1026F000012016BD017ABDF800202046FFF7F2FC4C
:1027000016BD70B582B006460D46002401E0641C7B
:10271000A4B2A888844229DA286810F8142000EBB3
:1027200044006946407802EB002080B2FFF74EFD7E
:1027300050B9286810F814100170286800EB4401A3
:1027400049784170012076BD017ABDF800203046FD
:10275000FFF7C8FC0100DAD0296811F814200A70CC
:10276000296801EB440252784A7076BD002076BD9C
:1027700010B50C4682B020886188814200D308B928
:10278000012016BD23799748621DFFF784FD08B923
:10279000102016BD00200090237961882088621DDA
:1027A000FFF7E5FC08B90A2016BD002016BD38B5B4
:1027B00004460D4669462888FFF708FD08B9012040
:1027C00032BD017ABDF800202B462046FFF7A5FC5C
:1027D00032BD022814D0042814D0062814D00828AA
:1027E0001AD00A2812D00C2812D00E2812D0102885
:1027F00012D0122812D0162812D0182812D013E0A6
:1028000079487047794870477948704779487047E8
:1028100079487047794870477948704779487047D8
:10282000794870477948704700207047022814D0D3
:10283000042814D0062814D0082814D00A2818BF59
:102840000C2812D00E2812D0102812D0122818BF2F
:10285000162810D0182810D012E06D4870476D4827
:1028600070476D4870476D4870476D4870476D48B8
:1028700070476D4870476D4870470FF20900704708
:1028800000207047002070475349496800E00968FC
:1028900029B18A6852898242F9D1081D7047002007
:1028A000704710B50C4600F010F860B104B120601C
:1028B0008078FE2801D1172010BDFF2801D100200B
:1028C00010BD162010BD022010BD10B5404A126880
:1028D000002100E0491C3D4C2478CBB2A34207D232
:1028E000C9B206234B43D45A8442F3D1D01810BD49
:1028F000002010BD10B50446A01CFEF7A9F8FF206B
:10290000E07010BD10B50C46FFF7DFFF30B1017964
:102910004A1C944204BF01F08001017110BD000007
:1029200010B582B004001EBFA078FF28FE280BD08F
:10293000002000901E232188E0781722FEF755F82A
:10294000FE20A070FF20E07013BD000070B50446AB
:102950004FF6FE70844282B037D008004FF6FF7603
:102960000AD12046FFF7B1FF78BB3046FFF7ADFF35
:1029700005002AD0048073BD012906D12046FFF747
:10298000A4FF050021D02E800BE002291DD10121DA
:10299000204602F0A6FEC0B92046FFF796FF0500CC
:1029A00013D0A878FF280ED0FE2807D00020009072
:1029B0001E23E87814222146FEF717F82846FFF771
:1029C00099FFFF20A8700020287173BDD748002010
:1029D000FC470020E4CC010008460020A946002066
:1029E000ECCC0100E0CC0100C55D0100F75D010009
:1029F000775E01006D5F0100DD5F01001B6001007B
:102A00000B5F01008D5F0100816001000161010029
:102A100083250100872501008F260100B1260100D2
:102A2000DF2601000327010071270100AF27010005
:102A3000DFF8581C0870704738B5DFF8544CDFF8E1
:102A4000545C20762878C00002F0FAFEE061C8B13C
:102A5000002108E04FF6FF7220F8312000EBC1039F
:102A600000225A60491C2A789142F3DB052000F0CD
:102A7000AFF8207EFFF732FBBDE83240DFF8180CDC
:102A800002F071BD31BD38B50C46200418D5DFF811
:102A9000000C007EFBF7E1FE05000ED02878B02880
:102AA00008D1284600F0FDF820B1297905F1080089
:102AB000FEF774F82846FBF763FE84F4004032BD4D
:102AC000002032BD7CB506001C460DD0ADF80010CC
:102AD0008DF8022001966846FFF792FA05001AD198
:102AE000CCB17689300001D1022514E00C2002F02F
:102AF000A7FE08B913250EE00021016086808460DE
:102B0000DFF8981B0A6812B9086004E00A461168E9
:102B10000029FBD11060284676BD30B50C46DFF8A1
:102B20007C1B0546086883B0002201E0024600686D
:102B300098B18388AB42F9D10368002A0CBF0B60BF
:102B4000136002F08AFE69462846FFF7A7FA0100E3
:102B500002D10CB1019921603EBD01203EBD70B58E
:102B600050BB012926D1DFF8280BC169002300E002
:102B70005B1CDFF8204B2478A34217DA31F833408E
:102B80004FF6FF75AC42F3D0002400E0641C467E93
:102B9000E5B2B542ECD201EBC305E4B26D680C2698
:102BA0006643AD5B002DF1D0012070BD1078BDE80B
:102BB00070400DE0182070BD022070BD002200287A
:102BC00003BFDFF8CC0A407E08700222104670472F
:102BD0002DE9F843DFF8B87A0446002078760C2512
:102BE000F869DFF8B06A406805FB04F870B102F0DC
:102BF00034FE002006E0F969C0B201EBC0010022FA
:102C00004A60401C3278C1B29142F4D3307808FB5C
:102C100000F080B202F014FE5FEA000928D030789C
:102C200008FB00F200214846FBF77BFD00200FE087
:102C3000516805FB0CF34FF0000E21F803E0194436
:102C40000CF1010CC1F808E0A445F1DBC144401CC3
:102C50003278C1B2914208D2F969C0B201EBC00228
:102C60004FF0000CC2F80490EEE77C76002000E004
:102C70001320BDE8F28301460020C90705D50023D3
:102C800010220121DFF8180C1CE77047DFF80C1A3E
:102C9000096821B18A888242FAD188687047002089
:102CA00070472DE9F04186B004460020ADF81000D1
:102CB00001208DF81200DFF8D859286A38B9FCF7DE
:102CC000CAF802F0BDFD0028286200F0E280182258
:102CD00000212846FBF725FD2079461C02284FF6E7
:102CE000FF7817D006282CD008282FD00A2833D0F8
:102CF0000C2857D00E2800F08B80102800F08D8013
:102D0000122800F08F80162800F09380182800F019
:102D10009780BBE0FCF79FF8288029466088FCF785
:102D20008BF900282189288804D0814228BF0146D8
:102D30002980A0E0814228BF01466088FDF79EFE01
:102D4000A4E004A9204600F0AEF87DE004AA00212A
:102D5000204600F02CF977E000F0A0F8070052D0F0
:102D6000608805AB42460B21FDF7DCFE03006B607B
:102D700024D02079BDF81620039000953946BDF87F
:102D8000140002900020019000F026FA070004D100
:102D900060882946FCF79AF929E0162F686808BF71
:102DA00000272BE000F07AF807002CD0608805ABF4
:102DB00042460D21FDF7B6FE686020B92089ADF8C6
:102DC0001000112745E02179BDF816200391034634
:102DD000BDF814100291618901910095394600F007
:102DE000FBF9070006D160882946FCF77DF9002829
:102DF00041D12AE0162F686808BF0027FEF7E3F9E3
:102E0000380001D121E001272089ADF810001CE035
:102E100004A9204600F06EF916E004A9204600F04F
:102E2000E9F911E00DF1120204A9204600F086FA3A
:102E30000AE00DF1120204A9204600F0C0FA03E0F6
:102E400004A9204600F029FB0746380011D0162FB0
:102E500011D0607814280CD0207928702F71294661
:102E6000BDF8100068806088FCF7DDF808B1012625
:102E700001E0162F0AD160882B46F2B21621FDF729
:102E8000F3FD18B1F1B22846FDF788FE2046FDF7A4
:102E900022FD9DF8120006B0BDE8F08120890DF1F9
:102EA0001601FFF793B92DE9FA47044686B060880A
:102EB000DFF8DC5703F0E6F980460DF1120000F070
:102EC000D4F8002781464FF0FF0AB9F1000F5BD01C
:102ED00009E0BDF810304354BDF81000696892B2A3
:102EE000000A8854571CBFB2A8F1050087424BDA8C
:102EF000207903900026A8F1070080B20290019685
:102F000005F11A0000902B6ABDF81220608849462E
:102F100000F0CCFB002802BF6A8B208A904214D1BB
:102F2000296A6069FBF7EFFB78B1686858B900F06F
:102F300055F90721FDF7F6FD686020B9069920894B
:102F40000880112030E0B9F80A60BDF812206189CC
:102F500004AB4846FFF760F9002E8146B5D068689B
:102F6000C655781C6A6880B231121154411C4A1C43
:102F70006868B9F1000F89B2ABD100F801A092B234
:102F8000686800F802A0571CB8B248B13F04B80CFA
:102F9000288029466088FCF773F828B1162003E0E2
:102FA0000699208908800A2008B0BDE8F0872DE93D
:102FB000F043044685B060888846914603F062F984
:102FC000851EADB2DFF8C87601E0401C2081A81E46
:102FD000398988422FDB5FEA08002CD104A800F071
:102FE00044F8060027D070892081BDF81020317A7E
:102FF0006088FFF777F85FEA00081CD120793B6A08
:10300000BDF8102003903146A81E80B200F0EBF806
:1030100000F0E2F85FEA00080DD173897A8B396A13
:10302000608800F02AF85FEA000804D120894FF692
:10303000FF718842C9D1388901000AD0798890FB94
:10304000F1F0388039466088FCF72AF850B1162034
:1030500008E05FEA08002089A9F8000008BF4FF0E7
:103060000A08404605B0BDE8F0830090237B6189E3
:10307000208904F10D02FFF77AB82DE9F84682465F
:10308000894615461E4603F0FDF8DFF8044607465C
:10309000208990B900F0A3F809215046FDF742FDC0
:1030A000606008B9112023E0A81C60803A1F2089C5
:1030B00001466B189A4206D203E06088A91C884238
:1030C000F4D0012014E0401C20816068465420891F
:1030D000411C2181310A62681154606823892A46A3
:1030E00049461844FBF7EBFA208928182081002074
:1030F000BDE8F2862DE9F047044686B06088DFF827
:1031000090750D4603F0BEF80026A0F10109A0F16C
:10311000010814E03888798B0346C9188845BCBF7C
:10312000A9EB0000788378687A8B396A1844FBF73A
:10313000C6FA3888798B0818761C3880B6B2A08910
:103140008642BCBF3888404534DAA06810F81620A3
:1031500000EB460004A9407802EB002080B2FFF7A4
:1031600035F8010009D14FF0010A00F02BF878681A
:1031700008B1FEF728F85046DDE02079BDF81020B0
:1031800003901FFA89F000F02EF83B6A00F024F853
:1031900000288246E9D178680028BBD100F01EF8EB
:1031A0000F21FDF7BFFC00287860B3D100F00AF8CA
:1031B0001120E1E760883946FBF7A4FF0028DBD047
:1031C0001620D9E7A06810F8161000EB46004078EA
:1031D00001EB002028807047608867E26088002348
:1031E0004FF6FF72704702900020019007F11A001D
:1031F000009070472DE9F047044686B06088DFF8FC
:103200009054894603F03EF8059004F10D0204A89D
:103210000090237B61892089FEF7A9FF0026B24632
:1032200007464FF0FF0810E0696801F8068080B299
:10323000696801F80080461C68686A8B296AB6B222
:103240008019FBF73CFA688B8619B6B2FFB1BDF85E
:103250001020397A6088FEF745FF5FEA000A13D133
:103260002079BDF81020039039460598801F80B260
:1032700002900020019005F11A0000902B6AFFF7E0
:10328000ABFF5FEA000A10D07889A9F80000002E91
:1032900048D0688896FBF0F0288029466088FBF7C4
:1032A00040FF002847D0162045E07EB9FFF796FF83
:1032B0001121FDF737FC686020B97889A9F8000072
:1032C000112038E0688B001D688009E0688B6988F0
:1032D000021D9142DDD10599891F80198142D8DBF9
:1032E00069687889885579896A68701C80B2090A8A
:1032F0001154461CBDF8102061890DF112033846A7
:10330000FEF78AFF0746701C002FB6B28CD06A68A1
:10331000BDF81210915580B2BDF812106A68090A02
:10332000115488E75FEA0A002089A9F8000008BF65
:103330004FF00A0A504606B0BDE8F087FEB50446D5
:103340000D462089164602A9FEF740FF07002ED041
:10335000387A80060BD5BDF8080000F0A1F903000B
:103360000BD06088122239469847070020D1607C34
:10337000002814BF5220207901E00E2718E00190A8
:10338000002000906389E2682189608800F08AFA51
:10339000070007D1607C68B96088FBF7D3FE48B1AD
:1033A0001620FEBD162F03D10027377002E001273B
:1033B00020892880607C00B100273846FEBD2DE9B9
:1033C000F041044682B00D4660889046012102F02B
:1033D00088F9002718B9142060700E205BE020895E
:1033E0006946FEF7F3FE060051D0307A80060BD511
:1033F000BDF8000000F054F9030013D060881222D9
:1034000031469847070043D16688304600F008F9F6
:1034100028B94FF6FF7000F003F9A0B30680002131
:103420009B4E02E00E2733E0491C737ECAB29A42DB
:1034300029D24268C9B20C234B4313441A88002A8C
:10344000F2D10C2204F108011846FBF738F90020EC
:1034500088F800000C2204F108013046FBF72FF930
:10346000A289608800231721FDF75CFBB06060B182
:10347000A2892169FBF723F960883146FBF768FED2
:1034800040B1162007E0092702E0112700E00127DC
:10349000208928803846BDE8F6812DE9F0430446AE
:1034A00083B06088894600F0BBF800265FEA000818
:1034B0004CD0207A012845D1414604F1080000F0A3
:1034C00051F8A0B1D8F804701820019078880090C5
:1034D000BB88BA683988608800F0E4F90646162E81
:1034E00002D10020B8602DE060B3388828E00027C2
:1034F0000EE0019068880090AB88AA68608800F0B0
:10350000D1F90646162E18D10020A8607F1CFFB204
:103510005F48407E874215DAD8F804100C227A43BF
:103520000A44154629880B000CD07B1C83421DBF22
:103530009089002816201820DBE7002EE6D0288886
:10354000A9F80000404600F080F82EB96088FBF72B
:103550000CFE20B1162003E0162E08BF00263046D0
:10356000BDE8FE832DE9F84F0C4600200027002619
:103570004FF00C0B46490DE0984202BFBCF80250D8
:1035800093B2AB4224D1BCF80430DF19BFB29A1811
:1035900092B2761C4B7E9E420FDA63680BFB06FCF0
:1035A0009C44BCF8003043B10028E5D1BCF804705D
:1035B000BCF802201846BA18EAE7022E2DDB3800C4
:1035C0004FF0000904D0FDF7E7FD5FEA000801D1E4
:1035D000002023E0CA461AE00BFB0AF14518A9684F
:1035E00059B1AA8808EB0900FBF769F8A888484494
:1035F0001FFA80F9A868FDF7E6FDBAF1000F04D0C4
:103600000C2200212846FBF78CF80AF1010AB2458A
:103610006068E1DBC0F8088087800120BDE8F28F98
:1036200010B51B4AD269002100E0491C194C2478CE
:10363000CBB2A34207D2C9B232F831308342F4D1BF
:1036400002EBC10010BD002010BD70B5044600257E
:103650000BE0B06808B1FDF7B6FD0C220021304642
:10366000FBF75FF8002030806D1C0949497EE8B205
:10367000884207D26068EDB20C2169434618308851
:103680000028E6D14FF6FF70208070BDA6460020CE
:10369000C8470020204800204B390100EC4700209B
:1036A00080B5FFF7F3FA00B1806802BD2DE9FE4F47
:1036B0000D468046287AC00693461E464FF0000A03
:1036C0000CD55846FFF7ECFF030000F0E4800A2217
:1036D0002946404698470028824649D128780C9FC1
:1036E0000D9CDDF83890022816D100F018F94FF43F
:1036F0002051401A012810D9801E3AD0401E14D003
:10370000FD3876D0401E00F07D80401E6AD0401EFD
:103710006FD0401E00F09180A7E0002C2AD1E8680D
:10372000017839800278416883E0002C22D10120A1
:1037300038800021E868007830706889401C80B2C9
:10374000FEF744FD398860B10278921C5118398027
:10375000418971704189090AB17002784168F01C91
:1037600068E0081D388004220021701CFAF7D9FF98
:1037700093E0002C62D1E86804880420388034701B
:10378000200A70700DF102012046FEF71FFD0500B2
:103790001ED0EC68BDF802204FF6FF786B4641461C
:1037A000FEF73AFD40B92B786A688B48022102F097
:1037B00018FD08B9ADF80080207802280AD16168A8
:1037C0000222301DFAF77BFF3888801C388001E028
:1037D000ADF80040BDF80000B070BDF80000000A70
:1037E000F0705AE054BBE8680168404605F09CF868
:1037F00002E01CBBE8680088022139803070000AB2
:1038000070704AE0E868FAF758FF82B2A242B8BF87
:103810004FF0070A41DB944208BF002206D009EBB3
:1038200004019142B2BF4A46121B92B23A80E96843
:1038300021443046FAF743FF2FE014B14FF00B0A52
:103840002BE0E86807213980017831704178717088
:103850004188B1704188090AF17001793171C188DC
:103860007171C088000AB07117E05846FFF70EFA70
:1038700000281CBFD0F800C0BCF1000F0BD00F987F
:103880000290CDF8049000943B46324629464046CB
:10389000E047824601E04FF00E0A5046BDE8FE8F39
:1038A000F84500202DE9FE438046894617461E460E
:1038B00002A94846FEF78AFC05002CD0BDF8080096
:1038C000FFF7E4F900281CBFD0F804C0BCF1000FDA
:1038D0001FD00A980B9C0090019433463A46294623
:1038E0004046E0470646B8B9FE2C15D02878022895
:1038F00012D100F014F842F6021188420CD1387847
:10390000797800EB012082B24946404600F047F842
:1039100002E00E2600E001263046BDE8FE8368681E
:103920000178407801EB002080B27047E0B58DF857
:1039300008200223120A8DF80920FE22019200229B
:10394000009202AAFFF7AEFF0EBD7CB50129044626
:1039500005D0022922D1012101F0C3FEF0B9204691
:10396000FFF75EFE08B1FFF770FE01A800904FF66A
:10397000FF750223194A29460120FEF7F8FB0BE0E8
:10398000F0680168204604F0B5FFBDF8042000236C
:1039900029463046FEF740FC0600F1D173BDF8B56C
:1039A0000F4F04463878FF280D46164611D00A20DE
:1039B000FAF7D4FE68B1B121017044800021417052
:1039C0000171C580068101463878BDE8F440FAF7F8
:1039D000E6BEF1BD00000000E4CC0100F0CC010027
:1039E000A6460020F8B5022702291CBF08290C2989
:1039F0000C4615461E4615D100F00CFC070011D1EF
:103A00000799069800F01AFC304600F024FC012CBF
:103A100014BF042C0025284600F06CF800F02CFBA5
:103A200004F0A2FF3846F2BDDFF800F0159900104F
:103A3000DFF800F04199001070B5DFF8105504462A
:103A4000286882B008B1112076BD00F087F801D156
:103A5000122076BD042001F0F3FE286078B3022026
:103A600001F055FA286804222146FAF728FE01F0F1
:103A700051FC28B10C2000F0C4FB05460D200DE0E0
:103A80006078022805D1122000F0BBFB0546132008
:103A900004E0102000F0B5FB0546112000F0B1FB5A
:103AA0000646DFF8AC04007800F0BDFC0346E07881
:103AB00000903246A0782946FFF7B6FF76BD132066
:103AC00076BD80B5DFF88414096809B9122002BDFB
:103AD0000978814201D0032002BDDFF87804007824
:103AE000012101F09DFF302000F0C8F9BDE802403F
:103AF000002035E238B5DFF8604405462078012122
:103B000000F0CDF800F02AF822D0257004F108006A
:103B100001F0EAFC6068C8B9207801001CD00501FA
:103B2000284601F08DFE606080B12A460021FAF738
:103B3000F8FD002005E06268C0B20301FF21D15406
:103B4000401C2278C1B29142F5D305E0132032BD6A
:103B50000020207001F0C8FC002032BDDFF8FC031B
:103B600000780A210842704770B5012442F20B0226
:103B7000801A09D0401E2FD18868007820B9DFF85C
:103B8000CC03006848BB23E088680578DFF8BC03F5
:103B9000006808B32900DFF8BC6310D14078022820
:103BA0000CBF0320022000F02CFB020003D0307871
:103BB000012101F003FF012000F0D2F905462800A1
:103BC0000BD03078012101F02BFF284600F056F988
:103BD000022001F0A1F900E00024204670BD80B56C
:103BE00028B9DFF86803006820B100207CE7BDE851
:103BF000024000E001BD2DE9F8430446E0780028CA
:103C00001CBF6568002D48D0242000F0FAFA4FFA56
:103C100080F80026DFF8349308E03861D9F8000016
:103C200000783946FAF7BBFD2935761CE178F0B209
:103C3000884232D295F928004045F5DB284600F04D
:103C40009EF800281CBFD9F800000028ECD0287A84
:103C5000143080B2FAF782FD0700E5D0D02038702A
:103C6000062200207870A91C0D20B8702878F87002
:103C700095F82800F87268783871781DFAF71FFDFA
:103C8000287A38730028C8D007F11400386105F18C
:103C900009013A7BFAF713FDC0E7BDE8F183F8B5F7
:103CA000AD4E044670680D4680B3002717E000EB68
:103CB0000710806830B101F0D0FD716801EB071189
:103CC00000208860706800EB0710C06830B101F018
:103CD000C4FD716801EB07110020C8607F1CA7427A
:103CE0007068E4DB25B101F0B8FD00207060F1BD23
:103CF00060B122010021FAF714FD0027FF2003E044
:103D000071683A017F1C8854A742F9DBF1BD10B5F8
:103D10009148416869B1002200E0521C0478D3B296
:103D2000A34206D2D2B21301CC5CFF2CF5D1C81845
:103D300010BD002010BD2DE9F041874E044670688B
:103D40008846C8B1002701E07F1CFFB23078874267
:103D500012DA70683D01415DFF29F5D040194178C4
:103D6000A142F1D106224146801CFAF7CCFC002882
:103D7000EAD07068401900E00020BDE8F08170B51D
:103D8000724E3168044682B000250020D9B12178F6
:103D900001290BD0227A04F109036946012001F0C0
:103DA0008CF800B105782178042912D0316849785F
:103DB000032918BF55EA01020BD020B1012904D113
:103DC00015F0030005D1002076BD0229FBD1E807DC
:103DD000F9D56078A11CFFF7AEFF0500207826D04A
:103DE000042814BFA868E86880B3227A0178914259
:103DF0000CD104F10901401CFAF785FC012805D11A
:103E0000232000F0FEF9002836D0DCE720780428D3
:103E100006D0A868D0B101F020FD0020A86015E010
:103E2000E86898B101F019FD0020E8600EE0042870
:103E3000C9D0FFF76CFF0500C5D020782870062296
:103E400060786870A11CA81CFAF739FC207A401C25
:103E500080B201F0F5FC60B12178042914BFA8609C
:103E6000E860217A00F8011B04F10901227AFAF7CF
:103E700026FC207A0028A6D0012076BD2DE9F84343
:103E8000DFF8C8800546D8F80000002600281EBFCD
:103E9000DFF8C490D9F80400002855D05DB9002798
:103EA00005E03901415CFF2918BF761C7F1C99F899
:103EB00000108F42F5DBF6B2F000083080B2FAF75E
:103EC0004DFC040005D10820FAF748FC0446002602
:103ED00013256CB3D020207065700120A070E670AF
:103EE00030001DD004F108056560002799F8000036
:103EF000874217DAF0B2A8B1D9F8041038010A5C89
:103F0000FF2A0AD008442A70062241786970761E7A
:103F1000811CA81CFAF7D3FB08357F1CFFB2E5E72C
:103F2000002060602146D8F800000078FAF737FCDE
:103F300099F800000021FFF7B2FED8F8000001F068
:103F40008CFC0020C8F80000BDE8F183C0470020C9
:103F500076450020EC450020D44500207545002022
:103F600010B50446232000F04CF901002046BDE8BE
:103F7000104018BF0121C9B2FFF75ABDDFF800F0A9
:103F80005D990010DFF800F09D9900102DE9F04FC9
:103F900005466F480078000789B058BF122068D5E1
:103FA00000F07CFF08B1102063E001F0B3F969492B
:103FB0000978884228BF15205BD2674C206808B179
:103FC000112056E00A2001F03BFC002820604ED072
:103FD000042000F09CFF20680A222946FAF76FFBB4
:103FE0002068407828B10E2000F00BF980460F20A1
:103FF00004E00C2000F005F980460D2000F001F9E6
:1040000081461C2000F0FDF8ADF820001B2000F0D8
:10401000F8F80746192000F0F4F805461A2000F0D9
:10402000F0F80646162000F0ECF88246152000F065
:10403000E8F883464948007800F0F5F9BDF82020FB
:10404000216807920697059504960190CDF80CA07B
:10405000081DCDF808B00090CB788A7849464046D4
:10406000FFF78CFF040003D000F000FE00E01324F3
:10407000204609B0BDE8F08F3548007800074CBFF6
:104080003748002000F0F5BE10B50124C01E19D03D
:1040900042F20A02801A0DD0401E08D0401F0DD0F7
:1040A000801F17D04DF6E672801A0FD018E000F08E
:1040B000DDFD16E0887800F02FF812E0887800F037
:1040C00051F80EE0084600F056F80AE0084600F005
:1040D0005CF806E08878010003D005F057FA00E0AC
:1040E0000024204610BD10B502461B4B12204FF68F
:1040F000FE741B68A14205D16BB11878904206D0BE
:10410000032010BD4FF6FF72914204D11BB1BDE8F0
:104110001040FFF737BF10BD010000D170470E49B6
:1041200000B5096887B081B100220592049203921C
:104130000292019200920B1DCA78097800F09AFC55
:1041400007B05DF804EB00F091BD07B000BD0000C2
:1041500075450020204800204C4500207645002071
:10416000E4450020010000D1704780B50021009196
:104170000023002206E080B5418900910389C288AE
:104180008188C07800F0B8FC01BD1FB50446607995
:1041900012281FD1E389A28961892089FBF746F89B
:1041A00018B1252000F02DF800B10120ADF80C0069
:1041B00003AA21796088FAF717FEBDF80C0048B908
:1041C00002900190E0890090A3896289218960882A
:1041D000FBF72FF91FBD0000DFF800F04998001031
:1041E000DFF800F0C9560010282808DA4FF6FF72F1
:1041F000914204D0CA4A22F81010002070470220D1
:104200007047282803DAC64931F8100070474FF686
:10421000FF70704770B504460D46C24E1C22002147
:104220003046FAF77EFA34777577F9F785FC0100A6
:104230000EBF012100211220317070BD10B5B94CA4
:10424000E160A06010220021FAF737FD012801D1BA
:10425000A0680CE010BD10B5B24C606010220021C7
:10426000FAF72BFD012801D1606800E010BDBDE820
:104270001040102105F019BBAA48406870472DE98D
:10428000FC41A84D0446002695F81E80042C0F46DC
:1042900024DA2878032818BF102054D101F03AF806
:1042A00028B900F0F9FD10B900F0F8FD08B11220AE
:1042B00049E0012C18BF022C1DD1BFB106220021FC
:1042C0006846FAF72EFA00F040F838B90622FF21C6
:1042D0006846FAF726FA00F038F808B1022032E012
:1042E000062239466846FAF7EAF90BE006216846E5
:1042F00005F0DBFA06E0032C04D16868694605F096
:10430000CDF90646884FAC770421387801F088FB58
:10431000002028849EB9ACB1684600F05BF80646E0
:1043200068B9032C0ED11D20FFF76BFF288448B11C
:1043300038784EF66022042101F058FB02E00EB1FD
:1043400085F81E803046BDE8F6810622694638466B
:10435000FAF7D9B970B5044600252000714E05D191
:1043600021B1062206F11000FAF7A9F930780128E8
:104370000CD10125200004D102203070FAF7DAFFB9
:1043800004E000203070204600F0A8F8284670BDF8
:1043900038B50024E0B10578624A290006D1417899
:1043A000837801EB0321D182C0781076107802283F
:1043B0000ED10124280006D103201070117ED08A6E
:1043C000FAF743FD01E000201070284600F086F85F
:1043D000204632BD10B5534CA17F81B10146062263
:1043E00004F12400FAF76BF9A07F04F1240100F036
:1043F00008F804F12400BDE81040FFF7EDBE0020EE
:1044000010BD79B102000DD04A79012808BF42F0F1
:10441000C00006D002F03F0203284A7102D142F0E8
:10442000400048717047010018BF012108467047DD
:1044300070B53C4D0446287FFF2815D00A20FAF7B6
:104440008DF9060010D0D020307074700820B07044
:104450000622A87FF07005F12401301DFAF72FF92C
:10446000287F3146FAF79BF9E87F01280FD12F48C2
:10447000006818B18068010018BF8047BDE870402F
:10448000294800784EF66022042101F0AFBA70BDD1
:104490002448806870472348C068006870472148F6
:1044A000C1680A68521C0A60007FFF281CBF4FF4D5
:1044B0008041FAF74ABA70471A48807F704738B58A
:1044C0000446184D05F11000FFF78AFE05F11000B3
:1044D0001CB9A97F09B105F1240032BD70B5114D99
:1044E0000446287FFF2819D00E20FAF737F9060076
:1044F00014D0D020307074700020B070062205F106
:104500001001F01CFAF7DBF8E88A70813146287E4A
:104510003073287FBDE87040FAF741B970BD0000E4
:104520008445002058450020EC450020F04500203F
:10453000DFF800F0259500102DE9F041044688468B
:10454000122740464FF6FE7188421646DFF82C5976
:1045500008D1A86950B30268100027D04146204610
:10456000904720E04FF6FF71884212D1A86938B118
:104570000268100004D0414620469047070005D04D
:104580003146204600F0DAFA07000FD12C706E7029
:104590000CE001F078F848B10078A04205D131462E
:1045A0004046FFF7C5FF074600E003273846BDE851
:1045B000F08110B5044684B000F072F808B902200A
:1045C00029E02088012101F08CF808B9142022E0AC
:1045D000208801F097F8042812D1DFF8A00881891B
:1045E0004FF6FF72914218BF112014D121888181AA
:1045F00061888180A188C180E18801812189418110
:1046000000200290019020890090E388A2886188B0
:104610002088FAF70EFF04B010BD30B5044685B00F
:104620002088402101F05DF8002836D02088ADF8C0
:10463000040000F035F8002500281CBFA07A0028EF
:1046400007D10021684600F0CEF9A07AF0B102252A
:104650001CE091208DF800008DF803503E208DF86D
:104660000100012106208DF80200A088ADF80800A5
:104670006088ADF80600E088ADF80A002089ADF842
:104680000C008DF80350684600F0ADF92088002238
:10469000402100F0C4FF284600E0122005B030BDE4
:1046A0002389E288A1886088FAF7C0BD70B50C46FE
:1046B000DFF8CC170978022918BF0129154601D166
:1046C000122070BD0DB9022070BD00F0DCFF0600A5
:1046D00001D1142070BD1CB1307940F0020030715E
:1046E0001022294606F11800F9F7E9FF2869B0629F
:1046F000002070BDF8B506000C4601D10220F2BDC5
:10470000308800F0C0FF050001D11420F2BDDFF8B1
:1047100070070078022818BF012803D0A87C082859
:1047200002D10CB11220F2BDDFF85077786908B1E0
:104730001120F2BDB02001F083F8786108B9132090
:10474000F2BDB02200F0C2FA786931884180A0221F
:10475000311D001DF9F7B3FF796902200870A87CAC
:104760007969328808280CBF012000200B1DDFF872
:104770001417097804F0A0FB06461CB12146284610
:1047800004F06FFD300018BF00F055FA3046F2BD5E
:1047900038B504460D4600F076FF08B9142032BD46
:1047A0008DF800506946204604F08EFC32BD38B5C5
:1047B0000022A0B101230624E4B2051915F8015C1A
:1047C000303D0A2D0BD203FB05220A256B43641EE4
:1047D000E5B2002DF0D11046BDE8344001E00220E2
:1047E00032BD30B505460C4685B0204600F04BFF83
:1047F00008B9122019E0DFF89006854228BF022090
:1048000013D2102200216846F9F78BFF280A8DF891
:1048100001008DF80050280C8DF802002146280E6A
:104820008DF80300684604F08EFB05B030BDF8B586
:104830000546DFF84C060078022818BF01280C4610
:104840001F4601D11220F2BD0FB90220F2BD284649
:1048500000F019FF060001D11420F2BDF06A08B182
:1048600000F0FBFF1C213846F9F73FFF0100F16221
:1048700001D11320F2BDB07C08280AD1069840B1BE
:10488000887E009001F112030A8A284604F014FD84
:1048900000E00020317941F004010CB141F0020147
:1048A0003171F2BD2DE9F0410D4600F0ECFE04003F
:1048B0001FD0A56200F007FA0546C0B200B92578FE
:1048C000A66A94F805801020F9F748FF070010D079
:1048D000D0203870062200207870A11D0920B87001
:1048E00087F80380381DF9F7EAFEFE603946E8B222
:1048F0001EE0BDE8F0812DE9F04104460D469046EA
:104900001F460E20F9F72AFF06000FD0D020307086
:1049100006220020707041460C20B070B580B01D9A
:10492000F9F7CDFE37733146204601E0BDE8F0814E
:10493000BDE8F041F9F733BFF0B50C0087B050D0B7
:10494000A079DFF83865002830690CBF08250425F8
:1049500008B9DFF838050778042D08D1DFF83005ED
:10496000006820B1416808001CBF00208847207DF6
:10497000059004F10803608A04903946208A039068
:10498000E08902900195A0880090E279E07800F03B
:1049900071F8E07880B9172004900122E089039033
:1049A00002950020019004F108000090E379A188AD
:1049B000384600F0E7FDE070306908B100F056F9C4
:1049C000307801000DD0717800F0B8F848B1E37884
:1049D000312B04D0A2883178184600F079F80020F5
:1049E000307007B0F0BD10B5044684B0A08851B156
:1049F000002102910191A189009163892289E188B6
:104A0000FAF7AFFC1FBD04B0BDE810403B21FAF738
:104A1000C1BC70B504460026A08800F034FE18B171
:104A20000678A08800F0E1FDDFF8505428780100F6
:104A300007D0864205D1697800F080F848B100209F
:104A40002870300005D0A379A288A078314600F004
:104A50003FF8686908B100F0EEF8A08800F052FE57
:104A6000042802BFA088A989884204BF4FF6FF70BE
:104A7000A88170BD2DE9F0410646884617461C46C0
:104A80001620F9F76BFE050020D0D02028706E703C
:104A90000520A870EF702CB106222146281DF9F7D9
:104AA0000EFE04E006220021281DF9F73AFE0698C2
:104AB00068812946079828730898E8810998288210
:104AC0000A9868820B982875404631E7BDE8F08166
:104AD000F8B504460D4616461F460820F9F73EFE77
:104AE00048B1D021017044700621817086808771A1
:104AF00001462846EDE0F1BD2DE9F04105460E46A0
:104B0000174698460C20F9F729FE040014D03046C9
:104B100000F0B9FD08B9DFF874030078D0212170E6
:104B200065700721A170E570A680E780A4F8088071
:104B3000069961812146FBE6BDE8F08110B50C467F
:104B400000F0B6FD28B140882146BDE81040FFF7CF
:104B5000EFBC122010BD2DE9F84F0746894692465A
:104B60001C46484600F08FFD5FEA000B1EBFDFF8D1
:104B70000C53696900295CD051F8A42F182002B1A8
:104B800034208A6802B1143004B11C30496801B184
:104B9000173080B2F9F7E2FD06004AD0182200F083
:104BA00095F800F090F85FEA000808BF9BF80080D5
:104BB000D020307077700A20B070A6F8049086F884
:104BC00006A006F118076969D1F8A40040B1B760E2
:104BD0003846D1F8A41000F11C071C22F9F76FFD2C
:104BE0006969D1F8AC0040B1F7603846D1F8AC1033
:104BF00000F114071422F9F762FD3CB13761384621
:104C000000F11C071C222146F9F759FD6869D0F80C
:104C1000A81031B177611722D0F8A8103846F9F7FB
:104C20004EFD31465FFA88F0F9F7B9FDBDE8F14F66
:104C300001E0BDE8F18F10B5904C6069A8B1D0F8E3
:104C4000A40008B100F009FE6069D0F8A80008B11E
:104C500000F003FE6069D0F8AC0008B100F0FDFD83
:104C6000606900F0FAFD0020606110BD10B5834C52
:104C7000206940B100F0F1FD002020610420BDE872
:104C8000104000F049B910BDF8B504460D4628465D
:104C900000F0F9FC060015D000F015F8070008BF79
:104CA00037780620F9F75AFD06000BD0062200F0EF
:104CB0000DF8D020307074700E20B070B580314681
:104CC000F8B206E0F1BD2620FFF79BBA0021F9F704
:104CD00028BDBDE8F440F9F762BD2DE9F84304466C
:104CE0008846914600F0CFFC070024D01420F9F745
:104CF00035FD05001FD0FFF7E6FF060008BF3E7830
:104D0000D0202870062200206870B91D0B20A870E2
:104D1000E81CF9F7D4FC6C8118F00101C5F810907B
:104D200018BF01212973F0B218F0020118BF012148
:104D30006973294601E0BDE8F183BDE8F443F9F762
:104D40002EBD2DE9F14F90460D469946404600F0A4
:104D50009AFC07000A9EDDF82CA0DDF830B00D9C0F
:104D60003ED09DF8000000283AD1387940F010007C
:104D70005FEA49714CBF40F0020000F0FD00002ED8
:104D800008BFBAF1000F08D1BBF1000F08BF002C1B
:104D900003D100F0FB00387122E040F004003871CC
:104DA0003CB12069B8621022214607F11800F9F7DA
:104DB00086FC3EB135B9F86A08B100F04EFD1C2101
:104DC00030460AE0BAF1000F0AD0012D08D1F86A86
:104DD00008B100F042FD1C215046F9F786FCF8624C
:104DE000264D6869002842D086B1D0F8A40028B9C1
:104DF0001C2000F025FD6969C1F8A4006869D0F89D
:104E0000A40018B11C223146F9F759FCBBF1000F80
:104E100011D06869D0F8A80028B9172000F010FD5B
:104E20006969C1F8A8006869D0F8A80018B117220C
:104E30005946F9F744FC8CB16869D0F8AC0028B940
:104E4000142000F0FDFC6969C1F8AC006869D0F875
:104E5000AC0018B114222146F9F731FC9DF800008E
:104E600053464A46414601B0BDE8F04F73E6BDE8FF
:104E7000F18F024988617047000000003C45002026
:104E800075450020EC45002040420F00744500208D
:104E9000F045002004F01EBC264800E026480068CB
:104EA00000B101207047010001D0172801DBFF2865
:104EB00001D101207047002070472DE9F04D0D46CB
:104EC00093460024BBF1200F80461F462C7003DB65
:104ED0000020BDE8F08D0419E0B25845F8D2E4B2E4
:104EE0003E5D641C002EF3D0E4B231198B45EFDB3C
:104EF00017F804A05046FFF7D6FF641C0028E7D03F
:104F0000701EC2452870E6D1E4B23819E1E70B49BA
:104F10000A7810430870704708490A7832EA00009E
:104F2000087006D10648006818B14068010018BF33
:104F300000477047C4470020C0470020D6480020E3
:104F4000BC470020F8B5144600250E46B24FB34BBF
:104F500030B1012811D0062814D0072818D022E03B
:104F600016291EDA16220021381DF9F7DAFB32461F
:104F70002146381DF9F7A3FB16E0022E11D1208837
:104F8000388011E0012E0CD1DA6903F1280104E028
:104F9000012E06D1DA6B03F14801207800F029F8E0
:104FA00002E0182500E002252846F2BD10B50B46A8
:104FB0000024994910B1012806D008E01522091DE6
:104FC0001846F9F77CFB03E00888188000E002240B
:104FD000204610BD01460020C90706D50FF2442324
:104FE0008E4810220521FDF76DBD70478C49086081
:104FF000704710B50B7884074CBF43F0020303F0F1
:10500000FD0304064CBF43F0800303F07F03040755
:105010004CBF43F0080303F0F70384064CBF43F092
:10502000200303F0DF030B70AA21084203D010789D
:1050300040F00C0003E018B9107800F0F300107095
:1050400010BD2DE9F0410F461546387802281E465E
:105050004FF000085ED1786801784078069C01EB3B
:10506000002080B221001CBFB0F5285F0B2056D174
:105070004FF42851401A08D0401E1AD0401E28D0A4
:10508000401E1ED0401E2AD044E0F868F9F715FBF8
:10509000079A80B2031B9342B8BF021B92B2101949
:1050A000162803DA3280F86801190EE04FF00D0877
:1050B00034E0F8680088022131802870000A6870A6
:1050C0002CE0062030800622F9682846F9F7F7FA26
:1050D00024E001203080F868007828701EE0F8682D
:1050E000B0B108213180018829700188090A6970EE
:1050F0004188A9704188090AE970818829718188ED
:10510000090A6971C188A971C088000AE87105E0BF
:10511000308003E0A6F800804FF001084046BDE86B
:10512000F0812DE9FC4B0E4680463078002702289E
:1051300091461D466BD17068017840780A9CDFF873
:10514000E0B001EB002080B24FF42851401A06D0A5
:10515000401E29D0401E4CD0401E38D057E0F06889
:10516000F9F7ABFA80B2A04204D32919162903DB60
:105170000D274DE007274BE0F3682A4649461819EA
:10518000F9F79DFA2C19F068A4B2C4F116020021B7
:105190002044F9F7C6FADBF80000002838D002688E
:1051A000100035D0002121E07CBB022DE0D199F820
:1051B000000099F8011000EB0120F1680880DBF88D
:1051C000000028B30268100022D001210EE0E4B9EB
:1051D000062DCDD1F06806224946F9F770FADBF8C2
:1051E0000000A8B10268100012D003214046904789
:1051F0000EE054B9012DBBD199F80000010013BF96
:105200000128F1680870802702E00B2700E00127E1
:105210003846BDE8F68B0000044800201046002008
:10522000004800204350010023510100000000000D
:10523000B1494870704710B5AF4C207004F06AFD5A
:105240002078BDE810400521F9F766BD7CB5AA4D70
:1052500028780C46210419D5F9F7FFFA060084F4E2
:10526000004411D000F058F858B93078A22806BF91
:10527000A24800786878FF2803D03146F9F78FFA02
:1052800002E03046F9F77CFA204676BDE10709D501
:10529000A86820B1416808001CBF0020884784F03E
:1052A000010076BDA10709D5686820B141680800F2
:1052B0001CBF0120884784F0020076BD610727D516
:1052C0008F4E31880A001DD0481E308080B2E0B970
:1052D000FFF7E2FD48B18B4901200870686820B1F2
:1052E000416808001CBF01208847FEF7C5FF6946DA
:1052F00004F0D4F96846FFF76DF81D20FEF781FF32
:10530000308002E0042100F08BFB84F0040076BDC5
:10531000002076BD00F0FCB938B502780124912A4E
:105320004FF6FF7102D0A22A76D07BE04278052AA0
:1053300049D00E2A04D00F2A48D03E2A69D071E005
:1053400082886D4941F20905531B2DD040F6F9754D
:105350005B1B2FD0DB1E31D05B1E08D09B1E022BA7
:1053600005D9DB1E012B15D9DB1E08D05AE0496890
:10537000002958D009680A0055D0884750E0624992
:10538000096800294FD04B6819004CD0014642F201
:105390000E003CE08968002945D00B68190042D016
:1053A0000146104698473BE08068411C0078FEF7B4
:1053B000D1FF35E08068FEF7EBFF31E080680078D0
:1053C000FFF736F82FE0FFF724FB2CE0828842F24B
:1053D0000D05531B13D09B1F02D09B1F0FD021E044
:1053E0004A4B1B888B420AD049490968D9B10A68DF
:1053F000110018D0014642F21300904710E04249D4
:10540000096881B14B6819000DD0014610469847D4
:1054100006E000F00AF803E00246408800F04BF88E
:10542000044600E00024204632BD70B50546012444
:10543000A8780128014611D0022806D0032811D0EF
:10544000062815D00A2809D032E02B48806880B39E
:10545000416808002DD0284688472AE02946FFF7F2
:105460006BFA26E0A8882A4600F025F8044620E0DA
:105470000E20F9F773F906001BD0A88801224021FD
:1054800000F0CDF8D02030703146E87870701120EF
:10549000B070A888B080E888F08028893081688959
:1054A0007081A889B08115480078F9F778F900E093
:1054B0000024204670BD70B50C46154600F022F958
:1054C0000126042804D11248006858B1026803E09C
:1054D0000D48006830B14268100003D029462046CC
:1054E00090470646304670BD0349886070470949B9
:1054F0000860704700000000EC4500207445002063
:10550000784500207745002054450020484500207C
:10551000B8470020BC47002038B5AE4C002200211F
:10552000204601F0EFFC20783025684300F088F930
:105530006060B8B100210AE005FB01F202444FF6B9
:10554000FF735380491C00231371D362C9B22278C0
:105550009142F1DB0020002104EB8002401C0C286A
:105560009160F9DB31BD00219A4A02EB8102936818
:1055700013B9906000207047491CC9B20C29F3DBB5
:10558000132070472DE9F04106460C461746984611
:10559000204600F078F808B1112024E04FF6FF70A3
:1055A00000F071F805001DD085F8058006220699E7
:1055B000A81DF9F784F80622002105F10C00F9F77F
:1055C000B0F86C802F712E700020E86200210898DE
:1055D000A8740998A8820A98E882204600F0E9F8A1
:1055E000002000E01520BDE8F08110B500F04BF878
:1055F000040012D06088012100F0DBF8E06A08B1F5
:1056000000F02BF9302200212046F9F78AF84FF6F6
:10561000FF7060800020207110BD022010BD38B5E1
:105620000C46154600F02FF858B10179002D14BF33
:105630002143A14301710221408800F0BAF8002003
:1056400032BD152032BD38B50C4600F01CF80500FF
:1056500017D028792070062268796070A91DA01CD7
:10566000F9F72DF8062205F10C0104F10800F9F70D
:1056700026F8A87CA073A88A2082E88A608200208D
:1056800032BD012032BD10B50022524B00E0521C49
:105690001C78D1B2A14209D25968D2B23024544305
:1056A00021444C888442F2D1084610BD002010BD30
:1056B000F0B5484B5C6800224FF6FF7700E0521CC3
:1056C00019788A420BDA302101FB02F561194E8804
:1056D000BE42F4D0655D8542F1D10846F0BD0020A0
:1056E000F0BD10B50C464FF6FE71884206D0FFF7AC
:1056F000CAFF00281CBF0079204201D0012010BD44
:10570000002010BD80B5FFF7BEFF00B1807C02BD58
:1057100010B5002000212F4A08E05368C9B2302498
:105720004C4323441B7903B1401C491C1478CBB271
:10573000A342F2D3C0B210BD26480078704710B51E
:105740000C46FFF7A0FF00281CBFC18AA14202D06F
:10575000C482002010BD012010BD80B5FFF793FF6B
:1057600000B1C08A02BD70B505460C461646FFF76B
:105770008AFF28B94FF6FE70854218D0142070BDFC
:105780000179C06A28B9CA0609D5C90609D40F200B
:1057900070BD01F01202102AF7D1002EF5D00520BD
:1057A00070BD20B1807EA04201D20C2070BD0020CF
:1057B00070BD70B504460D460026064800EB860015
:1057C0008268100002D0294620469047761C0C2E95
:1057D000F3DB70BD2048002002000A4A08BF0FF228
:1057E00021005060517070477047064A010004BFA5
:1057F0005178012902D01178526810477047000093
:10580000704700009444002000F10103810704D098
:1058100010F8011B89B18107FAD10268B2F1013198
:10582000914311F0803F04BF50F8042FF6E710F8C1
:10583000011B11B110F8011BFBE7C01A70470000F3
:10584000E0B50821ADF800100190042100F00FF838
:1058500008B100200EBD02980EBD00B583B008212E
:10586000ADF800100190052100F001F807BDADF87A
:105870000210684601490968084700008047002077
:1058800062F30F2262F31F42401810F0030308D0A6
:10589000C91A1FD3DB0748BF00F8012D28BF20F825
:1058A000022D130030B414461546103928BF20E9E4
:1058B0003C00FAD8490728BF20E90C0048BF40F84F
:1058C000042D890028BF20F8022D48BF00F8012DC3
:1058D00030BC7047C91818BF00F8012DCB0728BF8E
:1058E00000F8012D7047000000B583B00820ADF826
:1058F000000012209C490968ADF8020068468847FC
:1059000001980EBD10B5994C0020A060FFF7ECFF88
:10591000606010BD70B504460D46164600F018F8DC
:1059200008B1466070BD1020FFF78AFF78B184721D
:105930000581466000210160C1608C490A6812B986
:10594000086070BD0A4611680029FBD1106070BD67
:10595000864A12682AB113898B4204BF937A834224
:10596000F7D11046704708B10021018170472DE939
:10597000F041FFF7B9FF7D4E7D4977680C68C51B84
:10598000B4F57A7F14D0A4FB05014FF47A7200239A
:1059900004F0CEF94FF47A78A8FB0023054608FB03
:1059A0000133104619462246002304F0C1F9C019FC
:1059B00070602846BDE8F04104F032BAF8B50446FC
:1059C0006A4800680D46164608B9FFF7D0FF6948D7
:1059D0000068804700F01FF800F048F80446384699
:1059E00088470CB10020F2BD0820F2BDF8B504468E
:1059F000604800680D461646804700F00CF8040029
:105A00005D4918BFE6600968384688470CB1002038
:105A1000F2BD0820F2BD074632462946204679E706
:105A200070B500F026F8064629462046FFF790FF9D
:105A3000040018BFFFF797FF00F018F830468847BA
:105A40000CB1002070BD062070BDF8B500F011F853
:105A5000074629462046FFF77BFF002600B146682F
:105A600000F004F8384688473046F2BD42490968DC
:105A7000704704463F4800680D4600472DE9F1474E
:105A8000DFF8F080394DD8F80000DFF8ECA081B0E5
:105A900080470246A86801990818A8601046DAF8FD
:105AA000001088472E68002E4DD00027D8F800003F
:105AB00080478146BDF806000024002804BF9DF8F9
:105AC0000500002807D130799DF80420904202D3C8
:105AD000801A307106E07068019981423ABF401A1D
:105AE00070607460B08858B9F08858B9F06868B1CF
:105AF000318908000AD0B07AF8F727FFF0687060A3
:105B0000B08808B9F08808B1308930B93068002F02
:105B10000CBF28603860344600E037463668DAF853
:105B200000104846884764B1A088002804BFE08878
:105B3000002803D12189A07AF8F707FF2046FFF754
:105B40008CFE002EB2D1BDE8F3870848016841B150
:105B50000A484A680968824298BF10460029F8D16D
:105B6000704700207047000080470020A4470020B5
:105B7000AC44002084470020884700208EC2F528CE
:105B800000B583B00821ADF800108DF8040017218E
:105B9000ADF8021068461D49096888479DF8050060
:105BA0000EBD1B48002181800121017070472DE945
:105BB000F0410D461749097801248842064602D271
:105BC000134F387808B901201DE01348006880475A
:105BD0008046B88804FA06F64DB920EA0601B98075
:105BE00060B159B90020FFF7CBFF044606E010B9B9
:105BF0000120FFF7C5FFB8883043B8804046074909
:105C0000096888472046BDE8F081000080470020F1
:105C10009C470020A8DA0000844700208847002025
:105C200030B585B0144608220291ADF8002000225C
:105C30003A490968ADF80400ADF802201D466846EF
:105C400088479DF80C1021700499296005B030BD7B
:105C50001CB51420FFF7F4FD31490860142200211F
:105C6000F8F75FFD002000F0DBFE012004F02AF8C9
:105C7000022002F043FD032004F002F90420FFF7A4
:105C8000DAFA052004F052FA0620FAF738FE072067
:105C9000FCF7D2FE0820FAF71CFA0920F7F7BCFF40
:105CA00001AB6A4600211020FFF7BAFF9DF80010F3
:105CB0000920F8F742FD00249DF800102046F8F76F
:105CC00044FD641C092CF7DB13BD10B582B004F051
:105CD000A1FA144B144A15495020FFF7A1FF60B1F7
:105CE0000520FFF782FD0820ADF800000C200B49CD
:105CF0000968ADF80200684688470D48006880478B
:105D00000446FAF79FFDF8F788FE0A49096820461D
:105D10008847F8F7B8FE002016BD00008047002035
:105D200098470020A8440020D548002043EB0000FD
:105D30008447002088470020F8B505460C46AF8907
:105D40002FB3AA68167830060FD50D2F1FDB0C3F36
:105D5000BFB2D01900903B466888012103F042FE93
:105D6000002814BF0220012000E000202070B009AC
:105D700000F00100607006F03F00A070781EA08067
:105D800080B208B1A868401CA0600020F2BD0120CC
:105D9000F2BD0A7802704A8842704A88120A8270FC
:105DA000097918E104290AD10178117083784178C2
:105DB00001EB03215180C07810710020704704204E
:105DC000704705E0022B00D1D5E00420704700BFEA
:105DD0000A8802700988090A417002207047022966
:105DE00006D10178407801EB002010800020704738
:105DF00004207047E6E0042B00D1F4E00420704753
:105E00008A7802708878098801280CBF0420122043
:105E10004843401C80B2704710B50B001CD003787B
:105E2000491E012B89B207D14B0801EB93739B08E4
:105E3000B1EB830410D108E0022B0DD1122391FBAA
:105E4000F3F3122404FB131131B999B221B110F804
:105E5000011B917013800FE1042010BD10B50C469A
:105E6000022200F047F8001D611DF8F728FC208988
:105E7000801D80B210BD70B51E46062E144619DB7B
:105E8000049D2078617800EB012028800222A07810
:105E9000E17800EB01206880211D02202871681D37
:105EA000F8F70DFCB01F288180B200B1A01DE8609A
:105EB000002070BD042070BD08888004000C70476D
:105EC0004B0801EB93739B08B1EB830303D1890863
:105ED00001D011809AE00420704710B50C4600F004
:105EE00009F8611D2279001DF8F7E9FB2079001DF2
:105EF00080B210BD218801702188090A4170618833
:105F000081706188090AC170704710B5029C062B28
:105F1000104612D1022121714278017801EB022151
:105F20002180C278817801EB02216180011D2279F4
:105F3000601DF8F7C4FB002010BD142B08BF102112
:105F4000E9D0042010BD7CE010B50B000BD0037825
:105F50005380491E022B89B205DB91FBF3F403FB4E
:105F6000141101B986E0042010BD31E7022B00D1E5
:105F700001E0042070471078517800EB012000996F
:105F8000088000207047088870473CE010B5022B5D
:105F90000FDB029C207261721078517800EB0120B7
:105FA0002080981E608080B200B1901C606000204C
:105FB00010BD042010BDB2E009B9002070470420D4
:105FC000704700BF0A8802700A88120A42704A8825
:105FD00082704988090AC17004207047042B00D1DF
:105FE00001E00420704700981178537801EB0321F9
:105FF00001809178D27801EB022141800020704726
:106000000888704700BF118001B90020506000204F
:10601000704788884004000C704703EBD370400839
:10602000B3EB400007D15908022904DB00988180B6
:106030000260002070470420704708887047E2E73C
:1060400000BF4A8809880270514389B2481C80B257
:10605000704710B50B000BD003785380491E042BFA
:1060600089B205DB91FBF3F403FB141101B901E0E4
:10607000042010BD1480401C5060002010BD14E0AE
:1060800010B5042B0EDB00F062F8D478917801EBA8
:1060900004214180191F818089B201B1111D8160E5
:1060A000002010BD042010BD00BF0A8802700A88BD
:1060B000120A42704A8882704A88120AC27088881E
:1060C000001D80B2704710B5042913DB03784478B3
:1060D000091F03EB04231380C4788378918003EBBA
:1060E000042389B2002914BF001D00209060538052
:1060F000002010BD042010BD0978017001207047F8
:10610000012B04D1009910780870002070470420FA
:10611000704709B9002070470420704700BF0A8803
:1061200002700A88120A42704888801C80B2704748
:1061300010B5022B09DB00F00AF8991E418089B2E4
:1061400001B1911C4160002010BD042010BD0298D7
:106150001178547801EB0421018070472DE9F04754
:1061600084B080460C9D0C4691469A4655B917203E
:10617000FBF704F80126050005D11324204604B0DE
:10618000BDE8F08700262846012700F8019B14B1DE
:106190005146A047471C5FEA09600DD510214046D3
:1061A000FFF79FFAD8B9BFB2EA193946284603F07B
:1061B000CCFB044668B90C370420ADF8000001950B
:1061C000ADF8087069464046F8F7BBFD0028044664
:1061D000D4D0002ED2D02846FAF7F5FFCEE7192406
:1061E000F7E730B5022918BF102985B004461546D7
:1061F00003D1022B18BF102B01D0002017E00A4654
:106200009A4203D12946F8F77EFA10E01029694630
:1062100006D1284600F00DF810226946204604E019
:1062200000F007F8102269462846F8F76CFA05B026
:1062300030BD38B504000D4618BF002D0BD010221C
:106240000FF260012846F8F73AFA20782873607850
:106250006873012032BD002032BD38B504464FF6C8
:10626000FE7084420D460BD0172D09DBF8F7F3FDC5
:106270002946884204D32046BDE83440FFF75FBA80
:10628000012032BD80B54FF6FE71884205D0FFF780
:1062900064FA010005D1172002BDBDE80140F8F7FE
:1062A000DABD02BDFB349B5F80000080001000005F
:1062B00000000000DFF800F03DAC0010DFF800F057
:1062C00089D10010DFF800F0C9B40010DFF800F049
:1062D00019570010DFF800F061840010DFF800F0BB
:1062E0008D670010DFF800F041B50010DFF800F016
:1062F00055B50010DFF800F0BD800010DFF800F0A9
:106300001DB50010DFF800F02D8A0010DFF800F056
:1063100071940010DFF800F0FD750010DFF800F058
:1063200035A30010DFF800F0E1AC0010DFF800F05A
:10633000EDAB0010DFF800F065860010DFF800F02C
:1063400029840010DFF800F0B9860010DFF800F0B3
:1063500095D60010DFF800F00DB50010DFF800F062
:10636000B5770010DFF800F0F182001080B54FF42F
:106370009E720FF23001DFF8380C02F059F9DFF8A5
:10638000340C002101700122DFF82C1C0A73022258
:106390000A70DFF8281CC0F80D10DFF8B01DC0F837
:1063A0002D1001BD99040021190500217904002157
:1063B000F0B5174C40216118C878022805D009486B
:1063C0000021016008498847F0BD256E074E356001
:1063D000600728432066276824600E4880472760AE
:1063E0003560F0BD2C110440A56500002840044034
:1063F00010B5074CA17D002905D10121A1754802E6
:1064000004493E3988472068002800D0804710BDE5
:10641000540200218B39000010B50549054A72B6B7
:10642000C878012802DC01204870121D62B61047AE
:10643000940200216D470000F8B51A4E0546316BF5
:106440001948CC09E401002D11D018490978022916
:106450000FD0007B044372B60120154F4002B847AD
:10646000114820380088C109C90704D016E0C07A55
:10647000F0E7407BEEE70F493463CC61400AC00788
:106480000CD001208003F16A002D01D0014300E00F
:1064900081430846F1620749403948630020B84704
:1064A00062B6F8BD8002002188000021960200211A
:1064B000DF3C0000404004400749002800D0042091
:1064C000064A72B60978C90701D0105800E080204A
:1064D00062B640B2704700006B0200215860044071
:1064E0002DE9F0410FF24C00DFF86C1D2722036804
:1064F00044688568C6680769D0F814C0D0F818E009
:10650000D0F81C800B604C608D60CE600F61C1F8CC
:1065100014C0C1F818E0C1F81C8020302031521E90
:10652000E5D142688368006808604A608B60BDE816
:10653000F0810000546100007F1402000600050095
:106540000F0008004800520080FF3F0000000000DC
:10655000000000000000000000000000304000408B
:106560000140034007400F404F40CF40CF41CF4351
:10657000CF47CF4FCF3FCF2FCF1FCF0F000000000F
:106580000000000000000F00080000003F000000B5
:1065900040003F000000040068000E00DC00060020
:1065A00043001A0005000000000002000000000087
:1065B000000000000400C00000000400C000000053
:1065C00007000000000000000000000000000000C4
:1065D0000000000050C00091007070C00091007079
:1065E00082312100319110B10070018101B100A10F
:1065F0008231329110B101911110418141226340E9
:10660000F106007051C0019130181039833108D063
:106610001831416F3100319110B1831414166F6835
:106620000070251050C00091F4C340C12014036FC6
:10663000311041045082F0228440512622C0823120
:106640002100319110B163393110410482C082318F
:106650002100319110B163393110A2C08231210083
:10666000319110B15010153105140592007053642A
:1066700052C0311031066131C102566412C131106D
:10668000213971065131E1025664007051C0019107
:1066900001CCE2C05664536411C1C2C0566454B008
:1066A000007154A064B0F0800022B54011C122C135
:1066B000566451C00191E2C0823160820200329181
:1066C00010B100C3C86853644012B09032B000C328
:1066D000CE6840C2D0688012B09032B0007053646F
:1066E00001C122C1566401C1C2C0566453829D6477
:1066F000C012B09032B00070536472C281C0566450
:1067000022C111C1566402C011C1566462C031C3B6
:10671000566462C311C1566402C311C156645382E8
:1067200053399D64E2C35B641122F84042C281C8C0
:10673000566452C211C1566472C2E1CE566402C29E
:1067400081C8566402C201C85664B0C00C690070AA
:10675000536442C201C8566452C211C0566472C228
:10676000E1C0566402C001C1566462C001C35664F0
:1067700022C101C1566462C301C1566402C301C192
:10678000566453829D64007002C1623101C0A080D2
:10679000001E3241101A34612010101A136F236E3C
:1067A0001116121634690070E092D08200223B4527
:1067B000C0B20070000000000000000000000000F7
:1067C00000000000000000000000000000000000C9
:1067D00000000000000000000000000006730572C9
:1067E0000B720E7250B00071818060B050A0928028
:1067F000F0EFF19202933A65412278458080F1C131
:106800001004301601110114016C8B618C618D61D3
:106810008E618F61906191619361956197619961DA
:10682000706273629180F2C0210421318280422A19
:106830001214321601112114016CA661C761AC61FA
:106840007362A661C761AC6173629B619B619B616E
:106850009B619B619B61AC649B61D5649B61E264BD
:106860009B610E659B612A659B618280E0DFF292ED
:106870003A65B0B0A261B1B00673057230B058612C
:10688000D0CF3A6584C203C0C0C368649078509189
:10689000607810316178101400925078403161783E
:1068A00010004031717810001092B07860928178B9
:1068B00021923078403141781000309210C0F09130
:1068C0009B6154A0F0805022CF4540800022664654
:1068D000C76100C86091598150B0918041222E4615
:1068E000C0CF3A65128282318239423928107764EA
:1068F0001282F11212042F101F312F1440C12014E4
:106900000D6F6D39DE10F4C34E0482C082312E004B
:106910006D39A2C082312D001A828A3920828031DD
:1069200080390BC00B18AC7830824039021011C08E
:10693000013010C00118021882312100C126919146
:1069400003B013B063B053B0038239144180012205
:106950006646B481C491D5819518B51C1C4EC51CE2
:10696000544A6591F08010220C422C623D9110B186
:106970003E9110B165910F925981F914AB18BC107A
:10698000F0805022C74110222C460C62B0CF3A65ED
:1069900063B030820010F2C02004021011C0013038
:1069A00010C00118021882312100C12691919191E5
:1069B00013B003B063B053B064B054B00071418001
:1069C0000122664663B064B0F0805022C741B181B5
:1069D000C191D1819118619131B0446212828231AA
:1069E00082394239281077645981058259142082EE
:1069F0000BC00B18AC7880C0007163B0626A0C6287
:106A0000018262818231823DA0EFF19202933A6568
:106A100003A09B61A28077649B6150B000719B6171
:106A20002DE9F04FDFF8104ADFF8105A20700721E7
:106A30000020286283B0DFF8080A01700D21418030
:106A400040F222218180DFF8FC09DFF8FC1969623D
:106A50008A7E0270FF2ACB7E437008BFFF2B0E7F19
:106A600086704F7FC77091F81EC080F804C0C97F40
:106A7000417116D1FF2E08BFFF2F12D1BCF1FF0FBD
:106A800008BFFF290DD1DFF8341B0A7802704A785D
:106A900042708A788270CA78C2700A790271497924
:106AA0004171DFF81C1B0278DFF8188BDFF8187BC8
:106AB000DFF8186B0A70002342784A704FF0180A0A
:106AC00082788A70C278CA7002790A71002240798D
:106AD0004871FF21DFF8F80A017041708170C170C0
:106AE0000171417101202871DFF8E80A0271C28149
:106AF00003754FF42072012300F010F902824282E4
:106B00004375DFF8D40A00F009F98373002101719D
:106B1000C173818202820521428281750020DFF8E3
:106B2000BC1ADFF8BC3A0880D8F82C104878A87056
:106B300008783870801C8A782A700AFB00F08A680E
:106B40001279521E1A7080B2CA786A70CA682A61B5
:106B50008969DFF85C2BA9614FF496711180FEF70B
:106B60006FFEB06008B900F09DB83878010000F001
:106B70009C804FF49071484380B2FEF761FEDFF8CD
:106B8000449BC9F8040008B9B06889E038783C2112
:106B90004843FEF755FE686120B900F0BCF8D9F80B
:106BA00004007DE03878FEF74BFEE86128B900F07C
:106BB000B2F800F0ACF8686972E038780AFB00F0CF
:106BC000FEF73EFEDFF800ABCAF8000038B900F06F
:106BD000A2F800F09CF800F097F8E86960E03878D7
:106BE000DFF8E8BA4001FEF72BFECBF8000050B901
:106BF00000F091F800F08BF800F086F800F07DF8D6
:106C0000DAF800004CE038780001FEF719FEDFF8F2
:106C10003C1B086060B900F07EF800F078F800F0E6
:106C200073F800F06AF800F06BF8DBF8000037E06A
:106C300038780001FEF704FEDFF8141B086080B905
:106C400000F069F800F063F800F05EF800F055F825
:106C500000F056F8DBF80000FEF7FFFDDFF8EC0A65
:106C60001DE0387830214843FEF7EAFDDFF8E41AEA
:106C70000860D0B900F04FF800F049F800F044F88F
:106C800000F03BF800F03CF8DBF80000FEF7E5FD13
:106C9000DFF8B80A0068FEF7E0FDDFF8B40A006824
:106CA000FEF7DBFD4FF4804122E000F0D1FA074609
:106CB0000820ADF800001E20ADF802004FF400508F
:106CC000DFF8281B096801906846884703F0DCFA62
:106CD000D8F80C00697800880843DFF8C81C0880E1
:106CE000384600F0B1FA884700F0D4F94FF400516B
:106CF0002078F7F72AFEBDE8F78FE869FEF7ADBD0B
:106D0000DAF80000FEF7A9BD6869FEF7A6BDD9F85C
:106D10000400FEF7A2BDB068FEF79FBD017241728C
:106D20008172C17201734173704770B50C46E00700
:106D300088B00DD5FFF7BEFA38B100218160DFF8C9
:106D4000FC0A0068010018BF804784F0010071E070
:106D50002007DFF8E85627D5DFF87C08417D686911
:106D60003C224A431044DFF85C2952684FF4907388
:106D70005943114400220692CA8E120905928A8E46
:106D800004924A8E5208039200220292019200F16C
:106D900034020092002290F830308979002001F00E
:106DA00072FA84F0080045E0E00610D50020069055
:106DB000059004900390029001900090002300221F
:106DC0000021022001F05FFA84F0100032E0A005FB
:106DD00008D5DFF8900C016841F00041016084F4AF
:106DE000007027E0600504D5F9F764FD84F4806045
:106DF00020E0600405D5812001F07EFB84F4804012
:106E000018E0A00415D54FF0FF30286204F0FFF819
:106E10002E69366805F1380305F14C0205F12801A9
:106E200005F16800B047E86000F006F884F400500F
:106E300000E0002008B070BDF8B5DFF80046DFF8CC
:106E400084582369E068DFF88067183300221B68E4
:106E50004FF0FF319847DFF86C07DFF84C1BC06A32
:106E6000806840790870002704F0F8F8DFF83C0BE0
:106E7000FFF724FAFFF726FAFFF728FADFF8300BBE
:106E800000210170017141718171C1710172417202
:106E90000020DFF840178873DFF83C17C8730BE059
:106EA00068684FF49071794308444179012908BF1B
:106EB00003F0C8FC7F1CFFB230788742F0DBFFF79D
:106EC00009FAA078DFF8EC1A087004F0BDFB03F0B3
:106ED00023FBDFF8E41A00200870DFF88C1B087031
:106EE0000120DFF8881B08700020DFF8841B087081
:106EF000DFF8801B0870DFF8801B0880DFF87C1B40
:106F00000870F2BD2DE9F0411446DFF8BC5608B117
:106F10002A780270DFF8AC8711B198F80100087088
:106F2000002C3ED0002600271CE0C9B2DBB2605422
:106F300002F130000179E154591C427900F034F833
:106F4000827900F031F8C27900F02EF8027A00F070
:106F50002BF8427A00F028F80078C9B24E1C605431
:106F60007F1CFFB2287887421BDA3846FFF7B6F954
:106F70000028F5D1D8F804004FF490717943F6B2A7
:106F80000844DFF8B8144969A7553C220068007826
:106F90007A430A44711C4B1C80280CBF002001203E
:106FA000C3E70020BDE8F081C9B26254491C7047B4
:106FB00004040021A30300216C030021110400211B
:106FC00005460C46FFF78AB92DE9F8435FEA010947
:106FD000144618BF002C06461D4600D00DB91220DD
:106FE00056E0FFF77BF9010052D100F03BFF461855
:106FF00030680078802818BF0C2049D106F1E307DB
:10700000B87DC00758BF112042D5B87C012808BF01
:107010003A203DD000F01CF980460120B8740020D1
:1070200019F800103218401C082882F8AC10F7DB61
:1070300006F1B4002178017061784170002042426D
:10704000295C3244401C102882F8E210F7DB06F17C
:10705000A400FFF747F906F19800FFF747F900F0A1
:1070600019F8002086F866003870787096F892005B
:10707000012802D178730A2102E0002078730321ED
:107080003046FFF737F900F0DFF840468847002028
:10709000BDE8F2830C21DFF8100DFFF72FB910B512
:1070A0000446FFF71BF901001FD100F097FB0844CD
:1070B00000F1F8010A78022A06D1817900F1F9027B
:1070C000002000F0A1FF0FE002681278802A08BFBC
:1070D000082107D0402A07D14978090701D4112097
:1070E00010BD0E21FFF706F9002010BD10B50400F9
:1070F00001D1122010BDDFF8CC05407808B10C207A
:1071000010BD03F009FADFF8340D22784178114000
:1071100041706278817811408170002010BD38B5CF
:107120000C00054606D0DFF89C14C96A8968097905
:10713000884201D3122032BD03F0CCFFDFF868088B
:10714000057001202070002032BD00005104002194
:10715000DFF87024D26A92681279904201D312202B
:107160007047DFF87C1408700020704710B51400D9
:1071700019D011B1012908D015E003F0D3FF10F1A7
:10718000800F20700DD1302010BDDFF83804C06AA8
:1071900080680168007900EB4000084410F8030C97
:1071A0002070002010BD122010BD2DE9F8430C0006
:1071B00005469046994605D05FEA090018BFB9F127
:1071C000010F01D012203DE09C4F3878404504D299
:1071D0008A2001F091F9302034E02846FFF77EF84C
:1071E00001002FD1DFF8DC04DFF8C86700F020FBD6
:1071F0004518307820B90120FFF784F8072021E0F6
:1072000000F026F83178491E317000F01DF88847EB
:10721000B8F11C0FBCBF38781C280ADB4246214657
:10722000284603F003FE01000CD12046F9F7CBFFFE
:1072300007E0102000904B4642462146284604F0C5
:10724000C3F80020BDE8F283DFF8841C09687047AA
:10725000DFF8800C0068004700C0002130B5DFF87F
:107260001C08017883B009B121203EBDDFF8001C65
:10727000DFF8004C0B7B496003F0E00343F085032B
:107280000B7341F60A024B7B0A8003F0F00343F0D4
:1072900002034B73002266238B734A808023CB73D7
:1072A00040F6C412DFF8F83B8A600B614C615A600B
:1072B00001251A7A1D8002F0FE021A722525DA7A5B
:1072C0009D7002F0F002002542F00102DD705D7257
:1072D000DD60DA7225800D220270584CDFF8EC2B4D
:1072E000E068DFF8F43BCDE9002525690835022286
:1072F0002D68A8473EE030B5282983B003DA0500A1
:1073000018BF012D01D012203EBDDFF87047207854
:1073100008B121203EBD480000F6621081B2012074
:1073200004F0BEF8DFF8B41BDFF8AC3B496040F670
:1073300008000880002048808860012D087B00F04C
:107340006000087300F056F80CBF03200A20887311
:107350000022DFF88C0B4861002008828861CDE9AB
:107360000022C87C00F041F8C87402220B2000F013
:1073700048F8A847208100203EBD30B5282883B0BA
:1073800001DB12203EBDDFF8F446217809B121204F
:107390003EBD400000F6621081B2002004F080F88B
:1073A000DFF8401BDFF8303B496040F607000880FB
:1073B0000022002048808860CDE90022087B00F090
